:109C6A00414952434F544543004256332E33342020
:109C7A0048554E00414B4B5500532F4E2146414902
:109C8A004C555245005245454E54455221532F4E8C
:109C9A0000434F4E5441435420414952434F544587
:109CAA004300475053004032444000403344400090
:109CBA004B492021554A20404D454E75000A160051
:109CCA000180000300007E0000FE00001E00003636
:109CDA000003E60001C4000000000FFFE0534154F6
:109CEA005320404B4552455300414C54494043414F
:109CFA004C202023004B455045524E596F00534F7C
:109D0A005252454E44005445524B4550202000546F
:109D1A0045524D494B202000564152494F202020A0
:109D2A00004241524F4752414D005554564E414C04
:109D3A002020004B6F5A454C4920200046504F4E78
:109D4A00544B2020004A454C454B20202000414CD2
:109D5A004150202020002020202141544C21202045
:109D6A0020205441560020545241434B2142452061
:109D7A00200020545241434B214B492020004D41A1
:109D8A00524B004952414E592D46454E54004553B7
:109D9A005A414B2D46454E5400214B494C455020C3
:109DAA0020015554564F4E4056414C014D414720D3
:109DBA004245414C4C2001524550754C45534B6825
:109DCA006901464C4947485420414C4C0146504F82
:109DDA004E544F4B206869015554564F4E414C4BD7
:109DEA006869014C4547544552202068690142453B
:109DFA00414C4C4954206869004D41472042454135
:109E0A004C4C20004241524F404D414720200047D0
:109E1A005053204D4147202000514E4820202020F9
:109E2A00402148504100464C005245504E41504C4A
:109E3A004F207552455320003E214B494C45502036
:109E4A002000214B494C455001564A4154535A016E
:109E5A004B554C44202001544F524F4C2000214B6B
:109E6A00494C4550202001434F4D3A2020202020C4
:109E7A002001544E432031232035374B01544E43A1
:109E8A0020312320392E36010150574340313023E7
:109E9A004035374B01505743403130234031394B1D
:109EAA0001014D5850403130234035374B014D5850
:109EBA00502034232035374B014D58502031232070
:109ECA0035374B014D5850403130234031394B0121
:109EDA004D58502031232031394B002156495353D4
:109EEA005A412001465020554A2020202020014670
:109EFA0050204D4153494B202001465020546F5267
:109F0A004C2020200101434F4D3A0146505420462F
:109F1A004F4741442001465054204B754C44202061
:109F2A00016F535A40465054404B754C01014650FC
:109F3A00544F4B2054415620014D494E4046504003
:109F4A00546F524C0049524E5921544156004D45C6
:109F5A004E542000414B5455414C5340504F5A2EB9
:109F6A00005441524F4C20202020002053544F527D
:109F7A00452157505420002046554C4C2000214082
:109F8A00546F524C455300535A455200495244416A
:109F9A0000555342200055534220004C4953540067
:109FAA004B754C4400204154564954454C492E485F
:109FBA00494241202000214B494C4550202001555F
:109FCA0054564E4C4056414C01554A20465020208A
:0D9FDA002020200155545620535A45524B6B
:109FE7002001464F524449542055545601465020AB
:109FF700546F524C4553200155545620546F524CC0
:10A0070045530143594C2052414449555301434F4D
:10A017004D3A0155545620464F4741442001555467
:10A0270056204B754C442020015052454348454328
:10A037004B005554562156414C20200055404A406C
:10A04700200020554A2040504F5A402100214046C9
:10A057004F52444954204000464F5244495400212E
:10A06700404650544B40544F524C005554564E4066
:10A07700544F524C004E454D2075524553202000F9
:10A087002140555456404B754C44002020524144C2
:10A0970049555300214B494C4550014C45475452B3
:10A0A70040546F4C5421014C45475452404E455A39
:10A0B70020014F53535A214C4721544F520101431A
:10A0C7004F4D3A014C4547545220464F4744014CA7
:10A0D70045475452204B754C44004C454754522039
:10A0E7004E455A202020202020004D4F5A474154EA
:10A0F7002000464F524741534420202000534B41F4
:10A107004C2020582F592020564953535A20005489
:10A11700415620546F524C004155544F2E42452012
:10A12700004155544F2E4B4920002020534B414CA2
:10A137004100544156204B4D2000544156204E4D6E
:10A147002000214B494C4550202001564152494F90
:10A1570020202068690158432D4245414C4C6869CD
:10A16700015645522D4245414C686901414C544CBA
:10A17700414E4F536869014B455045524E596F68E0
:10A1870069010101414C41502D4D4F442001475970
:10A19700415249204245414C015445535A54524576
:10A1A7005020016F535A2152455021546F520021BC
:10A1B7004B494C455020200153754C5948414E4757
:10A1C7000153754C59212D0153754C59404D4F443E
:10A1D7000153754C5940494E56015641522054433C
:10A1E70040202040230148414E4745526F015641C8
:10A1F70052494F204E554C4C0148414E474D41471F
:10A207002001504552494F44555301564152204170
:10A217005640203040230154454320202040303011
:10A2270040250148414E475445535A542000537521
:10A237004C5948414E4700532D48414E47214B4901
:10A24700004E494E4353214455414C005641524913
:10A257004F204E554C4C005641524A203130205029
:10A2670045524349472020004E554C4C415A4153D3
:10A277002020202020202000214B494C4550202021
:10A28700015554564F4E414C20014155544F4345BB
:10A297004E54010141544C2F544156200153494B10
:10A2A7004C204B414C0153535A0101535A454C2101
:10A2B700542D55500143454E5421542D55500157A7
:10A2C700415950542142524700214B494C45502097
:10A2D700200153544152544049446F2001454C5387
:10A2E7006F200144454C54413A2001546F42535A60
:10A2F7006F526F53200155544F4C530143594C53E0
:10A3070049474020204023015554564056414C4C64
:10A31700200101010143594C520143594C21495233
:10A3270046454C00214B494C4550202001014547EB
:10A337005347014B41545440302C402023014B4F8D
:10A347004E5452535A54014E4D4541213138330131
:0DA35700494D502F414750530101432D56F1
:10A364004152494F014D454D4F525944554D5000AE
:10A374004D454D4F525944554D50004046504E5452
:10A38400204C4554455A494B202020400046504F0C
:10A394004E5420202000204B494C455020202100C1
:10A3A400464F474144202000535A414240003C2D2F
:10A3B400204C495354202D3E2020455849540053E5
:10A3C400454C004E455854004B6F562046502020B3
:10A3D40000454C6F5A6F20465000535A4152405426
:10A3E4006F524C006F53535A40546F524C004B49B8
:10A3F40020202020202020202000204B492000471E
:10A4040050532048494241202000205441524F4C8F
:10A41400202020005554564E4C004B4F5A454C4971
:10A42400004C4953544100455445004D4147403088
:10A4340000755245532055545620200054554C4025
:10A44400534F4B20200021404C49534056414C204F
:10A45400002046504056414C4C2120002140464F9C
:10A46400474144202040002020404F4B45402020BD
:10A4740021004F4B45005641520046495800474180
:10A48400544521580053545254564E4C2020200019
:10A49400535443594C2000404B4920005450200051
:10A4A400406A40494E20004067404F5554002020E8
:10A4B4004849424120202100204B494C5000535A26
:10A4C4004552004947454E00554A202020414C4CF6
:10A4D4002020535A45524B004B4F56202020202019
:10A4E40056414C2020204B49005843542D464C499A
:10A4F40047485420005553454400454E5445522086
:10A50400004D4D2E4D4D4D20004D4D2753532E5390
:10A5140000574753213834002040554054404D40A3
:10A524002000554054404D002055544320004C4FCA
:10A5340043414C005357495353474400414C540042
:10A544005355494058004156474020304023003578
:10A554003030003136343000205D203130404B63E0
:10A564002F70005D2020203140632F2300205D20C8
:10A574002035404B5453005D203230304046504D1E
:10A5840000406340204B63004654204B630040630B
:10A5940040204E4D004654204E4D004D2F53003266
:10A5A40030305E003530305E00312200322200331C
:10A5B4002200352200382200464C3700464C313602
:10A5C40000464C333300464C3635004631303000BB
:10A5D400463136300046323630005E252640534F31
:10A5E40047005E25264054415300414C54005641D7
:10A5F4005200225E2F24004B545300532F4E00224E
:10A6040024004B5400225E004E4D00302C350031A6
:10A614002C3000322C3000302C3600312C320032F9
:10A624002C3500332C3800372C35004031350040B0
:10A63400333000403630005441534B00464C2D44D7
:10A6440041544500545000544F4600535441004671
:10A65400494E004C414E00534554204F4646534505
:10A6640054004953412048454947485400415554F2
:10A674004F2D474F20005354415254002043484526
:10A68400434B40414C4C00524144204449535400F4
:10A694004053454C404845494748543A0047505375
:10A6A400404241524F40414C4C0053494E4B403183
:07A6B4002D3221632F23006A
:1064F400304D2475A7049005C2E0F51CE0F51DE0BD
:10650400F51EE0F51FE0F56DE0F56EE0F56FE0F5E2
:10651400541270B6126AF42275C70375C6E475B9CD
:1065240001E5BCB481431270B61256DC8E628F63EF
:106534007568F97569001265CA203C2D203B2B1241
:1065440066FF1266D3856D1C856E1D856F1E85548E
:106554001F126636203C12203243201D231266FF90
:10656400126AF4E532242850DC22126636203CF903
:10657400203DF6203205201DBD80EF301DB880EA95
:106584001266FF126AF4856D1C856E1D856F1E856B
:10659400541F1266E9126AF4203DCE8099126922D2
:1065A400201D0D7553107400126885203DBB808634
:1065B400E553540FC553C4540F20350512679A8010
:1065C40003126885808BC23CD23B126686FD12663C
:1065D40086FC126686C39573F565EC9574F564EDD7
:1065E4009575600504600A800EE56424E05011800E
:1065F40006E56424204009126686126686026686D1
:10660400126686FD126686FC126686C39576F56769
:10661400EC9577F566ED9578600904600122E566EE
:10662400F48002E5668562F0A474E025F04002C2BD
:0D6634003B22C23C126686A2E7923DA2E620
:10664100921DA2E592324026A2E492E592E692E7FB
:10665100FC1266862565F565EC3564F5641266867F
:10666100FC1266862567F567EC3566F56622A2E4BD
:106671009235540F79C6F712668609F7301D051257
:106681006686F55322E5697023E56860302404408D
:106691002CE56875F004A485F0C7F5C675B901E568
:1066A100BCB4811985BD68756902801E54037010E0
:1066B10005C675B901E5BC056953690F22D23C22B3
:1066C100147004E5BD80F0147004E5BE80E9E5BFF7
:1066D10080E575A7009006F6E56DF0A3E56EF0A3E1
:1066E100E56FF0A3E554F02275A7009006F6E0F5FA
:1066F1006DA3E0F56EA3E0F56FA3E0F55422E56428
:10670100B2E7F56D85656EAB67E566FC30E707C3FB
:10671100E49BFBE49CFCAA62A9631253DCE56630AE
:10672100E707C3E49DFDE49EFEEEB2E7F56F8D54ED
:106731002275380C12698B1269D6D553012275382E
:106741000C12695C1269CCD55301227538001269AB
:0E6751007412699BD553012275380012695CE1
:10675F0012699BD553012275380312698B126A0790
:10676F00D553012275380312695C1269FDD55301A7
:10677F002275380F126974126A2CD553012275389D
:10678F000F12695C126A2CD553262290679F2373D0
:10679F008091807780688059804A803B802C801D53
:1067AF00800E80DA80CB80BC80AD809E808F808011
:1067BF0075381512698B126A4ED55301227538152B
:1067CF0012695C126A43D553012275380912697434
:1067DF00126A14D553012275380912695C126A14B2
:1067EF00D553012275380612698B1269BED5530134
:1067FF002275380612695C1269B3D55301227538B8
:10680F00121269741269E4D5530122753812126994
:10681F005C1269E4D553012202673275381512698B
:10682F008B126A4ED553012275380F12695C126AAA
:10683F002CD553012275380F126974126A2CD55357
:10684F00012275380312695C1269FDD55301227557
:10685F00380312698B126A07D5530122753800125B
:10686F00695C12699BD55301227538001269741245
:10687F00699BD553262290688A2373809E80A980B6
:10688F00B480BF80CA80D580E08010801B802680B6
:10689F0031803C80478052805D806875380C12696A
:1068AF005C1269CCD553012275380C12698B1269B1
:0E68BF00D6D553012275381212695C1269E4B5
:1068CD00D55301227538121269741269E4D553013A
:1068DD002275380612695C1269B3D55301227538D9
:1068ED000612698B1269BED55301227538091269DA
:1068FD005C126A14D5530122753809126974126A33
:10690D0014D553012275381512695C126A43D5539B
:10691D00012202682A78C686040886037AED12538E
:10692D009A78CAA60408A60378C686040886037A50
:10693D006212539A78CCA60408A60378C68604087A
:10694D0086037AB512539A78C8A60408A603227551
:10695D001A6A751B0A78CA8618088619126B9F78F1
:10696D00CC86060886072278C88618088619E4F5AD
:10697D001AF51B126B9F78C886060886072278C603
:10698D008618088619751A00751B01026B9FE51D87
:10699D002519F51DE51C3518F51CC3E51F9FF51FC1
:1069AD00E51E9EF51E22C3E51F9FF51FE51E9EF5F4
:1069BD001EC3E51D9519F51DE51C9518F51C22E561
:1069CD001D2FF51DE51C3EF51CC3E51F9519F51F83
:1069DD00E51E9518F51E22C3E51D9FF51DE51C9EB0
:0969ED00F51CC3E51F9519F51F07
:1069F600E51E9518F51E22E51F2FF51FE51E3EF52F
:106A06001EE51D2519F51DE51C3518F51C22C3E5E7
:106A16001D9519F51DE51C9518F51CE51F2FF51F8D
:106A2600E51E3EF51E22E51D2FF51DE51C3EF51C57
:106A3600E51F2519F51FE51E3518F51E22C3E51DB0
:106A46009FF51DE51C9EF51CE51F2519F51FE51E86
:106A56003518F51E22E51A7009E51B70058C068DA2
:106A66000722ED851BF0A4A2F792D5ED851AF0A4B6
:106A7600AEF0FFEC851BF0A4A2D53FEE35F0FF92F9
:106A8600D5EC851AF0A42FFFE435F030D50104FECD
:106A960022E4F51AF51BEF4E7003051B22EF65196C
:106AA6007006EE65187001227808C3EF33FFEE33E7
:106AB600FEEF9519F5F0EE95184003FEAFF0E51AD6
:106AC60033F51AD8E5F4F51A751BFF7805C3EF33CD
:106AD600FFEE33FEEF9519F5F0EE95184003FEAF85
:036AE600F0E51BBD
:106AE90033F51BD8E5F4C403F51B22E51D9511E523
:106AF9001C9510500BE56E9511E56D95105001220E
:106B0900E51F9511E51E9510500BE5549511E56F9C
:106B19009510500122E51D9513E51C9512400BE5D2
:106B29006E9513E56D9512400122E51F9513E51E3B
:106B39009512400BE5549513E56F951240012253C8
:106B49002CF8C3E51F9554FFE51E956FFE92605022
:106B590007C3E49FFFE49EFEC3E56E951DF519E5A5
:106B69006D951CF5189261500BC3E49519F519E45C
:106B79009518F518C3E5199FE5189E9262500AE524
:106B890018CEF518E519CFF519126A97E52C5407AF
:106B990075F003A4F538E538906BA573026BBD0257
:106BA9006BD1026BDF026BF7026C0A026C1D026C7F
:106BB9002B026C43851C16851D17C3E4951FF5151B
:106BC900E4951EF514026C56851C16851D17851E45
:106BD90014851F158077C3E4951DF517E4951CF5F9
:106BE90016C3E4951FF515E4951EF514805FC3E4FB
:056BF900951DF517E4F5
:106BFE00951CF516851E14851F15804CC3E4951F34
:106C0E00F517E4951EF516851C14851D158039851E
:106C1E001E16851F17851C14851D15802BC3E49524
:106C2E001FF517E4951EF516C3E4951DF515E495AD
:106C3E001CF5148013851E16851F17C3E4951DF5CC
:106C4E0015E4951CF5148000C3E5179513E516950C
:106C5E001210D70122E5159513E514951210D701E0
:106C6E0022E519F92517FFE518F83516FED3EF952D
:106C7E0011EE9510500122E5119517FDE5109516B0
:106C8E00FC402A4D6027126A5BE5152FF515E514B9
:106C9E003EF514E5159513E514951210D70122E56E
:106CAE00199DF9E5189CF8851016851117E5172919
:106CBE00FFE51638FEE5139FE5129E500BC3E51354
:106CCE009517F9E5129516F8E51A700AE51B700688
:106CDE00AA00AB018013E9851AF0A4E5F0FBE88564
:106CEE001AF0A42BFBE435F0FAE5152BFBE5143A6C
:066CFE00FAE5119BE51010
:106D04009A10D70122EB9515FDEA9514FCC3E515FD
:106D14009511E514951010D717E5139BE5129A50B9
:106D240036E5139515FFE5129514FE126FD38027EF
:106D3400EB9511FFEA9510FEAA00C001126FD3D0A3
:106D440003E5172BFBE5163AFAEB99F517EA98F5E4
:106D540016851115851014C2D5E5466002D2D5AA50
:106D640056E98AF0A4ABF0E88AF0A42B30D5047578
:106D7400F00384F8700122E5172513FDE51635129A
:106D8400FCED8AF0A4ABF0EC8AF0A42B30D50475AA
:106D9400F00384FEE5152513FDE5143512FCED8A98
:106DA400F0A4ABF0EC8AF0A42B30D50475F0038486
:106DB400F9E538906DBB73026DD3026DDF026DE8A7
:106DC400026DF1026DF7026E03026E0A026E0FC3CA
:106DD400743E9EFFC3743E99FE8032C3743E9EFF90
:106DE400AE018029AF06C3743E99FE8020AF06AE83
:0D6DF40001801AC3743E9EFEC3743E99FFD9
:106E0100800EC3743E99FF8007C3743E9EFEAF019E
:106E110008EF2437FFE51B7007E51A700CE8800EB8
:106E2100A2E7E51A50030460F488F0A4E5F06001DC
:106E310004F923FA98FBC3E998C333F9906E43E54B
:106E41003873026E5B026E88026EBD026EEA026FDB
:106E510017026F44026F71026F9E05A7800BEB3022
:106E6100E7032A8002291E1FFBEEC45403F583EEBB
:106E71005408C42FF582EE5407243883F5F0E04519
:106E8100F0F0D8DA05A72205A7800BEB30E7032A3B
:106E91008002290E1FFBEEC45403F583EE5408C48F
:106EA1002FF582EE5407240B83F5F0E045F0F0D87E
:106EB100DA05A722804020100804020105A7800BF3
:106EC100EB30E7032A8002291E0FFBEEC45403F5C1
:106ED10083EE5408C42FF582EE540724EC83F5F0B9
:106EE100E045F0F0D8DA05A72205A7800BEB30E7E3
:056EF100032A800229C4
:106EF6000E0FFBEEC45403F583EE5408C42FF5823F
:106F0600EE540724BF83F5F0E045F0F0D8DA05A784
:106F16002205A7800BEB30E7032A8002291F1EFB00
:106F2600EEC45403F583EE5408C42FF582EE5407DD
:106F3600249283F5F0E045F0F0D8DA05A72205A7FC
:106F4600800BEB30E7032A8002291F0EFBEEC454A8
:106F560003F583EE5408C42FF582EE5407246583A7
:106F6600F5F0E045F0F0D8DA05A72205A7800BEB8F
:106F760030E7032A8002290F1EFBEEC45403F58373
:106F8600EE5408C42FF582EE5407243883F5F0E05A
:106F960045F0F0D8DA05A72205A7800BEB30E7030A
:106FA6002A8002290F0EFBEEC45403F583EE540823
:106FB600C42FF582EE5407240B83F5F0E045F0F07C
:106FC600D8DA05A7228040201008040201EC701FC1
:086FD600ED20E740D2E023CFDB
:106FDE0023CF30E7F980357B08801A7B1080167B33
:106FEE002080127B40800E20E4ED20E3EE20E2EFC5
:106FFE0020E1F07B80EE8BF0A4CF8BF0A4E5F02F98
:10700E00FFEC8BF0A4CD8BF0A4E5F02D2499838FAB
:10701E00F0A433E5F033FBE98BF0A4E5F0C88BF078
:10702E00A428F9E435F0F822FFFEFCFAF8F6F4F2A3
:10703E00F0EFEDEBEAE8E6E5E3E1E0DEDDDBDAD901
:10704E00D7D6D4D3D2D0CFCECCCBCAC9C7C6C5C45F
:10705E00C3C1C0BFBEBDBCBBBAB9B8B7B6B5B4B379
:10706E00B2B1B0AFAEADACABAAA9A8A8A7A6A5A465
:10707E00A3A3A2A1A09F9F9E9D9C9C9B9A99999829
:10708E009797969594949392929190908F8F8E8DD0
:10709E008D8C8C8B8A8A898988878786868585845C
:1070AE00848383828281818075A7009070DCE5469F
:1070BE00FA24FA50027A05EA2323F978107F049312
:1070CE00F60809E9DFF99070F4EA93F556227FC2CB
:1070DE00803E7F4680BA7E8C81747D1882E87A303D
:1070EE0085D074608BA08080402010081271000241
:1070FE007356D215D274D273C219C23A1256DC8E9E
:10710E0047757D0075460575520212914612022191
:10711E00E53524EB500E1291467F1990A11612768A
:10712E00F012DD51E55275F016A4F57012730C7560
:10713E007E151271D77F237E0990A0F1127702126D
:10714E00DD5110000810010D10021280E212727F44
:10715E0075330180DA1272C475330180D2757E00E8
:10716E001271D77E0090A1041277357F237E059091
:10717E00A0F912770212722812DD51E55210000F9B
:10718E0010010510028780D5045403F55280CE12EB
:10719E0071D77F237E0B90A133127702E5466007ED
:1071AE001460041412411A12DD51E5461000081045
:1071BE00010B10021180D860D6154680D2B405029C
:1071CE0080CD054680C902711B75320012DF277F04
:1071DE00017E1190A0E11277357E0012D5E8E57E92
:1071EE00D26612D63F75170812DA721241597571AE
:1071FE0000C20612D78F741BFFF5177E0F90A139B0
:10720E00305D0390A141127735129189125D0D12F6
:10721E0046BFC20612651C021E03E55260141460BE
:10722E001E1460297F647E2D791C1272721E1FD966
:10723E00F9227F6A7E1F79281272721FD9FA227F75
:10724E00487E2D791C1272720F1ED9F9227F567E3E
:10725E003379281F12DE6C0F0F12DE6C1F12DE6CDC
:10726E001ED9F0221E12DE6C0E0E12DE6C1E02DE17
:10727E006CE552605514606814606D800075709EE8
:10728E001272F98003757000E5732540F573E435CD
:10729E0074F574E43575F575227570161272968054
:1072AE000375702DE5762542F576E5773541F57750
:1072BE00E43578F57822E55260CB1460DC1460E199
:1072CE0080007570441272B2800375705AE5739522
:0972DE0040F573E5749400F574A9
:1072E700E5759400F575227570711272DB80037570
:1072F7007088E5769542F576E5779541F577E578F7
:107307009400F57822E54690732293F540FEAD4749
:10731700E4FFFC12546F8E418F4222020C1830603A
:10732700C07F40120E9E121E1912DD511275D1EB4D
:107337007005909E3B800B1273DF90A46B500390F7
:10734700A4B27F3F7E0412770212DD5112DE3212A1
:10735700DE6275370990A09B121CFF90736673025B
:1073670002930275260270FA0276020273560273BE
:107377007E0273970273287F2E12168680D17F367E
:107387007E0490A44012770212DD5112DE3280BFD4
:107397007F37120E9E121E1912DD511275B5124853
:1073A7004FD2AC1000A9306DFA12748F203BCF403A
:1073B700ED7568F97516001274DC40FB1276787F5C
:1073C700367E29E51612D3C812DD5105161277A8A5
:1073D70078C6B6F7E20275AF7C0512484F12DC6B30
:1073E700744112DC7C745312DC39EB12DC5A1277CD
:1073F700BA5003DCE5227515F975160010000EE585
:1074070015602512743140051274585002D3227F3B
:107417003F7E29E51612D3C812DD517F1412DE49CB
:107427000516E51664F870D4C322127D7075B9018C
:10743700E5BCB4811AE5BDF51570037516F778C676
:0B744700A616127EB9127EB1127EB1B3
:10745200C3027EB1D3227F0575F019D5E0FDD5F0C8
:10746200FA12484F12DC6B744112DC7C744212DC5B
:10747200397E0F78C6E60812DC39DEF912DC5D12BD
:1074820077BA400122DF012275F00080CEC23B12A2
:10749200484FD2AC12DBC4204C3CB440F712DBC9DB
:1074A200B4400312DBC9B4412DF53812DBC9B45321
:1074B2002512DBC9FA12DBC9E538701A12DBC9B42E
:1074C2000D1412DBC9B40A0EC3E5169A4003027703
:1074D2009FC2ACD23B22C2ACD3221277FE12484FDB
:1074E200D2AC1000F112DBC4204CEBB440F412DB3E
:1074F200C9B4400312DBC9B441DCF53812DBC9B4AC
:1075020042D47E1078C612DBC9F608DEF9E538707F
:10751200C512DBC9B40DBF12DBC9B40AB9C2ACC310
:10752200220273567F0A120E9E121E1912DD51128A
:1075320075B5124868D2AC1000E712DBC9B440F549
:10754200F53812DBC9B46EED12DBC9E538600A12F8
:107552004868744F12DC4580DC124868744012DCC3
:107562007CE51612DC4512DC4F7568F975160012BF
:107572004868D2AC10003912DBC9B440F7F53812B2
:10758200DBC9B44EC07E1078C612DBC9F608DEF93C
:10759200124868E5386007744F12DC4580D11276D4
:1075A200780516745112DC4578C6B6F7C212761504
:0C75B200027356751500751603127D67F4
:1075BE0075B901E5BC30E70205160515E515242061
:1075CE0050EB227B007515F9127D7075B901E5BC83
:1075DE00B481010B0515E515240450EC7515011247
:1075EE007D6775B901E5BCB481010B0515E5152460
:1075FE002050EC227F1C120E9E121E5C400675154A
:10760E00F9127615027356E51560372404401A24D4
:10761E001E5019E515240740028027127D70127640
:10762E00510515E515240450F2751501127D677587
:10763E00B901E5BC30E7031276510515E515242096
:10764E0050EA22127666124EE605C6124EE605C6C0
:10765E00124EE605C6024EE674FF800574048001E4
:10766E00E4F5BCF5BDF5BEF5BF22E568606AF5151B
:10767E000515E5152404501D751501127D6775B9A4
:10768E0001E5BC30E70280190515E515242050EB05
:10769E00751500800C241C60F750E0E5152406508B
:1076AE0037E56875F004A485F0C7F5C675BC81E5AD
:1076BE0015F5BDF56878C6B6F70375BD00081276E8
:1076CE00DB1276D51276D586BC0886BD0886BE0836
:0976DE0086BF08124EE605C62223
:10C09A0012AED612C19912828112C11E128289125F
:10C0AA00C12B02AEDA12AED612C1991282817F5A20
:10C0BA00C23C12816312835F783F79437F607EEAD4
:10C0CA0012C18D1282897F6512816312835F783D66
:10C0DA0079417F207E4E12C18D303C2012C34F120F
:10C0EA00C1AA783F794312C109783D794112C10941
:10C0FA0012C34F78D7E65480F675370002935BC3B4
:10C10A00E796FF1819E796FE0809C3E69FF718197C
:10C11A00E69EF7227F5B7E0690A5441277351F8044
:10C12A000A7F667E14745912D4E11F127FEC7E399D
:10C13A00E402D5007866E620E73418C3E69472086C
:10C14A00E694045029C318E6941F08E69404401E96
:10C15A007869E620E71818C3E6940E08E6940150B9
:10C16A000DC318E6947508E694004002D322C32250
:10C17A00E67D0030E7011D08E62BFB18E63CFCE4EF
:0EC18A003DFD22C3EB9FF6F71819EC9EF6F769
:10C198002212C13E400CE47842F608F67840F608D0
:10C1A800F6227864C3E6946AF55708E6944CF55687
:10C1B8000808C3E69458F55B08E694AEF55A753955
:10C1C80000AC56AD57EC12B283784C12B311AC5A8E
:10C1D800AD5BEC12B283785012B3117F2B7E867D53
:10C1E800777C1812B248785012B30512B15412B2C3
:10C1F80048785012B30512B15412B248785012B3AD
:10C208000512B15412B2487F367E847D257C6412B3
:10C21800B248785012B30512B15412B248784C1291
:10C22800B30512B15412B2487F3F7EA27D607C8B69
:10C2380012B248785012B30512B15412AF4212AF7D
:10C248004212B31D7F3F7E807D057CE6053912B121
:10C2580054784812B3117F2C7E937D477C7F12B2AD
:10C2680048785012B30512B15412B248785012B33C
:10C278000512B15412B248784C12B30512B15412D7
:10C28800B2487F357EB47DF87CDF12B24878501210
:10C29800B30512B15412B248785012B30512B15412
:10C2A80012B2487F3F7EED7D227CCD12B248784C99
:10C2B80012B30512B15412AF4612AF42784412B30A
:10C2C800117F317E397D9D7CE712B248784C12B3DC
:10C2D8000512B15412B248784C12B30512B1541277
:04C2E800B24878449C
:10C2EC0012B30512AF4612B2487F2C7E377D0C7C00
:10C2FC00A312B248784C12B30512B15412B248785A
:10C30C004C12B30512B15412B248784C12B3051248
:10C31C00B15412AF4612B31D7F3F7E807D027C9FCD
:10C32C00053912B154784412B311784812B305127E
:10C33C00B2BA8E428F43784412B30512B2BA8E4011
:10C34C008F4122753900AC42AD43EC12B283784870
:10C35C0012B311AC40AD41EC12B283784412B3115C
:10C36C007F2B7E537D507C0912B248784812B3055E
:10C37C0012B15412B248784812B30512B15412B229
:10C38C0048784412B30512B15412B2487F347EF28D
:10C39C007DCD7CA312B248784812B30512B1541269
:10C3AC00B248784812B30512B15412B2487F3F7E9E
:10C3BC000A7D2E7CAE12B248784412B30512B154E9
:10C3CC0012AF4212AF42784C12B3117F2B7E4F7DCD
:10C3DC00AF7CB212B248784812B30512B15412B203
:10C3EC0048784812B30512B15412B248784812B3C7
:10C3FC000512B15412B2487F357EB17D4B7C95123B
:10C40C00B248784812B30512B15412B248784412AB
:10C41C00B30512B15412B2487F3F7E497DCD7C45A5
:10C42C0012B248784812B30512B15412AF4612AF8B
:10C43C0042785012B311784C12B30512B2BA8D5522
:10C44C008E568F57785012B30512B2BA8D598E5A38
:04C45C008F5B786416
:10C46000E557246AF608E556344CF608E5553404D9
:10C47000F608E55B2458F608E55A34AEF608E435CC
:03C4800059F62248
:1091A90012AED612983A12AEDA7F6690A5261277D9
:1091B900331292177F5A78C41291F31291FB78C631
:1091C9001291F31291DE7F6578C81291F31291FB27
:1091D90078CA1291F37E2DE51B12D5007E33E51A6C
:1091E90012D5007E39E51902D500860408860302E6
:1091F90053397E15E51C12D5007E1BE51B12D500DF
:109209007E21E51A12D5007E27E51902D5007F5A7D
:109219007E01E53A12D4167E0B909C2EE53B930213
:10922900D513E6FF08E6FE08E6FD339217E4500180
:10923900F4FC12B32E75130A75390112B52C78D7BF
:10924900E6C2E775F00A84F9303D02A9F012B32E9F
:109259008913053912B50530170A053912B51805EC
:109269003912B518A80302B31112AED612983AC230
:109279003C7F5A7E0312851012921712DD5110009D
:109289000810011510022080EFE53A146004153A20
:109299008003753A3CD23C80DFE53AB43C05753A27
:1092A9000180F2053A80EE7E0312850B7E0B128552
:1092B9001012921712DD511000081001151002202A
:1092C90080EFE53BB40205753B158002153BD23CA6
:1092D90080DFE53BB41505753B0280F2053B80EE66
:1092E9007E0B12850B7F5A78C41291F31291FB12EF
:0792F900936412836F78C437
:109300001293BC78C61291F31291DE129396751CDB
:109310000012836F78C61293BC7F6578C81291F3F0
:109320001291FB12936412836F78C81293BC78CAAF
:109330001291F31291DE129396751C0012836F78CE
:10934000CA1293BC303C14E53B24F4500B78C9E6B8
:109350002410F618E63427F61293C212AEDA127E03
:10936000F102DD51C2247E15E51C128460F51CD289
:10937000247E1BE51B128460F51B1023E77E21E58C
:109380001A128460F51A1023E67E27E5191284600C
:10939000F5191023E822C2247E2DE51B128460F506
:1093A0001BD2247E33E51A128460F51A1023E77E5F
:1093B00039E519128460F5191023E622ECF608EB62
:1093C000F622129C4678C8E6FE0886073395E0FD33
:1093D000FC12B2487FE87E037D007C0012B52C129F
:1093E000B24878CAE6FE0886073395E0FDFC12B560
:1093F0000512B2487F807E697D677CFF12B505EC5F
:1094000012B27F12B2487F3F7E807D0D7C1D12B16B
:109410005412B2487F3D7E407D007C0012B24878F5
:10942000BC12B30512B15412B2487F3E7E807D005B
:109430007C0012AF4612B24878BC12B30512B15488
:0994400012B2487F3F7E807D00DE
:109449007C0012AF4212B24878B412B30512B1547B
:1094590012B1CC783C12B3117F407E807D007C0034
:1094690012B248783C12B30512B15412B3AB12B21E
:10947900487F3F7EA87D007C0012B24878B812B3BD
:109489000512B15412B15412B2487F407E007D00DA
:109499007C0012B248783C12B30512B15412B3AB36
:1094A90012B2487F3F7EC07D007C0012B15412AFDA
:1094B9004612B24878B812B30512B15412B24878BC
:1094C9003C12B30512AF46785412B31112B3957812
:1094D9005812B31112B24812B15412B24878C012DC
:1094E900B30512B154784412B311785412B305126A
:1094F900B3AB783C12B31112B24812B15412B2484C
:1095090078BC12B30512B154783C12B3117F3E7E78
:10951900C07D007C0012B248783C12B30512B154E8
:1095290012B2487F3F7E007D007C0012AF4612B226
:1095390048783C12B30512B15412B2487F3F7E807D
:109549007D007C0012AF4612B24878B412B30512FE
:10955900B154787012B31178C4E6FE0886073395C2
:10956900E0FDFC12B2487FE87E037D007C0012B565
:109579002C12B24878C6E6FE0886073395E0FDFC52
:1095890012B50512B2487FE07E5E7DF87CFF12B508
:1095990005EC12B27F12B2487F3F7E7F7DE57CC920
:0595A90012B2487870C9
:1095AE0012B30512B15412B1CC785012B3117F3FE1
:1095BE007EF07D007C0012B248783C12B30512B1E9
:1095CE005412B2487F3F7EC07D007C0012AF46121F
:1095DE00B248783C12B30512B15412B2487F3F7EA6
:1095EE00807D007C0012AF46783C12B31178BC121D
:1095FE00B30512B2487F3F7E807D007C0012AF42E1
:10960E0012B248783C12B30512B24878B412B305C0
:10961E0012B15412B154784012B311785412B305EA
:10962E0012B3E3783C12B31112B24812B1547874EB
:10963E0012B3117F417E107D007C0012B24878C0BB
:10964E0012B30512B15412B2487F407E807D007C69
:10965E000012B248784412B30512B15412B2487FC8
:10966E00417E207D007C0012AF4212B24878441237
:10967E00B30512B15412B2487F407E407D007C008B
:10968E0012B248787412B30512B15412B2487F4028
:10969E007EA07D007C0012AF4612AF4612AF421282
:1096AE00B248785012B30512B15412B24878501223
:1096BE00B30512B15412B2487F3D7E2A7DAA7CAB0F
:1096CE0012B15412B2487F3F7E007D007C0012AF73
:1096DE004212B248783C12B30512B248787012B3F7
:1096EE000512B15412B248784012B30512B1CC1221
:1096FE00B248785012B30512B15412B248785012D3
:10970E00B30512B15412B15412B248785412B305C3
:0C971E0012AF4212B2487F4A7E517DD249
:10972A007CCB12B15412B2BA78AC12B3117F407E1C
:10973A00007D007C0012B248787412B30512B1544D
:10974A0012B2487F3F7E807D007C0012AF4612B283
:10975A0048784412B30512AF4612B248785012B391
:10976A000512B15412B248785012B30512B154120C
:10977A00B248785012B30512B15412B2487F3E7EF5
:10978A002A7DAA7CAB12B15412B248785012B305A2
:10979A0012AF4212B248785812B30512B1CC12B2C3
:1097AA00487F4A7E517DD27CCB12B15412B2BA1292
:1097BA00B248AF3AEF3395E0FEFDFC12B2487F4063
:1097CA007E7E7D057C0012B52C12B2487F607E75C4
:1097DA007D587CFF12B50512B50578B012B3117821
:1097EA00AC751B641298118F1C78B0751B671298A0
:1097FA0011E51C75F00AA42FFF249C50027F007803
:10980A00D7E654802FF62275390012B30512B248F2
:10981A007F0A7E007D007C0012B5D8A81BE513F6EE
:10982A0008E512F608E511F6335004EFF404FF22B6
:10983A00C23D78647BAC12922BD23D78677BB01222
:10984A00922B129C467F007EE47D577C0012B24820
:10985A0078AC12B30512B50512B2487F007E537D6B
:0E986A00077C0012B5D812B26785133B7F80D1
:109878007ECB7DA47C0012B24878B012B30512B535
:109888000512B2487F407E7E7D057C0012B5D81255
:10989800B267E513F56F04F53A85126E85116D858B
:1098A800106C7F407E7E7D057C0012B248786C1279
:1098B800B30512B52C12B2487F607E0C7DA27C00E5
:1098C80012B24878B012B30512B50512B518786C03
:1098D80012B31178AC12B305EC12B27F12B2487F02
:1098E800347E9C7D2B7C5F12B154785412B31112D4
:1098F800B395785012B311786C12B305EC12B27F9D
:1099080012B2487F347E9C7D2B7C5F12B15412B218
:1099180048785012B30512B154784012B3117F4001
:109928007E007D007C0012B248785412B30512B153
:109938005412B3AB12B2487F3D7EC07D007C00124A
:10994800B24878BC12B30512B15412B2487F3E7EB9
:10995800C07D007C0012AF4612B24878BC12B30535
:1099680012B15412B15412B2487F3D7E407D007C42
:109978000012B24878BC12B30512B15412B2487F33
:109988003E7E807D007C0012AF4612B24878BC1241
:10999800B30512B15412B2487F3F7E807D007C002F
:1099A80012AF4212B248785412B30512B15412AF32
:1099B8004212B2487F407E807D007C0012B2487817
:1099C8005412B30512B15412B3AB12B2487F3D7EA4
:1099D800707D007C0012B24878BC12B30512B154F5
:1099E80012B24878BC12B30512B15412B15412AF76
:1099F8004612B24878B412B30512B154785812B36B
:109A080011785412B30512B3AB783C12B3117854E1
:109A180012B30512B3E3785412B311783C12B305AC
:109A280012B24812B15412B24878BC12B30512B13E
:109A380054783C12B3117F3E7EC07D007C0012B288
:109A480048783C12B30512B15412B2487F3F7E00E9
:109A58007D007C0012AF4612B248783C12B3051262
:109A6800B15412B2487F3F7E807D007C0012AF4621
:109A780012B24878B412B30512B154787012B31107
:109A8800785012B30512B24812B15412B24878C0D5
:109A980012B30512B154784412B311785412B305B5
:109AA80012B24812B154787412B311784012B30547
:109AB80012B24812B154783C12B3117F407E807DB7
:109AC800007C0012B248784412B30512B15412B2A5
:109AD800487F417E107D007C0012AF4612B2487864
:109AE8004412B30512B15412B248787412B3051275
:109AF800B2487F407EA07D007C0012AF4212AF4684
:109B080012B248783C12B30512B15412B2487F3DE4
:109B18007E2A7DAA7CAB12B15412B2487F3F7E00E8
:109B28007D007C0012AF4612B248785412B3051279
:109B3800B248787012B30512B15412B248783C1288
:109B4800B30512B15412B15412B248785812B30581
:109B580012AF4612B2487F3F7E7F7DE57CC912B1C5
:019B680054A8
:109B690012B2487F4B7E187D967C8012AF4612B2A6
:109B7900BA12B2487FE87E037D007C0012B5D81284
:109B8900B26778C8A61208A61308A60608A6077819
:109B99007412B30512B2487F3F7E807D007C0012AB
:109BA900AF4212B248784412B30512AF4612B24816
:109BB9007F3E7E2A7DAA7CAB12B15412B24878400E
:109BC90012B30512B15412B248783C12B30512B15E
:109BD9005412B248784012B30512AF4612B2487F08
:109BE9003F7E7F7DE57CC912B248787012B30512B9
:109BF900B15412B15412B2487F487EF47D247C00DE
:109C090012AF4612B2BA12B2487FE87E037D007CD9
:109C19000012B5D812B26778C4A61208A61308A60E
:109C29000608A607223F3F4344454647484A4B4C4E
:109C39004D4E5051525354555657583F3FE4F539FC
:109C4900F5A7909C5A791078B4E493F6A308D9F94A
:109C59002232A5C24A4A19DC3A885CDB3BFFD6DCD2
:019C69003BBF
:10AED600D2D58002C2D575A70490040078107F0BE6
:10AEE60012AF0278267F0512AF02783C7F2212AF9E
:10AEF60002786A7F0F12AF0275A7002230D506E6E8
:10AF0600F008DFFB22E0F608DFFB22D2D58002C282
:10AF1600D575A7049006FA78737F0612AF0275A757
:10AF26000022DA0CD902800BD906303701B350055E
:10AF360002B0B5923702B0A1D9F680F9D2368002B6
:10AF4600C23612B0E6303606C86002B237C892364C
:10AF5600DAD0D9E4B8000A12B12DA236923702B07F
:10AF66008A60FBB51300400F12B12DA23692F7A2EC
:10AF7600379236A2F79237C398F40424E740DF24C9
:10AF860019AD29AC28AB277A00C394084008CDCC6C
:10AF9600CBCAE4CD80F424086010F9C3ED13FDECB0
:10AFA60013FCEB13FBEA13FAD9F1A236303701B3DF
:10AFB60040308A17E5102BF518E5113CF519E51216
:10AFC6003DF51A501A13F51AE51913F519E5181374
:10AFD600F518E51713F5170513E5137002051402A6
:03AFE600B040E494
:10AFE900C39AF517E5109BF518E5119CF519E512BB
:10AFF9009DF51A500DB237C378177F04E496F60809
:10B00900DFFA7A047019E513C39408F51350021591
:10B0190014E4C517C518C519F51ADAE802B0E12014
:10B02900E7BAE5137002151415137817C37F04E600
:10B0390033F608DFFA80E8E51A20E7137817C37FAB
:10B0490004E633F608DFFAE513700215141513E563
:10B05900173378187F03E63400F6500E08DFF775CA
:10B069001A800513E51370020514E51420E75470DE
:10B0790027E513604E046020851A12851911851879
:10B08900105326F0AC10AD11A237E51313FFE512EA
:10B0990092E7FEA81302B267E4F512F511F510F56F
:10B0A900147513FF5326F043260580D8E5FFF512E2
:10B0B900F511F510751400F513D2375326F0432610
:10B0C9000980C15326F0432603E4F512F511F51062
:10B0D900F514F513C23780AC5326F080EC79017A68
:10B0E900018512F0E513A2F7339237751400F513B1
:10B0F9006002D2F785F012A813B8FF0809E512C259
:01B10900E75E
:10B10A006001098C278D288EF0A2F7EF3304700AAC
:10B11A000AC2F705F00AD5F0011A146002D2F785BF
:10B12A00F02922C88813C512C529C512C511C52818
:10B13A00C511C510C527C51022DA03B8000302B02D
:10B14A00B5D9028002D9F702B0A112B0E6303701B0
:10B15A00B392377004D9E78005DADEB8000302B08B
:10B16A00E1D9E2C3947E500215142513F513500257
:10B17A0005147815760008B81BFA78277915E608B9
:10B18A00FAE8FC78108AF0E608A427F709E5F03710
:10B19A00F7500989F00907E760FBA9F0B813E61927
:10B1AA0019ECF8B82AD802B04002B0CCB8FFFA02BB
:10B1BA00B0B5D9FB02B0A1DAF6B800F002B0E112DC
:10B1CA00B31D12B0E6303701B392377007D9E3B82E
:10B1DA0000E280DBDAE1B8000280E1D9D5C8C39881
:10B1EA0050021514247F50020514F513781A7600BC
:10B1FA007A1A7B80C3E5109527E5119528E5129503
:10B20A00294016C3E5109527F510E5119528F51183
:09B21A00E5129529F512E64BF648
:10B22300DA0302B040EB03FB30E703187600C3E513
:10B233001033F510E51133F511E51233F51240CA59
:10B2430030E7DD80B6E53905396010D0F0D0E0C0D5
:10B2530010C011C012C013C0E0C0F08F138E128D46
:10B26300118C1022E539146010D0F0D0E0D013D047
:10B2730012D011D010C0E0C0F01539227920800C13
:10B283007910800479087D007E007F003392D550C9
:10B293000312B2F7EC33400FEF33FFEE33FEED331F
:10B2A300FDEC33FCD9EE22EECCF5F0747E29A2D569
:10B2B30013FF92F7AEF022EF8EF0A2F7D2F733929C
:10B2C300D5C3947F5006E4FFFEFDFC229420400486
:10B2D30074FF80F304CCFEE4FFFAE5F0CC6012C304
:10B2E300CC13CCCD13CDCE13CECF13CF0450EEDA87
:10B2F300EC30D5D7C3E49FFFE49EFEE49DFDE49CC0
:03B30300FC22E643
:10B30600FC08E6FD08E6FE08E6FF22ECF608EDF688
:10B3160008EEF608EFF622CFC513CFCEC512CECD76
:10B32600C511CDCCC510CC22E4F513F512F511F5F7
:10B336001022E493FCA3E493FDA3E493FEA3E49319
:10B34600FFA322C0E012B24812B15412B37C12B36A
:10B3560038D0E0C0E012B24812B37312B15412B240
:10B366004812B33812AF46D0E0D5E0E722AC48AD7C
:10B3760049AE4AAF4B228C488D498E4A8F4B227478
:10B38600FF7809FFFEFDFCE52654F048F52622125B
:10B39600B43C04A2E1927F1420E01590B4BD74047D
:10B3A60012B349802912B43C30E102B27F20E0EBAF
:10B3B6008C4C8D4D8E4E8F4F90B4D1740412B34980
:10B3C60012B248AC4CAD4DAE4EAF4F12B154307FB9
:10B3D60004EF6480FFEE33EF337001FF2212B43CBA
:10B3E600C0E08C4C8D4D8E4E8F4F90B4F574031289
:10B3F600B34912B248AC4CAD4DAE4EAF4F12B1543C
:01B40600EC59
:10B40700C54CFCEDC54DFDEEC54EFEEFC54FFF909B
:10B41700B4E5740312B349D08212B248AC4CAD4DB7
:10B42700AE4EAF4FE58230E00712B1CCB27F809DC0
:10B4370012B1C98098EE33EF3324605007D0E0D0C3
:10B44700E002B385EFA2E7547F927FFF12B2487CF8
:10B45700837DF97E227F3E12B154EE33EF33248190
:10B46700501012B24812B2BA12B27FEFB2E7FF120F
:10B47700AF46EE33EF33602A2403F8C313FFEE928F
:10B48700E7FEE82481E4501A12B24812B2BAEF0478
:10B49700C2E0FCF58212B287EFB2E7FF12AF46E5D2
:10B4A7008203FAEE33EF33600B148FF0A2F713FF2A
:10B4B700EE92E7FEEA2283FA703AE4E9AABCF8E0E2
:10B4C700813EE6E99DBF0000803F1A3C2839666946
:10B4D70099BBE335A33DE75D25BFDB0FC93FCCDB58
:10B4E7008D41EE3649C43F91C9453DF8B0C50000CE
:10B4F700803F34F517C373FA2F45DDFD0AC6EF25E4
:10B5070013FFEE3512FEED3511FDEC3510FC02B2DE
:10B5170067C3EF9513FFEE9512FEED9511FDEC95C0
:10B5270010FC02B267EFF88513F0A4FFE513C5F02E
:0AB53700CEF9A42EFEE435F0CDFAA3
:10B5410088F0E512A42EFEED35F0FDE433CC851331
:10B55100F0A42CFCE5128AF0A42CFCE51189F0A4DE
:10B561002CFCE51088F0A42CFC89F0E512A42DFD3B
:10B57100EC35F0FCE51188F0A42DFDEC35F0FC8AEA
:10B58100F0E513A42DFDEC35F0FC02B267E4CCF834
:10B59100E4CDF9E4CEFAE4CFFB75F020C3E5133333
:10B5A100F513E51233F512E51133F511E51033F515
:10B5B10010EF33FFEE33FEED33FDEC33FCEF9BEE8A
:10B5C1009AED99EC98400CFCEF9BFFEE9AFEED99F9
:10B5D100FD0513D5F0C622C2D5EC30E705B2D51270
:10B5E100B2F7E51030E70DB2D512B5FB12B58E12E8
:10B5F100B2F7800312B58E30D515C3E49513F51358
:10B60100E49512F512E49511F511E49510F5102267
:10A6BB00E57124885002D2191256DC8E4712D2262D
:10A6CB00129189125A98305E0F125A3612887812EC
:10A6DB00596712C02C12425412393A1247FB1036EA
:10A6EB0029201F1C301219E412A84112A85612A9D6
:10A6FB005612A97830510302AA0212ACD320510989
:10A70B00C251E4F552F545F5442275A70075830750
:10A71B00E559C454F0F582E0F538A3E0F518A3A38E
:10A72B00A3E0F51E74FF12A8411256DC8E1C8F1B82
:10A73B007510DF751100E51164B4700612A80C7565
:10A74B00111012A7D94028AE1CAF1B125764203230
:10A75B001EAC03AB027A0C125371ED701275A7008D
:10A76B00758304851182ECF00583E510F00511D596
:10A77B0010C412A80C75C70375C6E075A704900525
:10A78B00007F0412A7C7DFFB75A700122B83125A99
:10A79B0036E4F5A7F8F559758307E8C4F582E0654B
:10A7AB00387011A3E06518700BA3A3A3E0651E70AE
:10A7BB000388592208C3E5589850DC22E0F5BCE029
:10A7CB00F5BDE0F5BEE0F5BF124EE605C622E5107D
:10A7DB0075F004A4F5C685F0C775B901E5BC334027
:0BA7EB001F05C605C675B90185BE64D8
:10A7F60085BF6505C675B90185BC6685BD6785BE1D
:10A806006885BF69C322E51124FE502E75A7007F17
:10A8160010AE111E7583048E82E0FD1582E0CDB563
:10A8260005005012F00582CDF00583E0FD1582E0AB
:10A83600CDF00582CDF0DEDCDFD72275A75490047B
:10A846000005A79005007FB4F0F0DFFC75A7002295
:10A8560012BE80C2517B077AFFE4FFF5A790040081
:10A8660012A93CED244C4035EC603075A7008D8272
:10A8760005A712A9027583058D82E02410401CF0FD
:10A8860005A7E02CF0500505A7E004F0BA000CBBC4
:10A896000009D251EF24DC50027F23DFC3EA6005B2
:10A8A60012A8B58006EB600312A8ED75A70022304A
:10A8B600E0047553082230E1047553182230E2048F
:10A8C6007553282230E3047553382230E404755357
:10A8D600482230E5047553582230E6047553682241
:10A8E60030E7037553782230E0047553882230E14F
:10A8F600047553982230E2037553AA22ED54F0C42E
:10A90600232390A90C735302FE225302FD22530205
:06A91600FB225302F722B0
:10A91C005302EF225302DF225302BF2253027F2243
:10A92C005303FE225303FD225303FB225303FB224A
:10A93C0012BDB812BC46E4F5F7C2B2C2B2ADF7F51F
:10A94C00F7C2B2C2B2ACF7D2B22290050078B4E032
:10A95C006015FD54F0C4CD7C00540FFE1583E0FF50
:10A96C0012546FEFF005830582D8E42275830478C6
:10A97C00FF088882E060FAF5D38812E512244C5067
:10A98C00012285D3D288D4881279FF0512E5126092
:10A99C00F00908E875F0B484A8F08882E060ECF562
:10A9AC00D3B9000280D5B9230050D0C395D292D12F
:10A9BC005002F40409FEE4FFFCAD0112547C740156
:10A9CC00FA25D475F0B484A8F0AC06AB0712536327
:10A9DC00EB30E7010CE5D22C30D1029C9C8882F044
:10A9EC000AEAB501DCE512244C50012285D3D2854C
:10A9FC0012D4A812809390040012AAC18C068B0565
:10AA0C0012AAC1E4FFF512F5118C148B13C3ED9B44
:0EAA1C00F9EE9CFA4012E51199E5129A500AE3
:10AA2A008C148B138A1289118F528F82E0F9C3ED2D
:10AA3A0099FDEE9400FEE582245A5002244C75F0EA
:10AA4A00B48485F082E0FA2DFDEE3400FEEB9AFB29
:10AA5A00EC9400FCE92BFBEC3400FC0FBFB4B0E52E
:10AA6A005224D3400224B4F552C3E51333FBE51450
:10AA7A0033FCE511FE2BFBE512FF3CFC1254D1E935
:10AA8A00F890AAD393F511FDEBF513FFECF514FE3C
:10AA9A007C0012546F8F44E890ABD393FAAB13AC9B
:10AAAA001412539AAF03AE04AD117C0012546FEF27
:10AABA007002F552F545227C007B007F5AE02BFBA1
:10AACA00EC3400FC0582DFF522B4B4B4B4B4B4B4F7
:10AADA00B4B4B4B4B4B4B4B4B4B4B4B3B3B3B3B331
:10AAEA00B3B3B3B3B3B3B3B3B2B2B2B2B2B2B2B234
:10AAFA00B2B1B1B1B1B1B1B1B0B0B0B0B0B0B0AF44
:10AB0A00AFAFAFAFAEAEAEAEAEAEADADADADADAC5E
:10AB1A00ACACACACABABABABAAAAAAAAA9A9A9A983
:10AB2A00A9A8A8A8A8A7A7A7A7A6A6A6A5A5A5A5B0
:10AB3A00A4A4A4A4A3A3A3A2A2A2A2A1A1A1A0A0E7
:10AB4A00A0A09F9F9F9E9E9E9D9D9D9D9C9C9C9B21
:10AB5A009B9B9A9A9A999999999898989797979660
:10AB6A0096969595959494949393939292929191A3
:10AB7A0091919090908F8F8F8E8E8E8D8D8D8C8CE3
:10AB8A008C8B8B8B8A8A8A89898988888887878728
:10AB9A00868686858585848484838383828282816E
:10ABAA0081818080807F7F7F7E7E7E7E7D7D7D7CB1
:10ABBA007C7C7B7B7B7A7A7A7979797878787777F3
:10ABCA00777676767575757474000203050608093A
:10ABDA000B0C0E101113141617191A1C1D1F212203
:10ABEA00242527282A2B2D2E303133343637393A6B
:10ABFA003C3D3F404243454648494B4C4E4F5052DC
:10AC0A0053555658595A5C5D5F606163646667685C
:10AC1A006A6B6C6E6F707273747677787A7B7C7EEF
:10AC2A007F80818384858688898A8B8D8E8F909197
:10AC3A00929495969798999B9C9D9E9FA0A1A2A459
:10AC4A00A5A6A7A8A9AAABACADAEAFB0B1B2B3B432
:10AC5A00B5B6B7B8B9BABBBCBDBEBFC0C0C1C2C326
:10AC6A00C4C5C6C7C7C8C9CACBCCCCCDCECFD0D035
:10AC7A00D1D2D3D4D4D5D6D7D7D8D9DADADBDCDC5B
:10AC8A00DDDEDEDFE0E0E1E2E2E3E4E4E5E5E6E79B
:10AC9A00E7E8E8E9EAEAEBEBECECEDEEEEEFEFF0F1
:10ACAA00F0F1F1F2F2F3F3F4F4F4F5F5F6F6F7F75E
:10ACBA00F8F8F8F9F9FAFAFAFBFBFBFCFCFDFDFDE2
:10ACCA00FEFEFEFEFFFFFFFFFFC251E4F544F8144B
:10ACDA00FB900400A9007C0FC2D112ADEEE8240556
:10ACEA00F8B8B4F08B13E5122403FA244C5001FA95
:10ACFA00BBFF012275112C8A1912AE258F16203D31
:10AD0A0012AA1975112312AE258F15751600303D3A
:10AD1A00E2801175112312ADCD751500303D05E89D
:01AD2A002FF9
:10AD2B0013F51575111212ADCD751400303D05E8F4
:10AD3B002F13F514EA2404F552244C5002F552E477
:10AD4B00F51AF51BF51CE516600AFB7A00AF137EAE
:10AD5B00FF12AD93E515600AFB7A4FAF137EFF121E
:10AD6B00AD93E516600DFB7A00E5146006FF7ECF10
:10AD7B0012AD93AE1CAF1B7C00AD1A12546F8F45F6
:10AD8B00EF2513F544D25122EFF5F0A4FCADF0EB17
:10AD9B00F5F0A49CFCE5F09DFDEB8AF0A4FAABF07A
:10ADAB00EF8EF0A49AF8E5F09BF9E833F8E933F964
:10ADBB007B00125515051AE51B2BF51BE4351CF50D
:10ADCB001C22EA2511F9244C5001F9C2D112ADEC29
:10ADDB00303D428F00C3EA9511F9500324B4F9D2E8
:10ADEB00D17C09E4FDFEFF8982E060062FFFE43E83
:10ADFB00FE0D09B9B4027900DCEDED20D118F51E7A
:10AE0B0024FE923D500F12547CEFB5030050068583
:10AE1B001E1FFB881222F51D80E612ADCD203D438F
:10AE2B00740212AEC412ADCD203D38740412AECCF8
:10AE3B0012ADCD203D2D740612AEC412ADCD203D0A
:10AE4B0022740812AECC12ADCD203D17740A12AE8F
:10AE5B00C412ADCD203D0C740C12AECC12ADCD2076
:10AE6B003D0122C3E89F605088148F158A16400855
:10AE7B001ABAFF0A7AB380060ABAB4027A0012AD84
:10AE8B00CD303D34C3E89FF9602EC3E5149515FB17
:10AE9B006930E7D4E930E703F404F9EB30E702F467
:10AEAB0004C3995002AA16E5142515C82F28FFE4F0
:10AEBB00FC33FE7D0412546F222AFA244C5001FA03
:0BAECB0022C3CA9AFA500324B4FA22F2
:10BC0D00758000C2B212DE47D2B275F8302275804F
:10BC1D0000C2B2F5F7C2B2C2B2D2B222758000C272
:10BC2D00B2F5F7C2B2C2B2856CF7C2B2C2B2856BC1
:10BC3D00F7C2B2C2B2856AF722758000C2B275F73B
:10BC4D0003C2B2C2B2856FF7C2B2C2B2856EF7C27D
:10BC5D00B2C2B2856DF72212BC9D740612BC1B7464
:10BC6D000212BC298FF7C2B2C2B2D2B222909F6B20
:10BC7D007F631276F012DD51D214120E9412766E8D
:10BC8D00124EE612BC9D740612BC1B74C712BC1B6F
:10BC9D0012BCA340FB22758000C2B275F705C2B27B
:10BCAD00C2B2C2B2C2B275F705C2B2C2B2C2B2C29C
:10BCBD00B2E5F7D2B2A2E022120E9485BF6C85BE1A
:10BCCD006B756A00E56B7015E56A701112BC9D7499
:10BCDD000612BC1B74D812BC29D2B2D21F22E54B5E
:10BCED000475F03C8485F04B12BFA8852E72E55F7C
:10BCFD00030354C0F8E55E543F28F57C305501220E
:10BD0D0012BD4212BCA340F7E54C60F312BC9D126C
:10BD1D00BD5912BD2780F112BC9DC21F740612BC05
:10BD2D001B740212BC29787086F708B880FAD2B25B
:10BD3D0012BD76808F787075A704758304E54CC4A9
:0CBD4D00F5827F10E6F0DFFC054C801949
:10BD5900787075A704758304154CE54C30E701E448
:10BD6900C4F5827F10E0F6DFFC75A7002274102568
:10BD79006A54F0F56AE4356BF56BE4356C540FF5EC
:10BD89006C22E54B75F010A4256A54F0F56AE5F0CC
:10BD990080E4E56A24F054F0F56AE56B34FFF56B4D
:10BDA900E56C34FF80D7E56A24FF80ECC380EBE5BE
:10BDB9006D24F054F0F56DE56E34FFF56EE56F34E2
:10BDC900FF540FF56F2212BE2712BE4FC22DC25467
:10BDD900C255E57F7002D255147002D254E54A303B
:10BDE900E00122B4061C20540D12BD9B12BEF712AD
:10BDF900BF8712BFBF2212852F7E0412DE3F754A0C
:10BE0900012220550D12BD7612BF6612BFA812BEBF
:10BE1900D02212852F7E0412DE3F754A0522740353
:10BE290012BC297870E4F5F7C2B2C2B2A6F708B815
:10BE390080F3D2B222740312BC29E4F5F7C2B2C26C
:10BE4900B2E5F7D2B222E575F8541F30E40244E0B6
:10BE5900F57585722EA2779226E57C543F30E5026E
:10BE690044C0F55EE57C54C02323F55FE57FC2E756
:10BE790079BCF709A77E22856C6F856B6E856A6D23
:01BE89002296
:10BE8A00856F6C856E6B856D6A22E4FEFF7407759B
:10BE9A00A704F5838E8274FFF0DFFD75A700227474
:10BEAA00067E007FB012BE99E4F55AF55B2275A7AB
:10BEBA0004758306E55A600A75F00A84E5F0700293
:10BECA00740AC4F58222307720E55A24024002051A
:10BEDA005A12BEB8E55AF0E573F0E574F0E575F06C
:10BEEA00E576F0E577F0E578F075A700223077F986
:10BEFA0012BEB87F1074FFF0DFFDE55A24F5500337
:10BF0A0012BF22155AE55AB4FF02055AC3E55A95DB
:10BF1A005B50D6755B0080D112BE807F0A056D0525
:10BF2A006D12BC46E4F5F7C2B2C2B2E5F7D2B2303E
:10BF3A00E704DF02800512BDB880E2056D12BC4637
:10BF4A0012BEB8E55A24F6F07F06E4F5F7C2B2C28B
:10BF5A00B2E5F7F0DFF4D2B275A70022053FE53F5C
:10BF6A00B43C17753F00053EE53EB43C0D753E00F6
:10BF7A00053DE53DB41803753D00024ABB153FE592
:10BF8A003FB4FF17753F3B153EE53EB4FF0D753EC6
:10BF9A003B153DE53DB4FF03753D17024ABB05421B
:10BFAA00E542B43C0F7542000541E541B43C0575D4
:0CBFBA0041000540221542E542B4FF0F93
:10BFC60075423B1541E541B4FF0575413B154022DD
:10BFD600AC40AB41A842EC75F03CA42BFBE435F039
:10BFE600FC7A3C125363EB28FBE43CFC22AC3DABF1
:10BFF6003EA83F80E178AE8604AB3EE53FC313F82A
:10C00600800C7800120E5DE5BE75F005A4FBE5BF59
:10C0160075F03CA42BFBE435F0FC7A1E125363EB5F
:10C0260028FBE43CFC2212C008AE04AD0312BFFBA1
:10C036008C148B13120E67E5BFFF24F650027F01A6
:10C04600E5BE75F096A4AAF0F9C3ED9513FBEE953F
:10C0560014FC924E4B701120110E30480B75364B66
:10C066003003037536FFD22E304E02DF1F7A0212DE
:10C07600536375A7009004EEECF0A3EBF0C3E5BFA5
:10C086009F04BF0102D2E79005CBF022ED29FDEE19
:04C096003AFE80B539
:10DE2C0012DE3512DE3512DE357E0480067E02806F
:10DE3C00027E017F0080087F6480027F017E00EFFC
:10DE4C004E6012E4FD0D1D0DEDC394AD40F7EF1FB8
:10DE5C0070ED1E80EA22753500C200C201C202229A
:10DF1300F5D8D2DCE5F520E7FBE5DA540FFEAFD9FF
:04DF230075D800228B
:10DB1A007F767E06909C7E127702740412DF137C55
:10DB2A00007D5212546FEFF875F00A84C0F07F76C8
:10DB3A007E2312D5007E29742E12D5137E2ED0E0B4
:10DB4A0012D5007E35745612D5137F6B7E1190DB89
:10DB5A008312D53FE824E04001220423F824E75049
:10DB6A0002781812DB73D8FB227F6CE82411FE7945
:10DB7A000512DE6C0E0FD9F922071DFFFFFFE080A8
:10DB8A00000020C0000038E0000008F0000038F86B
:07DB9A00000020FFFFFFE087
:10DBA10012DBC930E6022409540F75F00AA4F515F9
:10DBB10012DBC930E6022409540F25152212DBC9F4
:10DBC100540F2275F000800875F044800375F0074A
:10DBD100E4206D09D5E0FAD5F0F7D24C229247C284
:10DBE100ACE54F623885504FA26E926D859950C257
:10DBF1006FD2ACC24CA2472212DC03C4FA12DC037E
:10DC01002A2212DBC920E603540F225407240922D9
:10DC1100E612DC1818E608FAC412DC1EEA540F44B6
:10DC210030F924C6E950112407800D75F00A84C02B
:10DC3100F012DC37D0E0443030530975F00085E054
:10DC4100E0D5F0FA3099FDC299F599623822E538AC
:10DC510080F2E53812DC18800812DC39E53812DC74
:10DC610039740D12DC39740A80CE744012DC3974B7
:10DC71004080C5742C80C1742E80BD75380080B879
:10DF390085A0835383FE438380858384F0758400A1
:01DF490022B5
:10D9C80074A212DF3974A112DF3974A612DF397418
:10D9D800A412DF3974C012DF39742512DF3912DA64
:10D9E8005875C70375C6FC75B90112B611740812CB
:10D9F800DF13EE75F020A4FEEF54F80303032E2482
:10DA080092C313FE24EA50027E16EE90DA41932563
:10DA1800BCFE24E6501F24E8401B748112DF39EE57
:10DA280012DF3912DA65744012DF39742F12DF39C8
:10DA380074AF02DF397E2680E1F7F7F8F8F9FAFBD0
:10DA4800FCFDFEFF000000000101020202030303C7
:10DA5800A8BCA9BDAABEABBFACC7ADC62288BC894D
:0ADA6800BD8ABE8BBF8CC78DC6229D
:10DD5100C006C007C5F075A7019000007EB7E58C2D
:10DD6100240340FA12DD731EBEAFF3C5F0D007D015
:10DD7100062275A700EE12DF39741012DF39740420
:10DD810012DF3985A08343838185838475A7517F01
:10DD910020E0F0E0F0E0F0E0F0DFF6E4F5A7F58454
:01DDA100225F
:10DF270075A711900000E4C583F0C58330E2F8F5CA
:02DF3700A7221F
:10DE6C00EF20E723EE20E71F20E61C05A7C4540390
:10DE7C00F583EE5408C42FF582EE5407240983F57C
:10DE8C00F0E045F0F005A7228040201008040201C4
:10DE9C00EF20E723EE20E71F20E61C05A7C4540360
:10DEAC00F583EE5408C42FF582EE5407240983F54C
:10DEBC00F0E055F0F005A7227FBFDFEFF7FBFDFE8A
:10D4C000FDA42582F582E5F03583F583ED22906099
:10D4D000AC7A0475F00512D4C07D05805E7A0580B3
:10D4E000027A04547FC0E0C083C082C394205001FC
:10D4F000E490605C12D4D3802E9061BA7A058005E6
:10D500009062777A0675F00712D4C07D07802C7A76
:10D510000580027A06C0E0C083C082C39420500117
:10D52000E490620712D505D082D083D0E022905FCC
:10D53000D075F00A12D4C07D0A7A07C2D18002D217
:10D54000D1C0A7C082C083C007C006C0E030D109E7
:10D5500075A704E493FDE493FAEEFB75A704EBFED4
:10D56000EAFC7901D9067908E493F5D4E5D423F5EA
:10D57000D420E01612DE9C0EDCEA0FDDE1D0E0D014
:10D5800006D007D083D082D0A72212DE6C80E8902C
:10D590005F1075F00E12D4C07D0E7A0812D53B9044
:10D5A0005FB875F00212D4C0E493FDE4A393FACE01
:10D5B0002408CE7C0812D5BC7C06AD02ED23FD20EC
:0ED5C000E00712DE9C0FDCF42212DE6C80F716
:10D3AB00F5D2C2D58036F5D2D2D58030F5D224F65F
:10D3BB0050090E0E24A650030E0E0EE5D2F5D275B3
:10D3CB00F0648485F0D3C2D57009D2D5742012D500
:10D3DB0013800312D500CE2406CEE5D375F00A8454
:10D3EB0085F0D3700A30D507742012D51380031241
:10D3FB00D500CE2406CEE5D312D500E5D222F5D248
:10D40B0075F0648485F0D3C2D58022F5D2C2D58065
:10D41B0025F5D2D2D5801FF5D275F0648485F0D373
:10D42B00C2D57009D2D5742012D513800312D4F94A
:10D43B00CE2405CEE5D375F00A8485F0D3700A307F
:10D44B00D507742012D513800312D4F9CE2405CE40
:10D45B00E5D312D4F9E5D222F5D2C2D58035F5D277
:10D46B00D2D5802F30E70DF404C0E0742D12D4E137
:10D47B000E0ED0E0F5D275F0648485F0D3C2D57072
:10D48B0009D2D5742012D4E1800312D4CECE240459
:10D49B00CEE5D375F00A8485F0D3700A30D50774C6
:10D4AB002012D4E1800312D4CECE2404CEE5D312C5
:05D4BB00D4CEE5D222F1
:1076E700909F6B1276F002DD517E00800E7405FECE
:1076F700F51EE4FFF51DF51F203C3375A700E49345
:10770700700122A3B40204051D8003B4010A051FFA
:10771700EF2409FFAE1E80E612D5137D06B44002A2
:107727007D03B421027D02EE2DFE80D27E0075A777
:1077370000E493700122A3B40204051D8003B40181
:107747000F051FEF2407FFAE1E80E612D4DD800869
:10775700B45B0050F612D4E10EB4210280D30EB40C
:10776700400280CDB42C0280C80E0EB45F0280C1E7
:10777700B45B0040BC0E0E80B8E60812D513EE24A9
:1077870006FED513F422909CAC307409909CB0305F
:107797007303909CB502770275F019D5E0FDD5F01B
:1077A700FA12484F12DC6B744F12DC7C744B12DCFC
:1077B7005AC322C2501277FE12484FD2AC12DBC412
:1077C700304C1212DBC4304C0C12DBC4304C06D2E6
:1077D70050C2ACD322B440E512DBC9B4400312DB7C
:1077E700C9B44FED12DBC9B44BE712DBC912DBC9D1
:1077F70012DBC9C2ACC32230530975F008D5E0FDCE
:10780700D5F0FA227F0575F019D5E0FDD5F0FA120B
:10781700484F12DC6B745712DC7C745012DC3974DD
:097827008112DC39E56312DC3941
:10783000E56212DC3978D0E612DC3908B8D7F8E610
:10784000F8795F30E702792FE912DC3912DC39125E
:10785000DC3912DC39745812DC39744312DC39E437
:1078600012DC39E8C2E775F00A84C425F012DC396D
:107870007864E612DC3908B869F8E612DC5A127747
:10788000BA400122DF02800A20508B75F000808010
:10789000D250C2ACD3221277FEC25012484FD2ACA3
:1078A0002002EF12DBC4204CE7B440F412DBC9B471
:1078B000400312DBC9B457DAF53812DBC9B450D231
:1078C00012DBC912DBC9F56312DBC9F56278D0128D
:1078D000DBC9F924A0500353015FE924E040027999
:1078E0005FA60108B8D8E8780612DBC9D8FB12DB1E
:1078F000C9FC53040FC4540F75F00AA42CFC249C3B
:1079000050027C0078D78601E4B92F02D2E72CF62A
:10791000786412DBC9F608B86AF812DBC9E538608A
:107920000302789212DBC912DBC9C2ACC32290A356
:107930007F8003909FAF7F2012773312DD5102DEEC
:107940003D753400C26B1279FD12DE3D127DADE54E
:1079500016600312795902025912800F121E461244
:10796000DD5110002010010280F8127E1850131211
:107970001E5112792E10000D10010280F8121DF315
:0579800080D7127B9D81
:1079850022C26BD22775480A122B77753400127EF6
:10799500E5C26A1233CF106A0512024A80ED12025F
:1079A5004A127D3F127E97127EF178D0E6642660FA
:1079B5004412800F121E4612DD51100038100102CC
:1079C50080F8127E18501BE965156018121E5112B9
:1079D500792E12DE3510001D10010280F8121DF3FC
:1079E50080BCD26B127EC3751607855917122BF012
:1079F5007535008096020259127DAD127A1F127EEE
:107A0500F17F19127A3990A3AC7E121277357E2355
:107A1500E51602D47F90A4F980EF7862E4127A30FB
:107A250078D0745F127A3018E4F6227F08F608DF02
:107A3500FC227F7B7E007810742012D4E1CE2404D2
:107A4500FED8F5227F197E081277357E28909F9102
:107A5500305303909F96027735C26B127A1F127AC4
:107A650069020259C251127EF190A3A4127A4912F9
:107A75001E19127DAD7F20127A0812DD51E51670B0
:107A85000512DE32803675A6FF3051031277A81233
:107A9500484FD2AC200025306DFA127899400C126F
:107AA5007E184011127B9DD25180BB105003127974
:107AB50033C25180D1D25112792E80CAC2AC22D2A2
:107AC5002775480A122B77753400C26B127EE5C202
:107AD5006A1233CF106A0512024A80EB12024A126B
:0D7AE5007D3F127E97127EF1127AF550DA85
:107AF200020259909FAA127A49121E2B12DD51C31B
:107B020010001310010510020E80F412780B4001D0
:107B12002212793380DDD3C2AC22D227C26B7548E0
:107B22000A122B77753400127EE5C26A1233CF1027
:107B32006A0512024A80EDD26B127D3F127E9712C5
:107B42007D6775B901E5BCB2E7F5BC124EE6751664
:107B520007855917122BF080CB127DADE516601FF9
:107B620078D0E53D127B8EE53E127B8EE53F127B9F
:107B72008E765A08765F12C844127EC3027D7E7FDB
:107B82003E7E11909F8112770202DD5175F00A84C8
:107B92004430F608E5F04430F60822D26B127EC378
:107BA200127D7EE51775F01084240AF54824E8500A
:107BB2000375480A122B838558592275320012BE6A
:107BC2009475A704900700751500127D6775B901B9
:107BD200E5BC20E705E515F0801004600D648260C5
:107BE2000975BCFF75B90575B9020515E51524209F
:107BF20050D8E58224FE4003027C96A882187F00BA
:107C020075A7007583078882E0FE75F004A4127DD3
:107C120012A9BCAABDABBEACBF1582E0FD75F004D3
:107C2200A4127D12C3E995BC404C7052EA95BD4046
:0D7C320045704BEB95BE403E7044EC95BF95
:107C3F004037703DEE75F004A404127D12A9BCAA62
:107C4F00BDABBEACBFED75F004A404127D12C3E949
:107C5F0095BC4015701BEA95BD400E7014EB95BE98
:107C6F004007700DEC95BF5008EEF00582EDF01552
:107C7F0082E5826009C3EF95825003027C0A0FC32D
:107C8F00E89F4003027C0275A70490070075C703A5
:107C9F0075C6A8E0F5BCE0F5BDE0F5BEE0F5BF7533
:107CAF00B90575B90205C6E58224204006E5C6244C
:107CBF002050E00875C70375C68075B901E5BC1281
:107CCF007CFCF5BCE5BD127CFCF5BDE5BE127CFC71
:107CDF00F5BEE5BF127CFCF5BF75B90205C6E5C65A
:107CEF00245850D6E5320470FB75A70022B4FF016B
:107CFF0022F975A704900700E582686005E06970B6
:107D0F00F7E922F5C685F0C775B901E5BC645F7068
:107D1F000375BC27E5BD645F700375BD27E5BE64C1
:107D2F005F700375BE27E5BF645F700375BF2722C1
:107D3F0075C703E54875F004A42480F5C6E55975A9
:107D4F00F00484A8F00825C6F5C675B901A9BCAA28
:077D5F00BDABBEACBF8615F1
:107D660022E515242050037515DFE51575F004A4EA
:107D760054FCF5C685F0C722E51724204028E517F0
:107D860075F00484A8F00824A8F5C675C70375B96C
:107D960001A9BCAABDABBEACBFA61589BC8ABD8B6A
:107DA600BE8CBF124EE622E4F516F51579FF127D5C
:107DB6006775B901E5BCB4FF040516A9150515E5F7
:107DC60015242050E9891579FF75C70375C6A8756E
:107DD600B90109E5BC04601B09E5BD04601509E5A8
:107DE600BE04600F09E5BF04600905C6E5C6242088
:107DF60050DD09891722751600751501127D677504
:107E0600B901E5BC20E70205160515E51524205045
:107E1600EB227900E975F004A454FCF5C685F0C799
:107E260075B901E5BC20E73078D066702B08E5BD52
:107E360066702508E5BE66701F08E5BF6670190501
:107E4600C675B90108E5BC66700E08E5BD66700822
:107E560008E5BE667002D32209E9242050B6C32283
:107E6600127E86127E6EA8017F08E0F608DFFB22EE
:0B7E7600127E86127E7EA8017F08E6C7
:107E8100F008DFFB2278D0796275A704758307EBD0
:107E9100C454F0F58222127D6778D0127EB1E5BC20
:107EA100F9C23C20E702D23C127EB17862127EB167
:107EB10075B901A6BC08A6BD08A6BE08A6BF0805DF
:107EC100C622127D6778D0127ED3127ED3786212D9
:107ED1007ED386BC0886BD0886BE0886BF08124EC2
:107EE100E605C622125A3612DF2712866E02DD51CE
:107EF10012DF277F007E0990A3911277027F0A7E0D
:107F010012E5150412D3B77F1412CA2E121DF37F86
:107F1100277E0875130778D0127780E6793E30E71F
:107F210002792F7E34E912D5137F3D7E0190A5158C
:107F310012773520311B3030031291A9C23B1281D7
:107F4100A1127F57D23B1281A1127F691281E88071
:107F51007C12C09A80E6C23B7F447453201702749E
:107F61004E7E0012D5138017D23B7F4F74572017D6
:107F71000274457E0012D5137E06E51E12D5007EE1
:107F81000CE51D12D5007E12E51C12D5007E17747A
:107F91008112D5137E1CE51B12D5007E22E51A1233
:107FA100D5007E28742E302602742712D5137E2D1B
:107FB100E51912D5007E33E51812D5007E39302639
:0F7FC10007742C12D50F7E3BE53702D500742DC7
:107FD000201702742B7F707E1512D513127FEC7E52
:107FE0003A12D3607E0190A5400277027E1BE51C09
:107FF00012D5007E21E51B12D5007E27E51A12D589
:10800000007E2DE51912D5007E33E51802D5001249
:10801000808D1280B812838F127EF11283E72017B1
:108020001E10021B1248F012C844128075121DFE69
:108030007F347E2F12778D127F2A12DD5180E2125B
:108040001DF3203026203128C23B1281A11280CDA1
:1080500078661282A1D23B1281A11280E278691265
:1080600082A11281E812815C02834412927280F232
:1080700012C0AF80EDE57D75F01084AAF075F00AAE
:10808000A42A547FFA78D7E654802AF6227F277EE6
:108090000879D08700C001D224B9D002C22412844A
:1080A0006ED001A70010230909EE2406FEB9D7E31C
:1080B0002219EE24FAFE80DB7E3479D7E7A2E7921C
:1080C0001712841B79D7E7A21792E7F722C224C2BE
:1080D0003B751E007F447E0012842B801E1023ED12
:1080E000802AD23BC2247F4F7E00128433D2247E6A
:1080F00006E51E128460F51E1023E7D2247E0CE5EF
:108100001D128460F51D303BD41023E1D2247E1271
:10811000E51C128460F51C1023E17E1CE51B128413
:0381200060F51BEC
:108123001023E67E22E51A128460F51A1023E87EF6
:108133002DE519128460F5191023E87E33E5181232
:108143008460F5181023E87E393026027E3BE5373C
:10815300128460F5371023E3227F707E1512842387
:10816300C2247E1BE51C128460F51CD2247E21E50B
:108173001B128460F51B1023E77E27E51A12846027
:10818300F51A1023E67E2DE519128460F5191023E4
:10819300E87E33E518128460F5181023E82278D7B7
:1081A300E6C2E775F00A847866F537303B057869EF
:1081B30085F03712821130262BE53775F003A404BE
:1081C3000475F00584FBE51975F00AA4251875F00C
:1081D30006A42BFBE435F0FC125585F537125585C3
:1081E300F5188B1922E563FC339217AB6250031227
:1081F30055F6305C0A7AD21253717840125513AE99
:1082030004AF037C277D1012547C8F1C8037E6FD5E
:1082130033921718860418860350031255FE7A0901
:10822300792778C01255108B1EADD3ACD2AB06792B
:10823300EA786012550E8B1DAF06AED27C177D70A7
:1082430012547C8F1CAF05AE047C037DE812547C72
:0F8253008F1BAF05AE047C007D6412547C8F1A24
:10826200ED75F00A84F51985F01822EC3392175057
:10827200031255F6751D30301786751D2D808178D5
:10828200427B607CEA800678407B207C4E12C17A79
:108292007927781012550E8B1CAF06AED280AB3008
:1082A200262AE51975F00AA4251875F00AA42537BF
:1082B200FBE435F0FC7A051253638C068B077C00D5
:1082C2007D0312546F8E048F031281DBE51E75F05D
:1082D2000AA4251D75F00AA4251C75F006A4251B09
:1082E200FBE435F0FC7A0A125363EB251AFBE43CFB
:1082F200FC7A0A125371EB2519FBE43CFCE43DFDC8
:108302007A0A125383EB2518FBE43CFCE43DFD3072
:1083120017031255FEA60518A60418A60378D7E679
:10832200A2E7923DC2E775F00A84FCABF0303B0E47
:10833200AB37EC75F00AA42BA23D92E7F622AC37DC
:1083420080F012835F305C0A7A4012537178D21245
:1083520055133017031255F68C638B622212836F0A
:108362007A0A125363EB2518FBE43CFC22E51C75E8
:08837200F00AA4251B75F00AB6
:10837A00A4251AFBE435F0FC7A0A125363EB25199B
:10838A00FBE43CFC221283C112DE39C202C2231270
:10839A0083C110000810010510021B80F51031ED91
:1083AA0010300D102604D22680E3D230C23180DD8F
:1083BA00D231C23080D7227F3590A4FE1277339013
:1083CA00A51C20300F90A53820310990A50D202634
:1083DA000390A5051F7E1712770202DD517F357EB5
:1083EA0001909F5E1277357F347E3A128510744E63
:1083FA0012D51312DD5112DE39C2027F347E3AD20F
:10840A001775115975124E802675112E751227800F
:10841A001E75113E75122F801675112B75122D803F
:10842A000E75114E75125380067511457512571245
:10843A008510E511301702E51212D51312DD51101D
:10844A00000810010510020B80F5D23C1017E3D288
:10845A001780DF02850B4430F812846AE8540F2231
:10846A00C2218002D221A22492229223128510E8EC
:10847A0030E709D23C7430302102745FF812D51308
:10848A0012DD5110003410010510025D80F5D23C56
:10849A00102266102367B43909745F2021DF743013
:1084AA0080DBB45F04742D80D4B42D04744180CD74
:1084BA00B45A04743080C60480C3D23C30240610F7
:0F84CA002237102338B44104742D80B1B42D042F
:1084D900745F80AAB45F04743980A3B43009745AF4
:1084E90020219B74398097148094B48908D223E899
:1084F90012D513800DF8C223800874898001E8021F
:1085090084879085258003908521C007EF2408FF83
:1085190012D53FD00702DD510205F8F80205000027
:10DCF10075A70090DD2375F02D84C2D5C2D16017C0
:10DD0100D2D1146007D2D514600DC2D1E5F093FCD5
:10DD1100742D95F093FB22E5F093FB742D95F09310
:10DD2100FC220009121B242C353E474F58606870B5
:10DD31007880888F969DA4ABB2B8BEC4CACFD4D91F
:10DD4100DEE2E6EAEDF0F3F6F8FAFCFDFEFFFFFF96
:10DDEB00D23D8002C23DED8BF0A430E70205F0C3BB
:10DDFB00E895F020D50425F025F0FEED8CF0A4304D
:10DE0B00E70205F0C3E995F030D10425F025F0FFCA
:10DE1B00203D0B2487500122EF24CC40012202DE4F
:01DE2B006C8A
:10D78F00203A7A7E1C7F5312DE6C7F5912DE6C1E9C
:10D79F007F5712DE6C7F5512DE6C7E2312DE6C7F9C
:10D7AF005712DE6C1E7F5912DE6C7F5312DE6C1F18
:10D7BF007E2012DE6C7F5A12DE6C7E1E12DE6C7FB4
:10D7CF005212DE6C120E67E5BD20E0143006117F99
:10D7DF00357E1C90D84BE571700390D85502D53F1C
:10D7EF00E5716018E57012DCF1781F79567D09122A
:10D7FF00DDEF303A0312D81E0DBD16F3227E1C7FCB
:10D80F005390D83412D53F200CD612CA8A80C0C08C
:10D81F00060E30D5021E1E12DE6CD0061F30D1024E
:10D82F000F0F02DE6C070700386C446C38000505DB
:10D83F002070D8702005057088A8887008071038E8
:10D84F007CFE383838000807102844C628283800CE
:10C8690090A54A7F717E23127735120E67E5BC7E4B
:10C879003112D4CE30121AC23C120E67E5BCFB75D8
:10C88900F00AA4F904FAC23D12BE8012CB07303D6A
:10C899000122DAF712CA0E7C00EBF4042E4019AD1E
:10C8A9000312546FEFA2D1203C077E237F6502D18A
:10C8B9002DAE16AF1702C9AFAD0112546FEF12D2E8
:10C8C9001B203C077E237F6502D151AE16AF1702AC
:10C8D900C9D37F567E0512CA3A7F3D12CA4D7F6F72
:10C8E90012CA4D12CA8A7E0A7F4112CABD7E227FB0
:10C8F9005912CABD2012012212BE80857A1D855E99
:10C909001C857B1B855F1A7AC0C23D12CB03203D73
:10C919005212CA0E7C007D1412546F74562F20D106
:10C92900029F9FFF24CB40028037EF24885002806A
:10C9390030EA1475F00384FE12DE6CC3E51B957BA7
:10C94900FEE51A955F92D55004EEF404FEEEC3138A
:10C95900FE24E0400C741F2E30D5029E9EFE12DE8E
:10C969006CDAA8227F5212C97F7F5A12C97F7517C4
:10C9790053751600802B7E0012DE9C0EBE12F92222
:10C989007F157E28742012D5137F1C7E2812DE9C09
:04C999000EBE40F995
:10C99D00223012E712C98975171575162DD23C0272
:10C9AD00C882C23D6002D23D92D175F080305C04E8
:10C9BD00F5F08001A4A2E792D5E5F075F03284F888
:10C9CD00E5F075F00584C0E0E5F0A2D533C0E0E8F0
:10C9DD00601E12D500EE2406FED0E0F8D0E012D590
:10C9ED0000EE2406FE742C12D5130E0EE802D500AF
:10C9FD007420303D07742B20D102742D12D5138075
:10CA0D00D4C3ED957AFFEC955EFE92D1500312558D
:10CA1D00E6227F1512CA267F327E3E12DE6CDEFBC9
:10CA2D00227E0912DE6C0EBE36F9227E0112DE6CFC
:10CA3D000E0EBE3FF8227E3312DE6C0EBE40F92282
:10CA4D007E047D1112DE6C0E0E0EDDF81F1F7E357D
:10CA5D0090A553305C057E3190A55702773574054E
:10CA6D00305C097E32740112D4CE74067E3612D437
:10CA7D00CE7E3A740012D4CE7E3D02D4CE7F417E5E
:10CA8D001F7D0F12DE6C0F0F0FDDF8227F687D0307
:10CA9D0080047F677D0512DE6C0FDDFA227F667DD7
:10CAAD000780F37E1F7F5012DE6C1F1FBF3EF822E2
:07CABD007D0A12DE6C0E0E73
:10CAC4000F0FDDF722203D07123C767003D23D2282
:10CAD400056D12BC46E4F5F7C2B2C2B2ABF7F5F786
:10CAE400C2B2C2B2E5F7FA30E411EB251DF51DE43C
:10CAF400351CF51C0519EA30E3010ED2B280157815
:10CB04000380027801203D07123C767003D23D2257
:10CB1400D8F3056DE56D2409F56D12BC46E4F5F70F
:10CB2400C2B2C2B2ADF7F5F7C2B2C2B285F71BF515
:10CB3400F7C2B2C2B2E5F7FCD2B2543F30E50244C8
:0FCB4400C0CC54C02323F51AE56D24F6F56D22FD
:10D6B6007E017F0990D73412D53F2051097E037F22
:10D6C60000743F02D513E4FEFFC3E54512CF85FD86
:10D6D600940AED403D9464ED4002746312D3B17E2A
:10D6E600017F09E552240575F02D84AAF075F00531
:10D6F600A4CA75F00B842A90D71F9312DCF1BCB82C
:10D70600027BB87D04EE2DF8EF2DF90D12DDEBDD71
:10D71600FB227E0312D50080C6000C1622222D396C
:10D72600444F4F5A66707C7C87939EA9A9000909CD
:10D736000800410000000000888000000000410051
:10D746000800120E7BE5BCB4F8339004C3E0602CED
:10D75600FA24F340277F137E0012DE6C0F0F12DED1
:10D766006C0E12DE9C1F1F12DE9C0EDAEC7F147EFE
:10D776000012DE6C0E12DE9C0EBE12F5229005CC57
:09D78600E0C3941240F60480C7D0
:10CF8500305D0A75F08AA42480E5F034002220740F
:10CF9500157F017E1190D00D12D53F7F0A7E0AE5DF
:10CFA5002E540702D3C87F087E1190D01D12D53F9D
:10CFB50020730C7F0A7E1712DE9C0E0E12DE9C7FFC
:10CFC500007E0BE57112CF8512D3B77F0C7E11E57C
:10CFD50071602F0EE57064B4602864B475F0328416
:10CFE500C0F012D4F9CE2405CED0E075F00584C08A
:10CFF500F012D4F9CE2405CED0E023302D01040261
:10D00500D4F990886A027702070FFFFFC473BDAF9A
:10D01500A463B5FBCDE7FFFF030F0100FFFE03800F
:10D02500306701227F357E00748812D513E5516083
:10D035001712CF8575F06484F87E06E5F012D416D4
:10D04500E860E07E0002D5007E003074D6307316AD
:10D0550079BCE7FC09E7FB12530B781D201704E6A2
:10D0650070011802D2E1909CB0027702202C0122B7
:10D0750090D07B02D53F050EFFF0E01CF004F81CB4
:10D08500FFF0301201227F637E00909CC712D53FCE
:10D095007F1512CA267F1F12CA267F2912CA267F2C
:10D0A500177E06E53F30E00B90A567305C0390A541
:10D0B5007B80132074077E01909CE7800990A55C16
:10D0C500305D0390A571127702307306E54E60025C
:10D0D500154E205718E54EB40113120E8AC3E55CB0
:0DD0E5009560F5BCE55D9561F5BD124EE668
:10D0F2007F217E01E53F30E021305705909E0E8072
:10D1020016E54E7005909E19800D909CF3127702E1
:0BD112007E30E54E02D41C1277022292
:10D2830012530B7F207E05751900781DC2D5E63039
:10D29300D51712D4F9EE2405FE18B818F17E1F74C1
:10D2A30063305C02748202D5137005B8191880E2EA
:10D2B300D2D5CE24FACE7484301702742D12D5132E
:10D2C300EE2406FE80C8742012D50F80C8781C8017
:10D2D3000D7F007E23AC5EAB7A12530B781DC2D553
:10D2E300E630D50C12D500EE2406FE18B818F1224C
:10D2F3007005B8191680EDD2D53017E4CE24FACED6
:10D30300742D12D513EE2406FE80D5742012D51386
:10D3130080D512530B781DC2D5E630D51612D4CE64
:10D32300EE2404FE18B818F10E745E305C02742704
:10D3330002D4DD7005B8191680E3D2D53017DACEE2
:10D3430024FCCE742D12D4E1EE2404FE80CB742091
:10D3530012D4E180CBC23D12D36B0F0F0E0E746358
:10D36300305C02748202D51312530B781DC2D5E6CA
:10D3730030D50C12D52EEE2408FE18B818F1227001
:10D3830005B8191680EDD2D5301716740BCE24F8D4
:10D39300CE12D52EEE2408FE80D5740C12D52E8025
:08D3A300D5303DCB740A80E592
:10D85F007F797E24E55F30E70122AC5F1CAB7B1242
:10D86F005339E51B700E742012D513EE2405FE12EA
:10D87F00D8AD800C12D8ADE51B12D4F9EE2405FEFD
:10D88F00E51A12D4F9EE2405FE742C12D5130E0EE0
:10D89F00E51912D4F9EE2405FE745E02D513742D2A
:10D8AF00201702742B12D513EE2406FE22E55F30EB
:10D8BF00E70122AC5F1CAB7B125339E51B700E7472
:10D8CF002012D4E1EE2404FE12D906800C12D906E0
:10D8DF00E51B12D4CEEE2404FEE51A12D4CEEE24AC
:10D8EF0004FE742C12D4E10E0EE51912D4CEEE24E0
:10D8FF0004FE742A02D4E1742D201702742B12D463
:06D90F00E1EE2404FE22FB
:10D11D007F097E2530040512D2178028A275E57986
:10D12D00C23D6002D23D92D175F080305C04F5F0C5
:10D13D008001A4A2E792D5E5F075F03284F8E5F010
:10D14D0075F00584C0E0E5F0A2D533C0E0E8602AB3
:10D15D0012D52EEE2408FED0E0F8D0E012D52EEE3A
:10D16D002408FE0F0FE52B5403701F746012D513A6
:10D17D001F1FEE2404FEE802D52E740C303D0674FC
:10D18D000A20D1010412D52E80C9205904742E8095
:10D19D00DC205804747F80D5748080D13004051252
:10D1AD00D2178028A275E579C23D6002D23D92D199
:10D1BD0075F080305C04F5F08001A4A2E792D5E50E
:10D1CD00F075F03284F8E5F075F00584C0E0E5F017
:10D1DD00A2D533C0E07F3E7E1CE8602012D58FD0F3
:10D1ED00E0F8D0E07F3E7E2812D58F7F447E3274EA
:10D1FD002E12D5137F3E7E37E802D58F303DE07479
:10D20D000A20D1010412D58F80D59005CAE075F0A2
:10D21D000A84F8E4C5F0C2D522301105E54AB402FE
:10D22D0050C39006E9E0957AFB9006E8E0955EFC28
:06D23D0050031255F6EC4F
:10D24300C31360047B63800FEB13FB249C40F52422
:10D253004F4004C20480079005CAEBF0D204900645
:10D26300E6E09006E8F09006E7E09006E9F0E55E78
:10D273009006E6F0E57A9006E7F02212D26180DEAE
:10CB5300E54424F64001227800E552206607C39598
:10CB630070500224B40475F00384F9E928FE24C448
:10CB73005001FE12CB9512CBA11E12DE6CC3E998B5
:10CB8300FE5003243CFE12CB951E12DE6C08B81F28
:10CB9300DA22EE2420FE24C250032402FE22E824DB
:10CBA300F1E8C2D55006D2D5E8F4241F23FF90CC78
:10CBB3002393CF0493FAE545F5F0A4ACF0FB1253AD
:10CBC3009AE544F5F0A49BFBE5F09CFCEB2420FBE9
:10CBD300EC3400FC12CC04FAE5458FF0A430E702F4
:10CBE30005F0E5F020D502F4042A75F005201903B9
:10CBF30075F00384FF24DF50027F20C374329FFF4C
:10CC030022EC24F0500BEB2460EC340090CC7393B3
:10CC130022EB33FBEC33FCEB33EC3390CC4393222A
:10CC2300FF00FF03FA0BF318EA2ADE40CF58BE7366
:10CC3300AB8D96A880C068D64FE835F51BFD00FF85
:10CC430000080B0E101214151718191B1C1D1E1F9C
:10CC530020212223242526262728292A2A2B2C2D66
:10CC63002D2E2F2F3031313233333434353636379E
:10CC7300373839393A3A3B3B3C3C3D3D3E3E3F3FFA
:10CC83004042444648494B4D4E50525355565859CD
:10CC93005B5C5D5F60616364656668696A6B6D6E4A
:10CCA3006F7071727374767778797A7B7C7D7E7F0F
:10CCB300808182838485868788898A8B8B8C8D8EFD
:10CCC3008F9091929394949596979899999A9B9C07
:10CCD3009D9E9E9FA0A1A2A2A3A4A5A6A6A7A8A924
:10CCE300A9AAABACACADAEAFAFB0B1B1B2B3B4B453
:10CCF300B5B6B6B7B8B9B9BABBBBBCBDBDBEBFBF8D
:10CD0300C0C1C1C2C3C3C4C5C5C6C7C7C8C8C9CAD1
:10CD1300CACBCCCCCDCECECFCFD0D1D1D2D2D3D41F
:10CD2300D4D5D5D6D7D7D8D8D9DADADBDBDCDDDD75
:10CD3300DEDEDFDFE0E1E1E2E2E3E3E4E5E5E6E6D0
:10CD4300E7E7E8E8E9EAEAEBEBECECEDEDEEEEEF32
:10CD5300EFF0F1F1F2F2F3F3F4F4F5F5F6F6F7F799
:10CD6300F8F8F9F9FAFAFBFBFCFCFDFDFEFEFFFF08
:10CD7300E54524FD400122E552206607C395705026
:10CD83000224B40475F00384241FFE24C250032438
:01CD9300029D
:10CD9400FE12CDCEEEFD241EFE24C250032402FE5C
:10CDA40012CDCEE544240275F00520190375F00375
:10CDB40084F4042432FF24EE500F12CDC3AE051EBA
:10CDC4001E7C0512DE6C0EDCFA227F1512DE6C0F5F
:05CDD4000FBF2DF82245
:10D5CE007E00206615E5700475F0B484E5F075F004
:10D5DE000384FE6004C3743C9EFE745312D5F9742A
:10D5EE005712D5F9744E12D5F974457F2F12D4E126
:10D5FE00BE00077E3C12D4E17E00EE240875F03C9E
:10D60E0084AEF00F0F0F12DE6C0E12DE6C0F12DEF8
:10D61E006C1E12DE6CEE240775F03C84AEF02230E8
:10D62E00745C301259E54AB4040122B4060122E5B5
:10D63E007112CBED8F057C037E1E30662AE57004D9
:10D64E0075F00384241EFE24C6501C24FB500424B3
:10D65E00038013C00612D675D0E024C67C01600686
:10D66E000C1460020C14FE12D6810EEE24C1400280
:10D67E00DCF5228D0712DE6C0FEF24CE50F722E57B
:10D68E0053206607C39570500224B40475F00384CA
:10D69E00241FFE24C250032402FE12D6AC0E7F239A
:08D6AE0012DE6C0FBF2DF92202
:10DDA200AF177E00E53C12D3AB7E0C742E12D51356
:10DDB2007E12E53B12D3AB7E1E742E12D5137E2447
:10DDC200E53A02D3AB7E0E78ADE612D4167E187415
:10DDD2002C12D5137E1B18E612D4167E25742C1233
:09DDE200D5137E2818E602D416C0
:10CDD9007F797E00E54012D4167E0A743B12D50F86
:10CDE9007E0CE54102D4167F797E16743B12D50F6D
:10CDF9007E18E53F12D4167F797E0078AEE612D40C
:10CE0900167E0A743B12D50F7E0CE53E02D416300D
:10CE19005EE52043E27F6D7E0078AEE612D4167E91
:10CE29000A743B12D50F7E0CE53E12D4167F757E2F
:10CE39000075F00A84E5F012D52E0F0F7E08743ABA
:10CE490012D50F1F1F7E0DE53F75F00A84C0F01241
:10CE5900D52EEE2408FED0E002D52E851C1E851B9A
:10CE69001FAB1BAC1C305D0A7A1B1253717832124E
:10CE79005513C3EB33FBEC33FC923D125342303D67
:10CE8900087409F51DF51CF51B7F75E51D60157EF8
:10CE99002412D52E7E2CE51C12D52E7E34E51B12CC
:10CEA900D52E803D7E22E51C601912D52E7E2AE5FD
:10CEB9001B12D52E7F787E31742E12D50F7F75E522
:10CEC9001A8019E51B12D52E7F787E29742E12D56A
:10CED9000F7F757E2DE51A12D52EE5197E3512D5EF
:10CEE9002E7F777E3C125CCC851E1C851F1B227F02
:10CEF900397E1F12DE6C0FBF40F9781F79567A0010
:10CF09007D1A12DCF112DDEFEA2406FABAAEF378E3
:01CF19001BFC
:10CF1A00C3E5119570500224B4FA604214603E14BD
:10CF2A00603A2450603A146036EA24A540278A1EE3
:10CF3A00751D007D1912CF4A0D30740312CF4A0DA8
:10CF4A00781F7956AA1DEA12DCF112DDEF0AD3EA3C
:10CF5A00951E40F2228A1D751EB380D7080808085C
:10CF6A007F367E1C90D84BE571700390D85512D548
:0BCF7A003F7F3CAE0090852102D53FB8
:10DA7200787512DAC27453201702744E207406E5C8
:10DA82002E54074430AF1712DAEC7E3BE57DC454C6
:10DA92000F12D5002074077E07742012D5137878F0
:10DAA20012DAC2E5172409FF7457201702744520C1
:10DAB2007402742012DAEC7E3BE57D540F02D5002D
:10DAC200E6FD3392171886041886033017031255A1
:10DAD200FE7917787012550E8B13AF06AED27C000A
:10DAE2007D6412547C8F148D15227E0012D5137E14
:10DAF20007E51312D3C87E19748112D5137E20E56F
:10DB02001412D3AB7E2B742E2073030E742C12D5F9
:08DB1200137E2FE51502D3ABD1
:10DC8100E54A602E7A2420E00E7A26141460087A80
:10DC910028141460027A297F667E01EA12D51320C6
:10DCA1005505205406800B745B8002745C7E001263
:10DCB100D51320110778A9B60007802130261EC28E
:10DCC10026909D887F681276F07F66A85AE54AB44F
:10DCD100060108E875F06484E5F012CE5220080FC1
:10DCE100E537640260097F367E2E744112D4E12249
:10D9150020144F740512DF13EF33EE33F9EF0303D1
:10D92500541FF5F090D968E993A4C5F013C5F01319
:10D93500C5F013C5F013C5F0135403FCE5F013FB54
:10D94500E9242093C9244093C39BC4540FFBE99C4D
:10D95500C4FC540FF9EC54F02B2446F57BE934F65E
:10D96500F55F22FFFFFFFFFFE6C5AD9C8F857D7745
:10D97500726E6C6A696A6A6C6F747A828D9DB4D9AD
:10D98500FFFFFFFAE9DCD3CEC9C6C3C0BEBBB9B73A
:10D99500B5B4B2B0AFADABAAA8A6A4A2A09E9C99FF
:10D9A50096918C00381CE735D137246F00C5B3C17B
:10D9B500E61F66B60E68C21867AADBF4EDB94675B0
:03D9C50010A200AD
:10DEF300D2A27408D2A1D2A300C2A3C2A1D2A3000A
:10DF0300C2A3D5E0EF7405D2A300C2A3D5E0F822E3
:10DECC00C2A3D2A2D2A1D2A300C2A375F0083392EE
:10DEDC00A1D2A300C2A3D5F0F5C2A175F003D2A3C1
:07DEEC0000C2A3D5F0F822EB
:10C4830012DECCD2A300C2A3C2A175F008E4D2A3EA
:10C4930000C2A3A2A233D5F0F5FE75F008E4D2A33F
:10C4A30000C2A3A2A233D5F0F5FFD2A300C2A322F8
:10C4B300E478806608B88BFB70012274D512C483BC
:10C4C3007881C3EE13FEEF13F692D118EE2460F6D3
:10C4D30074D612C4837888EF33CE33CE33CE33CEC3
:10C4E30033A2D192E25407FCEEFB7A08125363ECB9
:10C4F300244FF608EBF674D912C483EF543F7882C5
:10C50300F67886EF33CE33CE33CE33CE335403F6C1
:10C5130008EEF618161608E6C4FF54F0F618E6C43B
:10C52300CF540F2FF674DA12C483EF232354FC780D
:10C5330083F67884EEF608EF54C0F67880E4660854
:10C54300B88AFBF62212C48B7889C3EF96FF18EEE4
:08C5530096FEA2E792165010BB
:10C55B001255E6740FF8F91253B0EF2CFFEE3DFEB7
:10C56B00788BEEF608EFF622E6182016072CF7E686
:10C57B003D19F722C39CF7E69D80F66A405E805614
:10C58B00E050F04B0044803DC0384031D02BA0250B
:10C59B00601F2018D014000F000AA001440158019D
:10C5AB00680178018801A001B401D001EC021002EE
:10C5BB0038026802A002DA030C034D78BE80208596
:10C5CB008E8A9D8F4D95BA9A97A0BEA631AC53B269
:10C5DB002AB801BD6AC1EDC4D1C78812C48B788D4E
:10C5EB00EEF608EFF67887798C1253B07883799052
:10C5FB0012C5737885798C1253B07881799212C5F4
:10C60B0073788DE624E4FE08E63392D13392D55449
:10C61B00FCFFEEA2D133A2D533FE780F79921253E1
:10C62B00B078947990C3EC97F61819ED97F6799446
:10C63B0090C5867F1F7D11EF93C3971F19EF9397BB
:10C64B001F091DED600240EF0F90C5A6798DEF938A
:10C65B00F7090FEF93F7788E79941253B090C5C604
:10C66B00EF93C39BFB1FEF939C2420FC7897E62B47
:10C67B00F618E63CF618E436F6740612DF13D237DA
:09C68B00EE24F7400624025002DF
:10C69400C237EEFCEFFD740712DF13C3ED9FFFEC0E
:10C6A4009EFE78B7E6FD337C0050011CEF2DFFEEB3
:10C6B4003CFE789CEF26F618EE36F6222014122063
:10C6C400370F789DE6B4050912C77812C7AD12C7B3
:10C6D400F62220145E7897799A12C82712556EC3F1
:10C6E400EE9420FE924550031255E67C007D05121F
:10C6F400547C3045031255E6E531B40C3612DA5851
:10C70400120E80E5BC2FF560E5BD3EF56120E71112
:10C7140024F8500DFAC3E5609AF560E5619400F5DC
:10C7240061120E8AE5BC2560F57AE5BD3561F55EDA
:10C7340012DA657897799AC3E697FB1819E697FC9D
:10C744007A0212536330370B7A02125363ECFEEB16
:10C75400FF800312C77812C7AD20140312C7F678FE
:10C76400957998E6F776000809E6F776000809E671
:10C77400F7760022799CE77700FB19E77700FC78CD
:0CC784009DE6B40506EB33FBEC33FCEC47
:10C79000A2E792D550031255F67A32125371ECFB90
:10C7A000EDFC30D5031255F6ECFEEBFF22EE24082B
:10C7B000FE74042037167406307511789DE6B405B2
:10C7C00004740C8007F42406C323540FFD7C00126C
:10C7D000534F789FE6FC08E6FBC374109DFA125392
:10C7E00071EFF8EEF912556EE878A02FF6FF18EE0B
:10C7F00039F62480FE22927540031255E678BBE696
:10C80000F5F02438400375F0E1EF33EE3378A8F605
:10C81000A485F07930E7020579C276307508E579AC
:10C8200024F15002D27622E627FB1819E637FC18CD
:10C8300019E637FD2212BE277F087871793A12C8AF
:10C8400050024ABB855E63857A62787379647F069D
:10C85000E6F70809DFFA227864797380F178737952
:09C86000AF80EB78AF797380E53D
:1052E900E4FEFFFC7D0A791DE7540F2FFFE43EFE23
:1052F900B9190280061912534F80ED301703125560
:10530900E622305C2BEC33921750031255F6EC244D
:10531900D950047C277B007AD2125371EB33CC33FA
:10532900CD33CC33ED33FBEC33FC3017031255F698
:10533900EC33921750031255F67919125585F7096E
:10534900B91DF8A70322EFF88DF0A4FFEDC5F0CE43
:10535900A42EFEEC88F0A42EFE22EB8AF0A4FBE535
:10536900F0CC8AF0A42CFC22EB8AF0A4FBE5F0CC6B
:105379008AF0A42CFCE435F0FD22EB8AF0A4FBE5CD
:10538900F0CC8AF0A42CFCE435F0CD8AF0A42DFDF4
:1053990022EB8AF0A430E70205F0E5F0CC8AF0A40C
:1053A9002CFBE435F0FC2286F0E7FDA4FAABF019FA
:0653B900E786F0A42BFBC7
:1053BF00E435F0FC18E68DF0A42BFBEC35F0FCE4A3
:1053CF0033FDE687F0A42CFCED35F0FD22EB89F0E0
:1053DF00A4CBAEF08AF0A42EFEE5F03400FDEC89EC
:1053EF00F0A42EFEE5F03DFDE433CC8AF0A42DFDB4
:1053FF00E5F03CCEFC22EB89F0A4CBAFF08AF0A411
:10540F002FFFE5F03400FEEC89F0A42FFFE5F03E0E
:10541F00FEE433CC8AF0A42EFEE5F03CFCED89F0DF
:10542F00A42EFEE5F03CFCE433CD8AF0A42CFCE581
:10543F00F03D8E058C068F04FF22C2D5EC30E705B8
:10544F00B2D51255EEEE30E70DB2D51255E6125425
:10545F007C1255EE800312547C30D5031255E62290
:10546F00C3EC13C0E0ED132FFFD0E03EFEBC000BEA
:10547F00BE0029EF8DF084FFADF022E4CCF975F07A
:04548F0008EF2FFFF4
:10549300EE33FEEC33FCEE9DEC994005FCEE9DFEF5
:1054A3000FD5F0E9E4CEFD22EDF9F5F0EE8420D23C
:1054B3001CFEADF075F008EF2FFFED33FD400799AB
:1054C3005006D5F0F222C399FD0FD5F0EA22EC3352
:1054D300EE3400FEEF3400FF7D007A007900780996
:1054E300C3ED9AFDEE9BFEEF9CFFB392D54009ED11
:1054F3002AFDEE3BFEEF3CFFA2D5E933F9ED33FD88
:10550300EE33FEEF33FFD8D92279007A00C380153A
:1055130079007A00C3EA13FFE913FEE8132BFBEECD
:105523003CFCEF3DFDE4F5D2F5D333FE7F19C3EE2A
:1055330098FEE5D299F5D2E5D39AF5D3B392D54047
:105543000DEE28FEE5D239F5D2E5D33AF5D3A2D54F
:02555300EB3338
:10555500FBEC33FCED33FDDF0122EE33FEE5D23308
:10556500F5D2E5D333F5D380C3EDC454F0FEECC4D6
:10557500FF540F2EFEEF54F0FFEBC4540F2FFF2204
:10558500EC75F00A84FCEB54F025F0C475F00A8440
:10559500C4CBC454F025F0C475F00A842BFBE5F0A8
:1055A50022AC10AB11125585A904AD03FA7C197B09
:1055B50099125363AE04AF03EA75F006A4F8AC1272
:1055C500AB131255852875F00A8485F014F8EF2B76
:1055D500FFEE3CFEEF28FFE43EFEE43DFDE439FC32
:1055E50022C3E49FFFE49EFE22E4C39DFDE49CFCF0
:1055F50022C3E49BFBE49CFC22C3E49BFBE49CFCF0
:10560500E49DFD2275D4107B807A0079807800EACC
:0A561500F5F0A4FCADF0EBF5F0A4F5
:10561F00FEAFF0EB8AF0A4C333C5F033C5F092D5DB
:10562F002DFDC5F03EFEE430D501043FFFB5150D4D
:10563F00EEB51409EDB51305ECB51201224006EADB
:10564F0098FAEB99FBD5D40ABB0001220ABA0001E4
:10565F000B22C3E913F9E813F8EA28FAEB39FB80B8
:10566F00A478087B807D807C00EDF5F0A4FAE5F04E
:10567F008EF0B5F007EA8FF0B5F001224003ED9BF5
:10568F00FDD827BDFF0122EDF5F0A4F9A8F0ED0438
:10569F00F5F0A4C399FAE5F09813CA1329F9E83A7B
:1056AF00F8C3E99FE89E50010D22C3EB13FBED2BCE
:1056BF00FD80B6C374689511FB74019510FC8004CE
:1056CF00AC10AB117A0B79B81253DC80177473F8E6
:1056DF00F9E627FB0809E637FC0809E637FD30E74E
:0556EF00031255FEEB63
:1056F40033FBEC33FCED3323FD242083F8ED241C31
:1057040083FFED241883FAED241483F9EF99F9E863
:105714009AFA1253DCEF9DFFE89EFE22FFFFFFB6CC
:10572400FED7FD63FB5DF8C4F59BF1E3ED9EE8CF86
:10573400E379DD9ED743D06BC919C153B91CB07945
:10574400A7709E06943F8A237FB674FF6A045ECBDB
:10575400535B47BB3BF1300423FB17DE0BB2FF80E6
:10576400C21DC232532CF8C3E5679576FBE56895F4
:1057740077FCE5699578FD30E705D2611255FE2482
:10578400F05003125838AA06A907125405EC2480D5
:10579400E43DFBF9F51AE43EFCFAF519E43F600236
:1057A400D2321253DC8B128C138D148E15C3E56424
:1057B4009573FBE5659574FCE5669575FD30E70525
:1057C400D2621255FEEBF9F51FECFAF51DED6002FD
:1057D400D232303201221253DCEB2512F512EC35B1
:1057E40013F513ED3514F514EE3515F51540E102F6
:1057F400560912576420323BEB242E40D3EA24018D
:10580400CB3400FC7A07793D1253DCC010C0118EF2
:10581400108D118C128B13E4FCFD7E077FD012B522
:0E5824008E851203851302D011D010BB000533
:10583200BA0002D21D22B261C374809BFB74F59C34
:10584200FC74209DFD22204D69204866303F637F15
:10585200697E0112CA3A7E1F12CAAA75A700900475
:10586200EDE0A2E792171392E7FC1582E013FB30FA
:1058720017031255F6BC003AEB603720E73420E6F6
:105882003110E513201707C3741F9BFE80027E1F91
:1058920012CA9F0EDBFA22FB2017097E00C3742076
:1058A2009BFB8008EB241FFE74209BFB12CA990EFF
:1058B200DBFA2275A700758307E559C4440FF58208
:1058C200E0A2E792522212C85D1258B5C2E775F003
:1058D2000A84FEAFF075A7045382F1786412593E30
:1058E200AE07786712593E75A700E57DC4540FFED6
:1058F200E57D540FFF7873125932AE07787612594C
:105902003274AF1256DE1257F68B148A1312092024
:10591200ACCCAB017A0A125363E5139B9004ECF012
:10592200FBA3E5149CF0FCA2E7923DD23F02C863C0
:10593200860308860408860518188006E0FBE0FC4A
:0A594200E0FD7A0A12538320E70CFF
:10594C00EB2EF608E43CF608E43DF622C3EB9EF69B
:10595C0008EC9400F608ED9400F622204D0920483E
:10596C0006C23F302A0522C23380F6E54824F640B1
:10597C00F5E5580460F075A700758307E559C42454
:10598C0008F582E0FEA3E0FF1209207437125A2AB0
:10599C00500B30381BC23878C586468013743212CF
:1059AC005A2A400C203809D23878C5A646754600CC
:1059BC00740D125A2A404A1258C8303D3820112210
:1059CC00204D1F20481C204019BCFF16EB243250E0
:1059DC0011D240120E62E5BF75F019A4F536D22E25
:1059EC00D22F205238E55965586032204D2F20486F
:1059FC002CD2338028201109204D062048037536FF
:105A0C0000303319204D1220480F1291460559C30E
:105A1C00E55895595003855859C233C2402229FB89
:105A2C00E435CCFCC3EB9FEC9E22E558B4FF01227D
:105A3C0085581175A704758307E54824F650028034
:105A4C005C201259202905202A02805112C85DE4DD
:105A5C00F516F517751000125AC2E510700312C82E
:0B5A6C0057125ADB302910E51B2517EC
:105A7700F517F51BE51C3516F516F51C125AE81235
:105A8700C8570510C3E511951050D175A70002C876
:105A970063E55AF51124F6500375110A75A70475C5
:105AA7008306751000125AC2125ADB125AE8051003
:105AB700C3E511951050EE75A70022E510C4F582D5
:105AC700E0E0F564E0F565E0F566E0F567E0F568C8
:105AD700E0F5692275A701125ED4123ED775A704B7
:105AE70022E9F0E51CF0E51BF022E510C454F0F5BF
:105AF70082E0F512E5822406F582E0F511E0F51C57
:105B0700E0F51B22E512B426157F757E34740D125D
:105B1700D52E20442575110012CEF8025C397F6D11
:105B27007E3BE012D513E5137E3512D513E5127EC1
:105B37002F12D51320440312CEF812CE64025C391B
:105B4700202852E558B4FF012275A704758307E59D
:105B570059F51030330965586005204802051012C1
:105B67005AF1E0F513305E07204304E5376095E00E
:105B77007F797E3D12D4E1E5137E3912D4E1E51237
:105B87007E3512D4E130480B7F7F7E3512DE6C0EF6
:105B9700BE40F980392012012275A7047583068556
:105BA7005B10125AF1305E0A204307E53770030293
:025BB7005D5B34
:105BB900E512700B7E3A7F79745D12D513800D75ED
:105BC900F06484E5F07E397F7A12D463E537B40254
:105BD90005128FDE8045B403028040E51C7006E59E
:105BE9001B24FB5036E511F964B4602F20062CE51F
:105BF90037600D200C0AC3E99570F9500324B4F9F4
:105C0900E912DCF1781D79547D1D90D83DE53F20DE
:105C1900E00390D84412DDEF12D53F751779751658
:105C29001930280375161DE51264266003125C7C81
:105C390075A7009006E3E511F0A3120E7BE5BC758C
:105C4900F01970040475F014A4951BFBE5F0951C7C
:105C5900FC922450031255F6ECF0A3EBF0C24FC2AC
:105C690063EC700EEB24E64002D24FEB24C84002ED
:105C7900D26322E51C24ED402BAE1CAF1B125E9EA5
:105C89007C007D3212547CC005EFAF17AE1612D4DA
:105C99001CCE2405CE742C12D5130E0ED0E023127F
:105CA900D416801B125E95125CD6CE2405CE742CB8
:105CB90012D513CE2402CEE875F0058412D4F9CE9C
:105CC9002404CE7422305D02748302D50FEE243D84
:0D5CD90050047EC37F4B7C017DF412547C8F
:105CE600C004C005EF6007AF17AE1612D41CD0076C
:105CF600D0067C007D3212547CA805EFAF17AE1695
:105D0600CE240ACE02D4F9125E95EE2450305D03FD
:105D1600EE24A150047EC37F4B7C017DF412547C9B
:105D2600C004C005EF6007AF177E2F12D469D007F5
:105D3600D0067C007D3212547CC005EFAF177E374B
:105D460012D4CE7E3B742C12D4E17E3DD0E075F0A9
:105D5600058402D4CE7F6D7E2F746312D513E512AF
:105D660075F06484E5F07E3512D3AB12CEF802CE20
:105D76006430480320740122E4FCF5A79006E3E0B2
:105D8600F9A3E0FE24FE40EFA3E0FF7D78E537604F
:105D960008304FE3200C2A800B120E67E5BD20E089
:105DA60010304F0DD206E57124FE5015125E8B8021
:105DB600107D3CE546600A7D141460057D0A14706A
:105DC600B6891112534F7D6F12546FBE00A9EF248E
:105DD600E240A4AD07E51112DCF1202404B2D5B2ED
:105DE600D1781F795612DDEFA806A907E511242DF3
:105DF60075F0B484E5F012DCF17407304F02740ECE
:105E0600FDFA12DDEFB2D5B2D112DDEFB2D5B2D1C5
:075E1600DDF0AD0212DDEF2B
:105E1D00850616850717B2D5B2D112DDEF85061EA0
:105E2D0085071F7A03304F027A06E511241675F0A7
:105E3D00B484E5F012DCF1A816A917AD0212DDEF5E
:105E4D00DDFBE51124EA400224B412DCF1A81EA901
:105E5D001FAD0212DDEFDDFBE5377021304F1E90D7
:105E6D00A61F305D0390A61B7F3C7E331277351243
:105E7D000E67E5BD20E00612CAB012D7DE22C3E9D7
:105E8D009570500224B4F922E51B2402FFE4351C61
:105E9D00FE305D1ABEC305BF4D028012AC06AB07C6
:105EAD007A1B1253717832125513AE04AF03227858
:105EBD007379641256E01257F6751CC3751B4B208F
:105ECD0032048B1C8A1B22125EBC30320122AC19AB
:105EDD00AE1AA91DAF1FB90005BC00028010C3E9A1
:105EED0013F9EF13FFC3EC13FCEE13FE80E8BF298B
:105EFD00005006BE2900500122C3EF13FFC3EE135D
:105F0D00FE80EB3E7FE3E3E3E3E3E3E3E3E3E37F01
:105F1D003E0C1C3C7C7C1C1C1C1C1C1C1C7F7F3EDA
:105F2D007FE3E3E3070E1C3870E0E3FFFF3E7FE302
:105F3D00E3030F0E0F03E3E3E37F3E070F1F3F77EE
:105F4D00E7E7FFFF0707070707FFFFE0E0E0FEFFBA
:105F5D00030303E3E37F3E1E3F73E0E0E0FEFFE358
:105F6D00E3E3E37F3EFFFFE3E30303070E1C383853
:105F7D003838383E7FE3E3E37F3E7FE3E3E3E37FBF
:105F8D003E3E7FE3E3E3E37F3F030303E77E3C0015
:105F9D000000181818FFFF18181800000000000066
:105FAD00000000FFFF0000000000003FF00000387F
:105FBD001C38F00180C1F020F0FC0038F03FE0000B
:105FCD000000007CC6C6C6C6C6C6C6C67C183878D4
:105FDD001818181818187E7CC6C60C183060C0C664
:105FED00FE7CC6C6061C0606C6C67C0C1C3C6CCCCC
:105FFD00FE0C0C0C0CFEC0C0C0FC0606C6C67C3CDC
:10600D0066C0C0C0FCC6C6C67CFEC6C6060C18302F
:10601D003030307CC6C6C67CC6C6C6C67C7CC6C6FD
:10602D00C67E060606CC78000018187E7E1818006D
:10603D0000000000007E7E00000000000000000057
:10604D000000000000C6E2E2D2D2CACAC6C6C20033
:10605D000000000000000000008080A0C0A0003003
:10606D004020C08080C0A0A0000060A0600000A003
:10607D0040A05098D090882050A850888850A850A3
:10608D002060806000000040E040000000000080C3
:10609D000000E000000000000040002040800040B3
:1060AD00A0A0A04040C04040E0C02020C0E0E020C3
:1060BD004020E02060A0E020E0C02020C06080E013
:1060CD00A0E0E020404040E0A0E0A0E0E0A0E02023
:1060DD00C0004000400000800080002060E0602093
:1060ED0000E000E00080C0E0C080E0E0E0E0E00023
:1060FD000000000040A0E0A0A0C0A0C0A0C040A033
:10610D0080A040C0A0A0A0C0E080C080E0E080C022
:10611D0080806080A0A060A0A0E0A0A0E0404040F2
:10612D00E0202020A040A0A0C0A0A080808080E022
:10613D00A0E0A0A0A0A0E0E0E0A040A0A0A040C0F2
:10614D00A0C0808040A0A0C060C0A0C0A0A0608002
:10615D004020C0E040404040A0A0A0A060A0A0A072
:10616D00A040A0A0A0E0A0A0A040A0A0A0A0404062
:10617D0040E0204080E02020A870202070A8202042
:0D618D0008F030D0100000F0A8A8000000BD
:10619A00E0000000902048708898984000E0E0E015
:1061AA0000A0E0E0E04060301030604040E0404055
:1061BA0060909090909060206020202020706090E5
:1061CA0010204080F06090102010906010305090A5
:1061DA00F01010F080E010109060609080E09090D5
:1061EA0060F0102020404040609090609090606085
:1061FA00909070109060C0E0F0F8F0E0C0000000ED
:10620A000000000000000000000000506050007014
:10621A007050000078807008F000F8888888F800CC
:10622A00C0C8102040981800C0B098B0C0006020C4
:10623A0040000000000090D8FCD8900000246CFCBC
:10624A006C24000020A870A82000002020F820203C
:10625A000000000000000080000000F000000000C4
:10626A0000000000606000081020408000708888EC
:10627A00888888702060202020207070880810206C
:10628A0040F8F810201008887010305090F810105C
:10629A00F880F008088870304080F0888870F80824
:1062AA00102040404070888870888870708888788C
:1062BA0008106000606000606000000080000080DC
:1062CA0000002040F84020000000F800F80000001C
:1062DA002010F8102000708808102000200000000C
:1062EA000000000070888888F88888F08888F0881C
:1062FA0088F070888080808870E09088888890E034
:10630A00F88080F08080F8F88080F0808080708843
:10631A0080B8888878888888F888888870202020BB
:10632A00202070381010101090608890A0C0A090A3
:10633A0088808080808080F888D8A8A88888888803
:10634A0088C8A898888870888888888870F088881B
:10635A00F080808070888888A89068F08888F0A08B
:10636A00908870888070088870F82020202020206B
:10637A00888888888888708888888888502088884B
:10638A0088A8A8A85088885020508888888888506B
:10639A00202020F80810204080F800CCAC9CACCC1F
:1063AA000000CCD4E4D4CC0004781828C800FC40FF
:1063BA00A04018202018000000000000F80000008B
:1063CA0000A040A05000788888986870884030887B
:1063DA0070200000F0A8A8A8A878484848487888FB
:1063EA0070888080887020A88898A8C8888880507B
:1063FA0048FC485080304C5C6060603C00E0F0082B
:10640A000808F88044485C484480F880808080808E
:10641A008078484848484888B8A8A8E8A8A8B8880A
:10642A0088888888F808500070888888708080F08A
:10643A0088888888F8888888888888F090909090DA
:10644A0090F0A8A8A8A8A8A8F8888888F808080832
:10645A0050008888888878A8A8A8A8A8F808000002
:10646A000000000000000000000000008888888802
:10647A00E8A8E8A8A8A870A8A8A80000000000003A
:10648A000000000000000000000000000000000002
:10649A000000000000000000006000606000600072
:1064AA0060006060205020000000005090B890D03A
:1064BA0090886050500070705000882020887000CA
:1064CA000080C0A090F8003048B4B448300030488A
:1064DA00B4B44830FC0098D02058C800F8E8D880F6
:0A64EA00D8E8F8404050F850404058
:0300000002005E9D
:03000B0002B61E1C
:0C000E00206E06859950D26E32D26F32FF
:0E00230010990AC298206DE385994FD26D3274
:10003800E4F537F534F52F12DE62C229C22AC26808
:09004800C227C214C215022D9C4E
:03005B00022B2A4B
:10B611008530F0C5F065308530F060F722C0D0C0CC
:10B62100E0C0F0C0A775A700C083C08275D00875BF
:10B631008A00300503758A7A758CEA0532E5327025
:10B641000215320530E530640A6026201520E53107
:10B65100B40C0BE530B4010612BA9912D915E531D3
:10B66100B4180BE530B4060612BA9912D91502B80E
:10B6710038C2AFD2C075C07AD2AFF5300531E531ED
:10B6810064197040F531201529C225C22C7D0A7438
:10B691000412DF13EF33EE339005CCF0EE24F540C6
:10B6A100112402400B24014005DDE4022B2AD2259E
:10B6B100D22CE5A6600215A678B5E660011678B62B
:10B6C100E6600116302E0BE5367007C22FC22E122E
:10B6D100B9C6E5367004C24B8002153678A9E6601A
:10B6E100011678D8E66001160535E5357002153585
:10B6F100E590307B0B30E008D278C27BC200801A23
:10B70100307C0B30E108D279C27CC201800C307DE3
:10B711000930E206D27AC27DC202E59044F8F470A3
:10B7210003753500304A09E53324FA5003753305B2
:10B73100E5336005153302B7DDE590F45407700376
:0DB7410002B7DDA2E09200A2E19201A2E2B7
:10B74E00920230100320143D75330820001B201088
:10B75E000C2011098013E59030E10E8006E53724A8
:10B76E00FC40F3E543541FF53320100375A6FF206C
:10B77E002E5D301004E536705620100C201109E5B0
:10B78E003524F55003753304D21BD2A5D2A612B9B7
:10B79E00C675B44075B24078D8E6700205342027DD
:10B7AE002E20682B202928202A25A2107211501F26
:10B7BE00E52054076019E53424375004C24A800F3F
:10B7CE002401400B200026200119D27D7534C8209B
:10B7DE001558E531702412DEF374E812DECC802A9F
:10B7EE0002B90BE53724FC40E6D27C80DF3011DF56
:10B7FE00E53724FC40D9D27B80D275F00384E5F086
:10B80E0070DE12C54874E812DECCE531B4060512BE
:10B81E00C6C08016B40C0512C6D6800EB412051220
:10B82E00C6C08006B4180312C6D6E59030E10530C6
:10B83E00E202800620100820110520103C807D2099
:10B84E0027F82068F52029F2202AEFE5342430402D
:10B85E00E9240750E5600B205E088590F020F20287
:10B86E00740190B88093D2A5201002C2A512B9B16E
:10B87E00806FC8A08269554646202F12E536603C7F
:10B88E0024AA500AE53675F01984E5F06040D2A678
:10B89E00201002C2A6D2A5202F0C7418304B0274B1
:0EB8AE006412B9B1803BE53675F00C304803EA
:10B8BC0075F00684A2E0744640E9743780E5E52B08
:10B8CC005403600C20100E301106E54A640260052A
:10B8DC0012B9CC800312B923101B08A25892A5A24E
:10B8EC005992A675A700D082D083D0A7D0F0D0E013
:10B8FC00D0D0201009C5A67003022B2AC5A632C2CF
:10B90C0018B40202D21812C5E630180874E412DE1C
:10B91C00CC02B81802B81378A7E5B4600924E0404B
:10B92C0005760002B9CCE534702920412220751F20
:10B93C00300D1CE57924CE40167AFFE5B110E701F5
:10B94C000A2325B3F5B3EA35B4F5B4C313F5B2E65F
:10B95C0060021622C2412075028075E579FF60589D
:10B96C0020120424FD5051206502C21CD265FF2414
:10B97C00B050027F4FEF90BA499375C70375C6FC60
:10B98C0075B90185BFF0A4E5F0F624F44002760CFD
:10B99C00301C2DE5BEC39FF5F0A4E5F024E0400378
:10B9AC0075F020E5F0C21C79AA770375B300F5B4E5
:10B9BC00C31375B100F5B222C26578A77680D24167
:10B9CC0079AA7703D21CE4F5B3F5B4F5B1F5B2223C
:10B9DC00C26579A1E57924CE500DE720E7E27628FF
:05B9EC00301CDD743287
:10B9F10080BE7680E720E7D3E5799740CE79AAE744
:10BA0100FAE5792323B4C500400274C42437300E0B
:10BA110031F42437300D15F7BA0302FA0AC39AF547
:10BA2100B175B300EAF5B4C313F5B222101C07D205
:10BA31001C76C802B9B3763274FF200E02749B02E1
:10BA4100B9B3C313247E80CCFFF3E8DDD3C9C0B8FA
:10BA5100B0A9A29A948F8A85817D7975716E6B6880
:10BA610065625F5C595653504E4C4A4846444240C9
:10BA71003E3C3A383634333231302F2E2D2C2B2A9E
:10BA81002928272625252424232322222121202079
:10BA91001F1F1E1E1D1D1C1CD2B5C28EAE8DAA8D70
:10BAA100AF8BAB8BE4F58DF58BD28E301401227800
:10BAB100B6BE0007EF24E24002800806E624EC50FF
:10BAC100027614206705E624F64005E4FEFAFFFB42
:10BAD1007C007D0A12534F7C007D5E12546F8F51A2
:10BAE100EE60037551FFEAFC7A33125363EBF5F014
:10BAF100A4E5F0CB8CF0A425E0C5F035E0CB92D5E0
:10BB010025F050060BBB0002D2D530E7060BBB0077
:10BB110002D2D5ECF5F0A42BFBE5F03400FC30D5D6
:10BB2100010C78A6E6C39BFF18E608F6EB18F61899
:0EBB3100E69CFE18E608F6EC18F63014012229
:10BB3F007A0050040A1255E67C007D6E12546F8F06
:10BB4F00F078A2E6A4FBACF0125585EBBA0002F434
:10BB5F0004FAE4F8FFEA30E70118E579600620758A
:10BB6F00031FF4042AF579EF38D27520E708600334
:10BB7F007579FF02C819C2750470F5E579F4046090
:10BB8F00EFF57980EE120E5D78BBA6BC120E7BE549
:10BB9F00BE78A2F624F65007E4F5BEF6124EE61272
:10BBAF000D46E5BEF54824F65008E4F5BEF54812FB
:10BBBF004EE6E5BFF54324F3503924F34035120E1A
:10BBCF007178A1A6BCE5BF789DF61424FB500874CC
:10BBDF0003F6F5BF124EE678B7A6BE120E67E5BDA7
:10BBEF00A2E39266A2E49267035403C253B4010224
:0EBBFF00D25322740DF5BFF543124EE680C0FE
:10005E0078FFE4F6D8FDF4F5A6D2B4D2C075C07A16
:10006E0075D75075AE1375AF017581D87590F8754B
:10007E00EFBC75FDFFD2A412DE39C2A47450122B50
:10008E0042758951D28C75A882D2BC12BC0D12DE7B
:10009E00F312C4BE12BB9412D9C8122A087F407E36
:1000AE0001909C73127702124D4A12DE3912DB1A3E
:1000BE0012DD5112DE627C1412DE43300003022B7D
:1000CE002ADCF512489F753A001248EDE53A701693
:1000DE0012DF277F437E0690A40312770212DD51B2
:1000EE003000FD022B2A75A6FF12489F12BB9412F8
:1000FE002A0812DD5112DE3512DE6278B5761E1236
:10010E00D9C812C4B3C215C214122A08909CBA7F61
:10011E00781276F0205E0A7F767E12909CC712D5FA
:10012E003F7F4012DDC77F497E0978AEE612D3AB22
:10013E007E15743A12D5137E1AE53E12D3AB7E2687
:10014E00743A12D5137E2BE53F20E00805A6E5A6EE
:10015E00700215A6E53F12D3AB7F5312CA2E7F57FE
:10016E007E0B12D2D812D3607F6020730302020876
:10017E007E0BAC5DAB5C12D2DC12D3607E3112779B
:10018E008D7F697E1212D8633025087E1290DB8334
:10019E0012D53FE5A60303543FFDFE0D7F7312DE1D
:1001AE006C0F12DE6C1EDDF478B5E57124F640029C
:0801BE00761E307419E660564C
:1001C6007F727E16744012D4E17E17E612D4697EE1
:1001D6001F745312D4E112DD51100037100137108D
:1001E600023712483FD2AC75369612DBC9B4E00529
:1001F600124935800AE53670F112488D12DE320258
:10020600010D2074097E2BE52E540712D5007E17AA
:1002160002018C022B2A022D628072E53524C85019
:1002260049E59020E244D0E0D0E012027102735614
:10023600E53524D25034E59020E22FD0E0D0E0120C
:10024600DF278038E53524D25020E59020E21BD008
:10025600E0D0E012DF27306B0B7F091276E7124FF2
:100266001E127BBD1202710206BE2212DF2790A467
:10027600BC7F001276F012DD5102DE3212DF2790CB
:10028600A4BC7F001276F012DD5112DE35C215C213
:1002960014C227C26812DE62753701909DA3121C34
:1002A600FF9002AB730200F70217C2020B56021F41
:1002B60012021F0E0206BE0206FB0273560202C699
:1002C60012DE6275370790A149121CFF9002D673A1
:1002D60002029302096B0209A50209D90202FA0277
:1002E60005AD0202C60202C60203180202FF024B55
:1002F600B30203261248F0805A7F517E00747212B0
:10030600D50F121E5C40B9124E3512D9C812BB94D5
:1003160080AE7F49A25E120D31925E120D5080A012
:100326007F64120E9E121E5C401DE5352480F47516
:0C033600F0198460157F727E1F12D50044
:1003420012DD511001E810000280E30202C612BC65
:100352007A0202C6124EE612DE6275370290A32BB3
:10036200121CFF900369730202C6020EA8020F0D4F
:10037200020F61020FB6020FFA02100902035902BC
:10038200051302038980D0D21412DF277F147E0561
:1003920090A374127702121E1912DD511248687569
:1003A200A6FFD2AC1000DE12DBC9204CF2B405EF7E
:1003B200E4F511F514F5151204411204D51248683A
:1003C20075A6FFD2AC1000BD12DBC9204CF2B415E9
:1003D200051204C880E7B406E712047FE51424FC82
:1003E20050D5E4F56FF56EF56D12048B1204D5123B
:1003F200486875A6FFD2AC10004212DBC9204CF24D
:10040200B415051204C880E7B406E71204B5E56F17
:1004120024F050D5124868743B12DC457A47909C10
:100422006A1224C9742A12DC39909C731224C9748A
:100432002A12DC39DAF912DC6212DE43020359AC09
:1004420014AB157A0412536375A704900400E4F008
:10045200ECF0EBF08514C78515C67F08120467DF40
:10046200FB75A7002275B901E5BCF0E5BDF0E5BE5C
:10047200F0E5BFF005C6E5C6700205C722E5152402
:1004820008F515E43514F5142275A704900400E567
:100492006F4410F0E56EF0E56DF0740312BC467F18
:0404A20020E4F5F766
:1004A600C2B2C2B2E5F7F0DFF4D2B275A700227489
:1004B60020256D54E0F56DE4356EF56EE4356FF587
:1004C6006F2205117F287E00E51112D42280069046
:1004D6000402E070177F287E15900400E012D422F3
:1004E6007E2A900401E012D42212DD51124868746B
:1004F6003A12DC7C75A7009004007F23E0A312DC8F
:1005060018DFF912DC533099FD2202035912DF2756
:100516007F0F90A6AE1276F0121E1912DD51C2148C
:10052600C21512DE327510651000DFE53170F9E58F
:10053600106465700D855E14857A15E4F512F51361
:10054600800C78A8E51326F513E43512F5127F1E04
:100556007E19E51012D3C8C3E57A9515F517E55E41
:100566009514F5167F287E0BAC16AB1712D2DC124B
:10057600D36012DD5112DE43D510ADAB17E516FC84
:1005860030E7031255F67A0A79001253DCA912A84D
:1005960013125515EBF510243840037510C8120ECA
:1005A6005D8510BC02035612DF27909CFF7F017EFB
:1005B60009127702909D087F0A7E091277027F133F
:1005C60012CA26751700120E6CE5BC12068DE5BD23
:1005D60012068DE5BE12068DE5BF12068D909D585A
:1005E6007F5F7E06127702121E9E12DD517517007E
:0605F60012066D10000862
:1005FC0010011510024880F20517E51724F7500377
:10060C0075170075100080E2E51764087015120E5E
:10061C006C75BC0175BD2375BE4575BF67124EE682
:10062C000205ADE51012069F12DD5112064D0510A4
:10063C00531007E51724FE400353100380AC02024D
:10064C00C6A9BCAABDABBEACBFE5171304F8E64007
:10065C00085407C42510C4800454702510F6027D7C
:10066C00A17800E875F009A42417FF7E3B7D20E8F3
:10067C00651770027D89ED12D51308B809E502DD06
:10068C0051F8C4120693E812069F7E030517E5176E
:10069C0002D500540775F009A4909D102582F582AF
:1006AC0050020583E51775F009A42417FF7E0C0290
:1006BC007702C26812DE62753705909EE5121CFF48
:1006CC009006D073020293027941027986027B1C58
:1006DC000206BE0206F4027A5E027AC402178B028C
:1006EC0006BE021771020C627F2E12168680C31290
:1006FC00DE62753706909FC0121CFF90070B7302C9
:10070C0002930217C802182A0218A30219700219C0
:10071C00A2021A19020750020749021A62021B07A9
:10072C0002072F7F64120E67E5BDA2E7120D31128E
:10073C000E67E5BD92E7F5BD124EE680B27F491219
:10074C00168680AB12090C122B6912DF27121DF3CF
:10075C00E55804607790A0921207F912871E12DDFB
:10076C005110000810011310021C80F50559C3E547
:10077C0058955950D575590080D01559E55930E721
:10078C00C985585980C4E559B40F02802FB51F0292
:10079C00802A75F007A42408F51775162774B82558
:1007AC0059F987001207E712DD51100028100128B3
:1007BC0010020280F574B82559F9A700E53524FA22
:1007CC00508878C7A64812090312DF2712DD511290
:1007DC00DE350206FB1880CC0880C9E875F005A44C
:1007EC0085F01CF51BC000125C7CD000221287AF78
:1007FC00B4FF0122751000751FFF1287C6E5106447
:10080C000F6017120830401274B82510F8E675F016
:10081C0005A485F01CF51B125D0D0510C3E558955C
:10082C001050D7221211AEF8602E6404602AE8141E
:10083C00B51025F51F120E7BE5BC70060475F0147F
:10084C00800375F019A485F01CF51B125D0D7E223A
:10085C0090A64F127735D322C322E558B4FF01225C
:10086C00751000E510640F602EE51075F007A424D8
:10087C0009FF74B82510F8E61208ED75F00A84C06B
:10088C00F07E2012D4697E28742C12D4E1D0E07E44
:01089C002A31
:10089D0012D4CE1208AD0510C3E558951050C322E1
:1008AD001211AEF8603964046035E8146510702FCC
:1008BD00120E7BE5BC1208EDF8C313923D7E1C129F
:1008CD00D47F7E28742C12D4E1E4303D067405B833
:1008DD000001147E2A12D4CE7E18742312D4E12284
:1008ED00305D1275F036A42432FBE435F0FC125560
:1008FD0085125585EB221209151276D5DFFB2212D2
:10090D000915127EB1DFFB2275C70375C6F078B8E5
:10091D007F042275C70375C6F375B901E5BFB548E8
:10092D0031E55924F1402BE55975F00484A9F024E3
:10093D00F0F5C675B901C5F0A9BC600CA9BD146070
:10094D0007A9BE146002A9BFE975F005A4F985F0E9
:10095D00CC22120E7BA9BD75CC0022124EE612DE02
:10096D006275370390A1B6121CFF90097B730202CA
:10097D00C6020C7B02131F020C90020C9B0216E6A2
:10098D000213A6020D5C0213DA02142002173802BC
:10099D00138E021465124EE612DE6275370490A2B4
:1009AD007F121CFF9009B5730202C6020CAA020C3D
:1009BD00B50209A5020CCB020CD60210230209A523
:1009CD00020CE5020CC0020CFF124EE612DE62753F
:1009DD00370B90A2D0121CFF9009E9730202C602D8
:0B09ED0010D10210D1020A6F020AAD07
:1009F800020A10020A330217CE02117602123E02D0
:100A080011E70212CF020D19120E67E5BF1470C16B
:100A18007F2E120E9E1F120E67E5BDA2E6120D3143
:100A2800120E67E5BD92E6F5BD80A37F37120E9ED4
:100A3800120E62A8BFE8120A6712DD5110000810F2
:100A4800010D10021280EE18B802EA780A80E60852
:100A5800B80BE2780380DE120E6288BF0209D67FE7
:100A6800367E2CE802D3B17F1C120E9E120E67A8A8
:100A7800BE120AA112DD5110000810010D10021457
:100A880080EF18B800EB780B80E708E824F450E111
:100A9800780180DD88BE0209D67F1B7E35E875F0B7
:100AA80005A402D3AB7F25120E9E120E67A8BF12B3
:100AB8000ADF12DD5110000810010D10021480EF3A
:100AC80018B800EB780980E708E824F650E17801C7
:100AD80080DD88BF0209D67F247E3BE802D500125C
:100AE8000E5DE5BF75F03CA4ACF0FDE5BE75F00504
:100AF800A42DFDE5F03CFC120E67E5BF14603675C9
:100B0800F005A485BEF0A42DFFE5F03CFE7C007D39
:100B18003C12547CC005EF75F01884E5F07F2D7EFB
:100B28002412D3AB7E30743A12D5137E35D0E0123E
:070B3800D3AB02DD517F2D5C
:100B3F007E0590A671127702120E67E5BDA2E67FC1
:100B4F002D12161502DD51D25712DF27121DF31287
:100B5F000B640202937F177E02909E031277027F2F
:100B6F004C7E02909E19127702AC5DAB5C7F577E74
:100B7F000412D358120E8A85BC6285BD63E56124C9
:100B8F00F84044909E237F371276F0AE61AF607CC1
:100B9F00017D5E12547CC3741F9FFAAC63AB62EC91
:100BAF0033921750031255F6125363AB047C003087
:100BBF0017031255F674F52BFB74033CFC125339D3
:100BCF007F377E1512D2D0909E307F697E0F1277BD
:100BDF0002E560240FFBE43561FCA25C923BD25C22
:100BEF007E1E12D2DCA23B925C7E30742012D51393
:100BFF007E36742012D513E5602562FBE5613563FF
:100C0F00FC7F227E0412D358E56245637016742E62
:100C1F007E3A12D51312DD5110000D10011510027E
:100C2F0026020B8C742080E81562E562B4FF0C1568
:100C3F006380080562E56270020563E53524F550AF
:100C4F0003753301020B8C120E8A8562BC8563BD5E
:100C5F00024EE67F637E00747212D50F121E5C4047
:100C6F00087F631276E7124EED0206BE120E71E593
:100C7F00BCA2E77F0A120D34E5BC92E7F5BC02096E
:030C8F00687F1C5F
:100C9200A20D120D31920D80097F25A20E120D3187
:100CA200920E120D5002096B7F0AA20F120D3192A1
:100CB2000F802A7F13A208120D319208801F7F52E3
:100CC200A20C120D31920C80147F25A20B120D3151
:100CD200920B80097F2DA209120D319209120D503B
:100CE2000209A57F49120E67E5BDA2E3120D31127A
:100CF2000E67E5BD92E39266F5BD0209A27F5B1223
:100D02000E67E5BDA2E5120D31120E67E5BD92E553
:100D12009243F5BD0209A27F6D120E67E5BDA2E006
:100D2200120D31120E67E5BD92E0F5BD0209D61231
:100D32000D468F1F9217120E9EAF1F1F7E3912840F
:100D42000BA21722120E7685BC2B85BD2122120E14
:100D520076852BBC8521BD024EE6203714120E711A
:100D620085BE12120D89120E718512BE124EE680D8
:100D7200057F3F120D7B02096B7E0390A24812771A
:100D82000212DD5102DE3275A6FF12DF2712B61102
:100D9200740712DF138FF0740612DF13EF2512C3EC
:100DA20095F0A2E7923D4010FD24CD50027D32AC79
:100DB20005C3743F9DFD800FF404FD24C850027DDD
:100DC20037AC0574402DFD7F4012CA267E1212DE1A
:0F0DD2006C0EBE1EF91F303D020F0FEF6D70ED5E
:100DE100E536700A753606EC2513F5148C13120ED0
:100DF1000712DD51100007100108300207221512F9
:100E01008002051280827F377E28742E12D5137FCF
:100E1100347E21740A303D010412D52EE514FC24E0
:100E21009C50027C637F347E2DEC12CE527F437E38
:100E31001E12D2D87E00E51212D46F7F057E029079
:100E4100A2531277027F6D7E0190A25E1277357FE9
:100E5100747E0490A26F127735021DF375C6F4807B
:100E61003575C6F5803075C6F6802B75C6F78026B8
:100E710075C6F8802175C6F9801C75C6FA8017758C
:100E8100C6FB801275C6FC800D75C6FE800875C64E
:100E9100FF800375C6FD75C70375B9012274721F02
:100EA10012D50F0F02DD517F0A120E9E7E2A1248C3
:100EB100F0120E7BA8BF120EDC10001210010510FB
:100EC100021580F508E824E750EC781880E818E866
:100ED10030E7E3780080DF88BF805F7F097E05907F
:100EE100A532B80C0390A52C1277027E27E53D2888
:100EF100240C75F01884E5F012D3AB7E33743B12E9
:100F0100D5137E35E53E12D3AB02DD517F13120EB0
:100F11009E120D46120F3E10000810010510021717
:100F210080F2105C07205D0BD25C80E8105DE5D299
:0D0F31005D80E1D25C80DD852BBC020356A3
:100F3E00205C10205D1890A5857F127E231277020B
:100F4E0002DD5190A599205DF090A58C80EB90A5C7
:100F5E009280E67F1C120E9E120E76A8BF120F987C
:100F6E0010000810011110021A80F2E824F250034A
:100F7E001880EA780D80E6E824E740030880DE78E2
:100F8E001980DAE8F5BFF54380A37F1B7E26E412B5
:100F9E00D500E82323B464087E26740112D500E43C
:100FAE007E2E12D3AB02DD517F25120E9E120E85C0
:100FBE00A8BCE8120FF112DD5110000810010D103F
:100FCE00021F80EEE824E050E9188006E824CF40A6
:100FDE00E108120E8588BC124EE6D21512D9C880D1
:100FEE00D180157F247E3724E202D41C7F2EA20AE4
:100FFE00120D31920A120D500203597F37120E67ED
:10100E00E5BDA2E4120D31120E67E5BD92E49267C2
:10101E00F5BD0203567F367E00747212D50F0F7E19
:10102E0016743F12D4E1120E71A8BD12109C12DD7F
:10103E005110000810010510021080EFE8248750AF
:10104E0004240A800224E8F880E17F377E1674209B
:10105E0012D4E17E2C743F12D4E112109C12DD5199
:10106E0010000810011410022080EF18B80904783F
:10107E007880E7B878E478E780E008B87904780AF1
:10108E0080D8B8E8D5787980D188BD0209A2E82445
:10109E0087923DE8500224917F367E30C313923BF7
:1010AE0012D41C7E3CE4303B02740512D4F97E1A35
:1010BE0090A47A303D0390A47E1277027F3C7E3A54
:1010CE0002DE6C7F127E00747212D50F0F7E2074BA
:1010DE003F12D4E1120E5D85BE1085BF111211585C
:1010EE0010000810011110021B80F21511E511B449
:1010FE00FFEB75111780E60511E51124E850DE753A
:10110E00110080D91211587F137E20742012D4E161
:10111E007E31743F12D4E112DD511000081001111E
:10112E0010021B80DF1510E510B4FFD875100B8070
:10113E00D30510E51024F450CB75100080C6120EA6
:10114E005D8511BF8510BE0209D67F127E24E51182
:10115E0012D3AB7E30743A12D5137E35E51075F08E
:10116E0005A412D3AB02DD517F49120E9E1211AEB1
:10117E00F81211B410000810010D10021280F218AE
:10118E00B8FF02780480EA08B80502780080E212FF
:10119E000E5D88BD124EE6B800030209D902123E5A
:1011AE00120E5DE5BD227F487E0590A49412770253
:1011BE00E8601CB4040A7E0590A489127702800CA4
:1011CE0090A4A01277027E38E812D50002DD51906D
:1011DE00A49B7E2912770280F31211AE601D640467
:0211EE00601986
:1011F0007F5B120E9E120D46121219120E7610000F
:101200000B10010810020C80EF0209D9105FE9D21F
:101210005F80E5852BBC0209D61211AE601F640405
:10122000601B7F5A7E0590A4941277027E2390A4BF
:10123000A4305F0390A4AB12770212DD5122121189
:10124000AE70030209D97F527E11120E9E120E7BE0
:10125000A8BC12127E120E7B1000081001081002AA
:101260000880EF1880EC0880E9120E7B88BC124ED3
:10127000E6120E85E875F005A4F5BD0209D6121137
:10128000AE604BE875F03270040475F028A4ADF040
:10129000FC305D11ACF0FB7A8A125371EB30E7053C
:1012A0000CBC00010DAE05AF047C007D6412547CC3
:1012B000C005EF7F517E1A12D3C87E2C742C12D534
:1012C00013D0E07E2F12D3AB1241B712DD51227F33
:1012D00064120E9E120E7BA8BD121300100008109F
:1012E000010F10021680F218E824CD50EC783280FD
:1012F000E808E824CD50E2780080DE88BD0209D6F7
:101300007F63E823C2E012CF8575F06484C0F07E6D
:101310002612D5007E2C742C12D513D0E080A47F29
:1013200013120E9E120E71E5BCA2E7923DC2E7F8C1
:10133000E812135E12DD5110000810010D100212A8
:0313400080EE1824
:10134300B800EA783280E608B833E2780180DEE854
:10135300A23D92E7F5BC79A1F78079547F305C0117
:10136300237F127E2375F00A84C0F012D41C7E2DD5
:10137300742C12D513D0E07E2F12D4F90F7E359042
:10138300A59F305C0390A5FB0277357F64120E9E08
:10139300120E7BE5BE7F637E2C128460F5BE79A2BC
:1013A300F780317F37120E9E120E76A8BC530003CE
:1013B3007F367E32E812D50012DD5110000810018D
:1013C3000710020780E718180880E2E5BC54FC48C0
:1013D300F5BCF52B0209687F49120E9E120E85A8F3
:1013E300BE12141112DD5110000810011110021A5F
:1013F30080EFE8240AF8242450E778DB80E3E8242C
:10140300F6F8247F40DB788180D788BE80C6E8F475
:1014130024DC75F00A847F487E3B02D5007F52129C
:101423000E9E120E85A8BF12145812DD511000082B
:1014330010011110021A80EFE82408F8245750E72E
:1014430078A880E3E824F8F824A040DB786080D70C
:1014530088BF0213D7E8F424A923C47F517E3B023B
:10146300D500122C74754A00D210C211D214D27551
:1014730075791475340012DF277F007E0290A22A4B
:101483001277029041E07F087E2612D53FE52B5468
:10149300030F7E3912D500121E0E12D1A9128ED15E
:1014A30012DD5110000810011A10022480C52075A6
:1014B30004057980BE1579E579B4FF05C2757579A0
:1014C3000180B02075EB1579E57970A7D27580A3FB
:1014D300C210C21402096B120E76E5BE7F097E3A72
:1014E30002D500120E7BA8BF120EDC120D46120F9E
:1014F3003EA8BF120F98120E85E5BC120FF17F2D87
:10150300A20A1216157F36A267121615120E5DE592
:10151300BC7F487E3202D422120D467F1BA20D12DD
:1015230016157F24A20E121615120E71E5BC1213A6
:101533005E7F09E5BCA2E7121615A8BF121724E5C2
:101543002B54037F367E3212D500120E7BE5BE7F0D
:10155300637E2C12D500120E85A8BE121411A8BFEB
:10156300121458120E67A8BC021769120D467F09A0
:10157300A20F1216157F12A208121615120E67E596
:10158300BDA2E37F48121615E5BDA2E57F5A1216E8
:10159300157F51A20C1216157F24A20B1216157F6C
:1015A3002DA209121615120E71A8BD02109C120E5F
:1015B3005D85BE1085BF11121158120E67A8BE12A9
:1015C3000AA1A8BF120ADF120AE7120E76E5BE7F50
:1015D3003F7E3A12D500120E62A8BF120A67120E9E
:1015E3005DA8BD1211B4120E7BA8BC12127E120E9E
:0415F3007612121941
:1015F700120E7BA8BD121300120E67E5BDA2E07F95
:101607006C800B7F098040120D467F48A25E744EA6
:10161700400274597E3A02D513127DAD7F73127A58
:101627000B127DFC7F6C127A1A7F2D801A120E67BF
:10163700E5BDA2E77F63121615120E76E5BE7F0998
:101647007E3A12D5007F4812166EB40104BF090115
:10165700E4F51075F005A47E1E909F912582F58212
:1016670050020583027702120E67E5BD035403C2D9
:1016770034C25330E103D2342230E002D253221273
:101687000E9E1F12164E12DD51E5101000121001AA
:101697000610020280ED22045403B4030AE4800713
:1016A700145403B403011423C5BD54F925BDF5BD76
:1016B700124EE680CE1275D1EBF516F5147F6C123B
:1016C7007A1A1275B57F647E23E51612D47FC3E5B7
:1016D700169514F5167F73127A0B7F2D02164E7F1F
:1016E7002E120E9E120E71A8BFE824FA400330375F
:1016F70002780312172412DD5110000810010D1093
:10170700021280E518B800E1780580DD08B806D92F
:10171700780180D5799DE8F7F5BF0209687F2D7EAE
:101727002C7420B80502742E12D5137E32E802D528
:0C173700007F5B120E9E120E67A8BCE83B
:1017430012176912DD5110000810010D10021280EA
:10175300EE18B800EA780380E608B804E27801805E
:10176300DE88BC0209687F5A7E2CE802D500D26865
:1017730075480A1248F0D214122B77127EE5123301
:10178300CFC26B12024A80F3D214751501127D6722
:1017930075B901E5BC20E71C127E9775A6FF127E82
:1017A300F1121E1912DD5112780B10000F500512A1
:1017B300793380E70515E515242050D10206BE12C2
:1017C30017D40202931217D40206FB1217D402098C
:1017D300D91217E0120E768548BE024EE6122B6927
:1017E300122B83125A3612DF2790A039D24912875F
:1017F3004B128704121DC912DD511000141001058C
:1018030010021B80F50548E548640A7002F548801C
:10181300CF1548E54864FF700375480980C28548C1
:1018230049122B83E558221248F0122B6985484947
:10183300C250E558B40F02D250125A36803AD2271A
:1018430075480A122B77125A3612DF2712866E90CA
:10185300A44A20290390A455121E8BC26A1233CFC7
:10186300106A0280E1C227127D3F854948121C3667
:10187300122B83D229125A3612DF27909F4F1287D9
:101883004920500E121E7512DD511000101001AECA
:1018930080F8121E1912DD5110000280FB0206FBB4
:1018A300122B69E55830E7137F1B90A4357E051290
:1018B300770212DD5112DE350206FB122B83125A18
:0A18C3003685594912DF27121E0373
:1018CD0090A45512874912870E12DD511000081091
:1018DD00010A10020C80F512193B80DB12194880A9
:1018ED00D612DF27121E0390A04912874912870EC8
:1018FD0012871212DD5110000810010A10020C801F
:10190D00F512195480DB12196280D6121BFC122BB2
:10191D0083125A3612DF2790A39A128749121E415D
:10192D0012DD5110000510028880F80206FB0559E2
:10193D00C3E55895595003755900221559E5596459
:10194D00FF7003855859220549D3E5491495584030
:10195D0003754900221549E54964FF70058558490D
:10196D00054922122B69E55830E7057F240218AD91
:10197D00122B83125A3612DF2790A0541287491268
:10198D001E8012DD5110000A10010280F8121CA5F4
:10199D0080DE0206FB122B69E55830E7057F2D022C
:1019AD0018ADC26B7559FF125A3612DF27121DF38F
:1019BD00E55930E703121E0E90A066128749128773
:1019CD001E12DD51E55820E7061000081001111018
:1019DD00021B80F00559C3955950CF7559FF80CA28
:1019ED001559E55964FE70C285585980BDE55920D9
:1019FD00E711D26B75A700758307C4F582E0B2E7D6
:101A0D00F080A7306B03121C530206FB122B69E505
:101A1D005830E7057F360218AD122B83125A361255
:101A2D00DF2790A072128749121E5C4009121C9A82
:091A3D00121CCF121A460206FB2E
:101A4600120E7BE5BD75F00584F5BCF5BDF5BEF55A
:101A5600BF120915124EE605C6DFF922122B69E5FB
:101A66005820E7087F5190A07C0218B012DF27901B
:101A7600A460128749121E1912DD5112484FD2ACCA
:101A860010001FE55830E7F8306DF5121B9C7E20DC
:101A96007F00501390A4B212773512DD5112DE3555
:101AA60080CAC2AC0206FB1B8B13909F6B12773564
:101AB60012DD51C26B7B007514B8121C8F127E6644
:101AC600127E185025A814E824384004A6010514EF
:101AD6000BC3E5139B50E678B8121CD1306B03128A
:101AE6007BBD122B83125A368082127DADE51660BD
:101AF600E6D26B127EC3C003127D7ED003A9158089
:101B0600C4122B69E55830E7057F5A0218AD122B2F
:101B160083125A3612DF2790A087128749121E3683
:101B260012DD5110003510010280F8754605121BB2
:101B36006450157F007E357407954612D47F12DDFA
:101B46005112DE35D546E7D390A46B500390A4B26C
:101B560012874912DD5112DE3580B30206FB1248A8
:101B66004F12DC6B745212DC7C745412DC39E5586B
:101B76000475590012DC5A1277BA4016127D3F12CC
:101B86007E9712780B400B0559C3E558955950ECD2
:101B9600C322C2ACD32212484FD2AC12DBC4204CB3
:0D1BA600F1B440F712DBC9B4400312DBC9F3
:101BB300B452E2F53812DBC9B454DA12DBC9FA6065
:101BC300D424EF40D012DBC9E53870C912DBC91247
:101BD300DBC912779F7B007E03127896501020504A
:101BE300B412DBC9204C03B440F7DEED80A7127EAC
:101BF300760B12779FDAE0C322121CE0E55924C862
:101C0300F88602E54924C8F9986013146010500F50
:101C130018E608F618E86970F7A702121CCF22E548
:101C230059640F60F91908E618F608E86970F7A710
:101C33000280E8121CE078C8C250E6B4FF028007B5
:101C430008B8D8F6D25022B8D702D250A615807C55
:101C530078B8121CE2E4F9F5A7758307E9C4F582A5
:101C6300E030E70AE924B8F82438400276FF09C3D4
:101C7300E5589950E7121C9A78B879C8E6B4FF0280
:101C83008002F70908E8243850F2804079B877FFDA
:101C930009E9243850F82279C877FF09E924285044
:101CA300F822121CE0C23D78D7B6FF04A900D23D4A
:101CB30018B8C7F5203D0279D81978C8B6FF0122B4
:051CC300C3E899500781
:101CC800C6C7C6081980F478C8121CF1127ED31250
:101CD8007ED3127ED3027ED378C8121CF1127EB155
:101CE800127EB1127EB1027EB175C703E54875F068
:101CF80004A42480F5C62212DF27C23C1276F4E53C
:101D080037605314604D14604514603D14603514F9
:101D1800602D14602514600E14600B14600D14609F
:101D28001414600C803012160E802B1216BC8026FC
:101D38001215B1802112160A801C1216348017124F
:101D48001620801212156E800D12151B80081214B1
:101D5800E680031214DA12DD5112DE39121DF31275
:101D6800B9D2A81F08E814C23BB51D02D23B75F0D2
:101D780007203C0375F009A4FF7E00303C0C74205A
:101D8800303B02743E12D4E1800A740B303B02747B
:101D98000A12D4F9D8CF12DD51E51D100008100140
:101DA8001010021880B9651F7003751DFF051D808E
:101DB800AE7005851F1D80A7151D80A375F003A4AF
:101DC800227F7B7E0090A3B2127735E54824F64047
:101DD800087E0A90A41812773522127A377E057485
:101DE8005B12D4DD7E1D745C02D4DD121DE27E34EC
:101DF80090A3C3027735127A378003121DE27E3131
:0E1E080090A3C7027735121DE27E3190A4BD73
:101E1600027735127A377E008005127A377E2D904A
:101E2600A4BD027735121E367E31909FA502773506
:101E3600121E197E1A909FAA027735121E1980C0AB
:101E4600121E197E18909F58027735121E197E1A97
:101E560090A4C2027735121E197E1A90A4C7127773
:101E66003512DD51D3100006C310010280F622128E
:101E76001E197E1A90A043027735121E197E1890FD
:101E8600A05F0277357F007E2012773502DD511282
:101E96007A3790A4CC027733127A3790A4DC027793
:101EA6003312BE94120E94E5BDF55EF56CE5BCF5F5
:101EB6005FF56B756A007561FF75A70490070012E0
:101EC600BE3EB4FC23E582C313F561E56CF0E56B19
:101ED600F0E582600F12BDB5E56C655E70E1E56BFD
:101EE600655F70DB75A700223024EA0460E7240FE3
:101EF60040D380E1E560758307C333F582E0A3F53F
:101F06006CE0F56B756A0022D2248002C224D214DA
:101F1600C21F121EA7756000E561B4FF1612DF2707
:101F2600909E337F0A7E0512773512DD5112DE321E
:101F3600020293C210C21112DF27121DF3301F0ACC
:101F46007F07909E4212773380647F007E01C3E54F
:101F56006012D47F7E0E742812D4DD856048740723
:101F6600F51FFF7E00743E12D4E1E548121EFC12F6
:021F7600C8356C
:101F78001224D80548C3E5619548FD401CE51F2497
:101F880007F51F24C850E17F387E01ED0412D47F85
:101F98007E0E742912D4DD800DE51F2407FF7E0113
:101FA80090A4BC127735201F0312251B12DD511097
:101FB800001910012C10020280F5120236301F3D64
:101FC800020282101F02D21F021F39E56160F4E588
:101FD8006065617005201FF080E9201FE6056080BC
:101FE800E7E56160DEE56065617005201FD5800961
:101FF800201FD5E560700280CA156080CB121EA72D
:10200800121EFA12C83512260F756A1012BE271250
:1020180026C6909E4CD23C1276F4121D649020295C
:1020280073021F3902330F022049022035121E5C49
:1020380040CB121EFA12BE3EC2E2FF12BC64021F5F
:102048001212DF277F6490A6941276F07F7990A60B
:10205800A11276F012DD5175160010000A10010960
:1020680010020280F505160516C253121EFA12C890
:102078003575370A909E68121CFF902086730220DF
:10208800050220AD02227C0222810220710220B4C6
:102098000220B90220710220F70220FB0220FF0271
:1020A800210602210A7F0A12168680BD124868801E
:1020B8000312485D780A1221D9740912DC371222FA
:1020C8001812DC5312225312BE2712BE4F12BD76CD
:1020D80012BF66122362D5150C75150A12226612F4
:0C20E800248912DC53100204E57F70DB39
:1020F400022005780A800678048002780112486874
:102104008009780A8002780112485D1221D9740985
:1021140012DC2C122218E54812DC18E5165403448C
:102124003012DC39742A12DC3912DC3912DC531215
:10213400225312BE2712BE4F12BD7612BF6612235F
:1021440062D51548854815122266E51C12DC18E58F
:102154001B12DC18E51B2548F51BE4351CF51CE4B3
:10216400A27792E7A27492E0A27392E112DC18AD16
:1021740075AC74AB73E57DC412219AAD78AC77ABC2
:1021840076E57D12219A1224A712DC53100204E58D
:102194007F709F022005540F2375F00584F8C3EB6C
:1021A40033FBEC33FCED33FDC3EB33FBEC33FCEDE1
:1021B40033FD20E713EB28FBE43CFCE43D12DC1880
:1021C400EC12DC18EB02DC18C3EB98FBEC9400FC7B
:1021D400ED940080E88848121E20E4F54AF549751C
:1021E4006A2075150112BE2712BD76D5150E8548D5
:1021F40015E5492401F549E4354AF54AE57F70E5DA
:10220400744012DC7C747812DC39746312DC397427
:0F2214002102DC2C122464E56012DC18121EFA81
:1022230012C835E53A12DC2CE53B12DC2CE53C12F6
:10223300DC2CE53D12DC2CE53E12DC2CE53F12DC08
:102243002C740112DC18E54A12DC18E54902DC188B
:10225300121EFA756A20E4F51CF51BF514F51375C7
:10226300150122753800E51412DC18E51312DC1889
:102273000513E513700205142212486880031248FF
:1022830052121E201223BC12DE3D756A2075150101
:1022930075A6FF754A0112BDCF12BD7612BF661235
:1022A3002362D5150975151E12238612DE471224E3
:1022B30089E57912DC18E412DC18E5711223471260
:1022C300DC18E57012DC18E57B24ACFFE55F34090C
:1022D30012DC1EEF12DC18E51520E033857D56E491
:1022E30012DC18E52EC412DC1E12DC6212DE47106B
:1022F300021A30559B744012DC39744512DC397470
:102303004F12DC39744612DC3912DC62022005E517
:1023130056122321C4FAE57D1223212A80C2FBC46D
:1023230012232E2323CB12232E2B22540FFC24F60D
:1023330050027C0090233DEC932200000101010236
:1023430002030303FA2440400A24804003EA3322B1
:10235300D2E72274FF2220E703C3132224C022E51D
:102363003F701F7F7B7E0078AEE612D469EE2404B3
:01237300FE6B
:10237400743A12D4E1EE2404FEE53E12D46312DD75
:102384005122C015C016D21212A6ECC212D016D019
:102394001578AEE612DC2CE53E12DC2CE53F12DCAF
:1023A4002CE54512DC18E55212DC18740A12DC180C
:1023B40074C012DC1802DC62744012DC39745412EA
:1023C400DC7C744E12DC39743012DC39E5165403AB
:1023D400443012DC39122464742112DC2CE53D12E1
:1023E400DC2CE56012DC18121EFA12C83578ABE654
:1023F4000812DC2CE60812DC2CE60812DC2CE612AF
:10240400DC2CE53E12DC2C1229EFE51212DC2CE563
:102414001112DC2C740112DC1890A4ED1224C9757D
:102424006A1012BE27057F057F787F12DC11787B46
:1024340012DC11787D12DC11787712DC11E4FEFFD6
:10244400780712DC1112DC11E57412DC18E5751240
:10245400DC18E412DC18E412DC1812DC1102DC6271
:1024640075C70375C6FF75B901C217751D0085BC14
:102474001C85BD1B85BE1A85BF191252E9EE12DCFC
:1024840018EF02DC18E57512DC18E57412DC18E5A7
:102494007312DC18E57812DC18E57712DC18E5769F
:1024A40012DC18E51664016011E55E12DC18E57AA9
:1024B40012DC18E516640260012278BCE612DC180E
:0A24C40008E602DC1875A700E49397
:1024CE00700122A312DC391A80F4AF1F7E0478AD9E
:1024DE00E612D4637E0C742C12D4E17E0E18E61232
:1024EE00D4637E1A78AEE612D4637E22743B12D485
:1024FE00E17E24E53E12D4637E2FE54012D4697E40
:10250E0037743B12D4E10E0EE54102D463753200EE
:10251E00121EFA12C835857946787A796412C84E39
:10252E0074641256DE8E4712260F756A20D23D1243
:10253E00BE2712BE4F122646303D09307406C23DEC
:10254E008E1E8F1FE57F602BE54C24FFF54CE54D6D
:10255E0034FFF54D454C600512BD8B80D2751D3C88
:10256E0012BE2712BE4F12BD76122646E57F6003BD
:10257E00D51DED1226A79026BF12D53F203D0DAEDC
:10258E001EAF1F1226A79026B812D53FE546FD7046
:10259E000B90A623305D1190A61F800C0470109036
:1025AE00A61F305D0390A61B7F381241B2804BE40C
:1025BE00FFFC7E05305D047E027FB312546FAC06C5
:1025CE00AB071253397F38C23DE51C6007D23D7E02
:1025DE002C12D4CEE51B203D026007D23D7E301278
:1025EE00D4CEE51A203D026007D23D7E3412D4CE01
:1025FE00E5197E3812D4CE1241B7E53224C850FA0E
:10260E0022E54075F03CA42541FFF54CE435F0FE83
:10261E00F54D7C007D1012547C0F8F4BAF4CAE4DA0
:10262E007C007D3C12534F7C00AD4B12547CEE4F20
:10263E0070010F8F4C8E4D2278647973C2D11226A1
:10264E005DFF78677976D2D112265DFE02DE6CC30D
:10265E00E796FB0809E796FC0809E796FDA2E792C4
:10266E001750031255FE75135A30D10E751320B242
:10267E0017AA47125383AB04AC05E546600B046002
:10268E000BAA4612539AEB03FBEB03FBEB543FFBF7
:10269E00E5132B2017029B9B22EE141430E701E466
:1026AE00FEEF141430E701E4FF2205057088A888B8
:1026BE007005052020F8202075320012DF277E1EBF
:1026CE007F1C12DE6CDFFB12DE6C7E1E7F1C12DEA8
:1026DE006CDEFB7E1D7F1D12DE6CDEFB7F007E211D
:1026EE0078ADE612D4637E29742E12D4E17E2D18B5
:1026FE00E612D4637E35742E12D4E17E3918E612BA
:10270E00D4637F077E21745412D4E17E25744F1258
:10271E00D4E17E2D78AEE612D4637E35743A12D4AF
:10272E00E17E39E53E12D46378AE1229EF7F0E7E3C
:08273E0021744C12D4E17E2548
:10274600744112D4E17E2DE51212D4637E35743ABB
:1027560012D4E17E39E51112D4637F157E257444C7
:1027660012D4E17E2DE54012D4697E35743A12D436
:10277600E17E39E54112D4637F217E0190A5EE12F8
:1027860077357E0EAC77AB7612D3157E2B85795FC7
:1027960085787B12D8BC7F287E0190A5F21277350A
:1027A600751D2B751E10E5741229A37E25742F1234
:1027B600D4E1751D2D751E2BE5751229A37F367E76
:1027C6000290A5DE127735E5721228501228E8121B
:1027D6001EFA756A209004E6E56CF09004E7E56B56
:1027E600F0AE4DAF4C7C007D4012547CBF00010F13
:1027F6000FAC07AD07E4FED23D12BE2712BE4F1244
:102806002891E57F602CE54C24FFF54CE54D34FF1F
:10281600F54D454C600512BD8B80DE751D3C0E12D4
:10282600BE2712BE4F122896E57F600612BD76D5EA
:102836001DED1228667F7812CA387F767E007430C6
:1028460012D4E1E53224C850FA227E2112CF851235
:10285600D47F7E2F90A5F6305D0390A5FB027735D9
:102866009004E6E0FD9004E7E0FCC3E56A9420FBF3
:10287600E56B9CFCE56C9DFD50032410FD12556E26
:0D2886009004E8EEF09004E9EFF022DD038D
:10289300AD040E7F78E55E20E72AE57A8549F0A44A
:1028A300A9F0E57A854AF0A429F9E435F0FAE55E62
:1028B3008549F0A429E435F02AFAE55E854AF0A4B7
:1028C3002ACF9FFF12DE6C103D18C3EF9B50131BE2
:1028D300EF6B600E8F018B0712DE6C1FEF6970F8D0
:1028E300AF01AB072290A5A3305C0390A5BC754A4A
:1028F30040754900AF76E577FE20E76B7005EF245E
:10290300105064EF24A8EE34FD401190A5A8305C6C
:102913000390A5C0754A1975499A8075EF2450EE46
:1029230034FB401190A5AD305C0390A5C5754A0CEE
:102933007549CD805CEF24A0EE34F6401190A5B02C
:10294300305C0390A5CA754A067549668043EF2437
:10295300F0EE34F1401390A5B3305C0390A5CF752E
:102963004A04754944802A8028EF2490EE34E840D5
:102973001190A5B6305C0390A5D4754A0275498FB2
:10298300800F90A5B9305C0390A5D9754A017549AC
:102993009A7F401277337F4612CA387F5F02CA3864
:1029A300AE1E75F064305C0375F03284C0F0F870CD
:1029B30004EE2404FEE51D12D4E1EE2404FEE860D7
:0129C300070C
:1029C40012D4CEEE2404FED0E075F00A305C037518
:1029D400F00584A8F012D4CEEE2404FE742C12D494
:1029E400E10E0EE8305C012302D4CEE53E2541F52C
:1029F4001124C45003F511D3E63540F51224E850F0
:102A040002F5122212B9CCC21012DF277F057E090B
:102A1400909C6A1277027F137E08902A3C12D53F5D
:102A24007F2B7E01902AA412D53F20370A7F277E70
:102A340027902B1612D53F22113007FE1FE001E12B
:102A440001F80F00061B00F80C00180E007C1000A3
:102A54007006003C2000E006003E4001E004001E39
:102A64008003C004001F0003C004000F000780009F
:102A7400000F800780000017800F00000027C00FA0
:102A840000000043C00F00100083E00F002003018A
:102A9400F00700C00F01F80383007F87FE01FC00EC
:102AA4000E3E1800000300000000180000030000A0
:102AB40000003800000000000000300000000000AA
:102AC4000000FC761F0E1C6030ECFCBC3F172DF0A0
:102AD400F978613866264F619A706070C60E1EE3FD
:102AE40030E06060C60C1CC360C0E0618C0C18C789
:102AF400C0C0C0E18C1C39C611C0C4C19C993196B8
:102B04003180C8C1FF1E31E7E180F0C0EE1C31C343
:102B1400818006163091882892884924904927900C
:102B24009248A0E3C8BCC2AFD2C075C0107581D8AA
:102B340074FE122B42E4F5F9F5FBC2B480F7D2A679
:102B4400C2A512B9B112DE3902B9D275C703E5487C
:102B540075F004A42480F5C6C23C75B901E5BC0433
:102B64007002D23C22120E76E5BEF54824F65003DC
:102B7400754800753400753704C228D229D22A75E5
:102B8400C703E54824E75003754800E54875F00499
:102B9400A42480F5C6751607751700C23C122BC411
:102BA400122BC4122BC4122BC485175815587559EF
:102BB40000E548B40A09E5586005F46002055922A5
:102BC400203C1D75B90105C6AABCABBDACBEADBFEA
:102BD400EA122BE5EB122BE5EC122BE5ED122BE5BB
:102BE40022203C07F515B4FF03D23C22C0C7C0C65F
:062BF400127D6775A704C5
:102BFA00851683E517C4F8F58275B90105C6E5BCE3
:102C0A00F0C582F82406F92403C582E5BDF0E5BEC5
:102C1A00F0E5BFF075B90105C6E5BCF0E5BDF0E524
:102C2A00BFF08516838982E4F075B90105C685BCB3
:102C3A001385BD14E4F0F08882E5BEF0E5BFF075B7
:102C4A00B901E5BCF0E5BDF0E5BEF0E5BFF075837E
:102C5A0006E51723541E24B0F582E513F0E514F0B7
:102C6A0075A700D0C6D0C705172212BB9478BEA696
:102C7A004808E4F6F55908761808F6D23608760AAE
:102C8A0008F6060876BEC254C25512BEA9122B77A0
:102C9A00C229C22AC207C227C268120E67E5BDA2AC
:102CAA00E59243C24AE4F52EF534F536F52F78B6A7
:102CBA00F678B5F678A9F6789EF678B8A65E08A6EC
:102CCA007A12D27EC26BC233C238C240C223C22237
:102CDA00122CF475460278C5A646C23AD221C21908
:102CEA00C226E4F542F541F54022E45407205E0984
:102CFA00B4040040027403801B120E6CC313A9BCF7
:102D0A00600C14A9BD600714A9BE6002A9BFE940FE
:102D1A0001C45407F53722122B69125A3612090CCC
:102D2A0012DF27121E41E55804700A7F327E059091
:102D3A00A43512770290A68B12874B1208667F720F
:102D4A0090A6801276F012DD511000051002048060
:102D5A00F8D322C3220200F7120E67E5BD20E70569
:102D6A00122D2140F0754E50122C7412852C754488
:102D7A00031248ED12AF11D54403022B2A201EF18B
:102D8A00789F7680754A0012BCC5D210C211C21350
:102D9A00C21212483F75A60C12D9C812C4B3E5A6CE
:102DAA0024FA400612488D75A60C20250CE590548D
:102DBA00057009E53524E25003022E54E532241841
:102DCA00400D75F00C84E5F070D41233D280CFD266
:102DDA001ED2AC306DC87532F012DBCEB4E0BF1231
:102DEA004935E53124F39205201203123264122E7A
:102DFA001AC014128E17D014200A03122F3D123350
:102E0A00D212A6BB1233D212852F1233D2022D9CB4
:102E1A0030122EE54024F0401C7A0AC3E53F954B58
:102E2A006013401E24E2400D305405C254757F01E0
:102E3A0012BCEBDAE679BCE7D2E7F57F09877EC2F6
:102E4A007722F40424E250ED80DE12DF277F2A7E07
:0C2E5A000E90A4F112770275A6FFC210C2
:102E66001012137F367E08909F8812770212DD516A
:102E760012DE320200F7D22112491112BCF57F1E72
:102E86007E0B90A40E12770212DD51122EA77F3E02
:102E96007E0790A12812770212DD5112DE2C022B3A
:102EA6002AD215D21412BE80120D4675B90575B90F
:102EB6000212BE8AD25512BDAF7F0012BC6412BE8A
:102EC6008AE56A600512BD7680F7857A62120E94ED
:102ED60085BEBC85BFBD856BBE856CBF75B90575E6
:102EE600B90285BD6C85BC6B756A2012BE80123036
:102EF600DE12BE8A756A0012BE27E57064FE703463
:102F06007570FC854077854178851F797818797AC0
:102F160012C84E12BD2412DE4712BE8A756A1012FE
:102F2600BE277F087810797212C85085627C855E4C
:102F36007D12BD24C2152212486812308A745212BC
:102F4600DC39744D12DC39744312DC3912309912B3
:102F5600DC747441207402745612DC39122FE612A6
:102F6600303012DC74E53C12DC2CE53B12DC2CE53F
:102F76003A12DC2C12306612DC74744512DC3912FB
:102F860030CF12308A744712DC39744712DC397438
:102F96004112DC39123099122FE612DC74E43074D7
:102FA600010412DC3712DC749004C3E012DC2C122C
:102FB600DC749004E4E075F00A84AFF012DC2C12A5
:102FC600DC78EF12DC37AC5EAB7A1230ABAC5DABC3
:102FD6005C1230AB12DC7412DC741230CF02483F44
:092FE6007875C23D122FF17878D4
:102FEF00D23D12DC74128211303D05E51E12DC3722
:102FFF00E51D12DC37123073E51812DC37E57D2042
:10300F003D01C4540F12DC3712DC74303D09744596
:10301F0030170274578007744E301702745302DC56
:10302F0039207408123066123066802775A7049015
:10303F0004BFE0FCE0FB7A1B125371783212551378
:10304F001253391230709004C1E0FCE0FB12533977
:10305F0012307075A7002212DC74E4F51AF519808E
:10306F000D12DC74E51C12DC37E51B12DC37E51A98
:10307F0012DC3712DC78E51902DC37742412DC39E4
:10308F00744712DC7C745002DC3912DC74E53D129B
:10309F00DC2CE53E12DC2CE53F02DC2C12826D129B
:1030AF00DC74E51D12DC39781CE612DC3718B81712
:1030BF00F812DC78E412DC3712DC74744D02DC3960
:1030CF00C038742A12DC39D03812DC5302DE47784C
:1030DF00107F0EE4F608DFFCF564F565F567F5681B
:1030EF007515FC751AC0751DC075664075694075FC
:1030FF004A0112BDCF30550302319412BD76E571EE
:10310F00B510004002F510E4F511E512207502E547
:10311F0013C395795006207545857913D3E57A95B4
:10312F0014E5156480FFE55E64809F400C857A147A
:0E313F00855E15857B16855F173074B3C2D18F
:10314D007864797312317278677976123172D2D1CF
:10315D0078187973123172781B79761231728091E9
:10316D0085791280B9D3E7960809E7960809E664D0
:10317D0080FFE764809F20D101B3400AE7F618195C
:10318D00E7F61819E7F622E51AB4C00E7873791828
:10319D0012C84E7873796412C84E78187964C2D10A
:1031AD0012320574181256DE8E47AE1EAF1F781BF5
:1031BD007967D2D1123205C3E51F9FE51E9E5004DB
:1031CD008E1E8F1F7EFF7FFFAC1EAD1F12547C7AAB
:1031DD0004EF8AF0A4E5F0CE8AF0A42EFEE435F0DB
:1031ED00BEFF011E60051460057EFF8E1F22EE7E60
:1031FD000020E7F77EFE80F3C3E697FB0809E6970C
:10320D00FC0809E697FD1818191930E7031255FE49
:10321D00C3EB33FBEC33FCED33FDEB33EC33FBED68
:10322D0033FC30D105AA4712539A0BBB00010C7524
:05323D001E03751FFFD8
:10324200EC24FC40048C1E8B1FE627FB0809E637A2
:10325200FC0809E637A2E713F618EC13F618EB138D
:10326200F62210131978B5E624FA401AE57124F60D
:103272004008E57924F6400280360606803212DEE6
:1032820043E59030E2DF753612D22EE4F534F55A7A
:1032920012BEDB1232B5C219C257122CF412914679
:1032A200129173D212853F4B754C00205E02D228D8
:1032B200022CECD214123304E6F008DFFB857A62AA
:1032C2001232FA7570FE783A797112C84E12BD2424
:1032D2001232FA85627A855E7B120E8A85BC7E8501
:1032E200BD7F7570C012BD24123304E0F608DFFB07
:1032F20075A700D254C2142274FF7870F608B88001
:10330200FB2275A7049004F078707F1022121EFA37
:10331200122C7412DF2712DD51C258C259754A01AC
:10332200753901756A2012BDCF1256DC8E47C21064
:10333200D211D214D21212BEDB1291461291731222
:10334200D9C875A6FF753609753200E59020E206E8
:10335200E5352405400CE5905405701FE53524E25F
:103362005019C211C21212DF2712DD51E4F535F5F0
:083372002F7E0612DE3FC202AD
:10337A00022005C221E54AB40202D22112BDCF12AF
:10338A00A6BB30260F125A9812852F753606E536D7
:10339A0070FCC22612852C1233D2E54A20E021B4F1
:1033AA000209753900E53670F9808CE53960FAFD55
:1033BA0024E24002053912BDCF2026C9DDF880E992
:1033CA0075390080E475370410003A1001161002AE
:1033DA0016E52F5407600312B9C620783D20790AF2
:1033EA00207A1F220235C802351CE53760091460AD
:1033FA00091460090236740235E7023645C27902B9
:10340A00369102354FE53724FC500FE537640760E3
:10341A000302370C0236D00234E62011FAE5902076
:10342A00E2028056753400201203D2132278A9E6EC
:10343A007017C226767DE5377005106B02D26BD203
:10344A0077753614D22E02BED0E537604314604039
:10345A00B40227200B24E6249B401F2414501C127C
:10346A00914690A3DE7F207E0812770212DD517505
:10347A003608D22E78A9E624ECF622241940FB2439
:10348A001450F712914612917390A3E87F2980D7BE
:10349A002028E7E54824F640E1E5580460DC7F5D32
:1034AA007E10E6249B40D324145015C2330559C319
:1034BA00E55895595005855859D22690A3CC80A92C
:0434CA00241940B6CB
:1034CE00241450B2E55960021559102606E55960CC
:1034DE0002155990A3D5808D10780122753900E51B
:1034EE003424384007754A0175340022700AE54AC3
:1034FE0030E0F2754A0280F0146008754A061291A7
:10350E00738006754A0412914675390180DA3029A6
:10351E0009C229D22A7559008005302A1BD22912D8
:10352E0086FA1286C8E53524AF400475340022753C
:10353E003700C229C22A80F3206841302703D26A9D
:10354E0022D2221238A812DD51107A0122E534243B
:10355E00384007122CF475340022700FAA37122C43
:10356E00F46A70F27401122CF580EB04122CF5241F
:10357E00FC50E3E537B40706D22880DA8036C2283D
:10358E00E53724FC2324BEF879C4E7F9A74809A738
:10359E005979C4E8F78648088607E537B4050575F6
:1035AE004818D236122B838F59E53764067002D233
:1035BE000702356412388402382EE537601B14601A
:1035CE007614600F146009E53724F9400902378636
:1035DE000236740236BF023753D223124096107948
:1035EE000122E534243840077546017534002278EF
:1035FE00D87020304A0BC24AE624F85004B24380F9
:03360E000AD24A93
:103611007614E54624FE40DDE54660D9154680D89E
:10362100B600D5B40500500C04F54624FA50C9750E
:10363100460580C424F95005127B5B80BB100FB88E
:10364100D20F80B4D223E53464C8600312409610CF
:10365100790122E534243750097011105B32D25BB5
:10366100802E100802D2081240968024100C21D21C
:103671000C801DD22312409610790122D24BE534E1
:1036810024374010C258C259201105D22E75360771
:103691007534002224FD401524037006D258C25906
:1036A10080EEC258D2591460E7D25880E3120E71ED
:1036B100E5BCB2E7F5BC79A1F7124EE680D278B845
:1036C100A65E08A67A2011C8753605D22E80C130B3
:1036D100122B128734055BE55B75F00B84E5F0F581
:1036E1005BE55A24F64009E55A955B5003755B008A
:1036F10012873812DD51E5346003D534D2753400B8
:1037010022D229D22A75480A0237F4C2401007F1A1
:103711003029030237F41286F612870A102A1BC2D7
:10372100330559C3E558955920E7025008755900EA
:10373100E548B41816E558B4FF0375590012871E01
:1037410012DD51E5346003D534C122D22A1286FA42
:1037510080EE301223128734155BE55B30E70C7580
:023761005B0A01
:10376300E55A24F64003855A5B12873812DD51E58A
:10377300346003D534DA75340022D229D22A75484D
:1037830017804CC2401007F22029441286F6128794
:103793000A102A22C2331559E55930E71C855859B6
:1037A300E558B4FF03755900E548B41802800AD2FE
:1037B3002A1286FA800E855859E558B4FF037559C5
:1037C3000012871E12DD51E5346003D534B5222083
:1037D300106220115F7F180548E54864187008F5EA
:1037E3004830270375480A122B4F303C2DDFE88001
:1037F3002620105A2011577F181548E54830E70551
:10380300754817800A640970063027037548171234
:103813002B4F303C05DFE275480A122B83125A36D0
:10382300E532244C50051286C8800312866E753427
:103833000002DD5112386B7F15E5486B70048A482E
:1038430080020548122B4F303CD0DFED80CC12387C
:103853006B7F15E5486A70048B4880021548122B6C
:103863004F303CB6DFED80B27A007B09E537B40414
:1038730001227A0A7B17B40601227418FAFBF54871
:103883002275A704758307E559C4F582E0E0F57353
:10389300E0F574E0F575E0F576E0F577E0F5787539
:1038A300A700025A36E59020E23EE534243750382B
:0638B3001238EC1238C9C6
:1038B900205E4F7F2C909D22123933909D2B806A78
:1038C900E534243775F009A42435FF205E0624BEAB
:1038D90050027F3EEF249B50027F627E3274891230
:1038E900D5132275A7049000317E087F3AE4F0DFF2
:1038F900FDE5822446F582E43583F583DEED75A77F
:1039090000227F2C120E6CE5BD12391CE5BE12395E
:103919001CE5BFF8C4123922E8540775F009A490D0
:103929009D102582F58250020583EF2409FF027656
:01393900F09D
:108529000285E312DF27E53724FC40F4B4FE14206A
:10853900110EE590F45407600122E532247450EFDE
:10854900028E2312DF2712D6B612D74812CF931202
:10855900D2D412D11D7E197F3612D07112DC81124C
:10856900D087C206E53760051460338053C23A12DA
:1085790086871241591242EE1245D41264F41265EB
:108589001C123E04E54864186009E54824F65003C6
:108599001246BF128DB912CE181241F48014D23A84
:1085A9001286AD1239421241C312C99E128DB912F7
:1085B900CDD9125D7712D78F125848125B478012B6
:1085C90012869312C8DB12D85F12C96D128DB912C7
:1085D900CDF030101112D025800C12DF27E5372499
:1085E900F9401E1286703022091238A8E53470024B
:1085F900C222302309124096E5347002C22302DDFB
:1086090051121DF375170012DA727F1212CA263041
:10861900124A75100075A704758306125AF1E51000
:1086290075F009A42415FFF5177E00E512602F7572
:10863900F06484E5F00F12D4631F7E0EE51112CFAA
:10864900DB751623125CAD0510C3E55A951040067B
:10865900E51024F550BF3012031287388088745D05
:1086690012D51380D5C249302905121DC9800312BC
:108679001DF3909F4F12874B202A7602871E3012D6
:1086890023305E2030501D028A2F301217305E06CB
:03869900200B11A2
:10869C0002909012CA1F7F1712DDC775172002DADD
:1086AC007212D62D12D5CE30121120510512D68D44
:1086BC00800612CD7312CB531251AB22E4FEFFE5B0
:1086CC004824F6400D90A4181277357E16E5480222
:1086DC00D4CEB40E0690A41E02773590A425127742
:1086EC00357E12E54824F702D4697D20800C7D3F4D
:1086FC00302A077D633029027D3C7F0080247D2059
:10870C0080127D3E800E7D3CE54975F007A4240661
:10871C00800A7D3FE55975F007A42409FF640270B7
:10872C0001FF7E1CED02D4E17D2080027D3FE55BE4
:10873C0075F009A42416FF7E09ED02D4E1C249129A
:10874C0087AFB4FF01227510001287C67920E03084
:10875C00E702792F3049171211AEFAB40408E5106C
:10876C00700C79658008EA14651070027923E97E33
:10877C001812D4E17E20E51230E708909F8812771A
:10878C00358016E51112883C125D0D201005201164
:10879C000280063012031287EE0510C3E5589510BF
:1087AC0050A7227E207F001277351286C87E007F6C
:1087BC000690886E12D53FE5582275A7047583077D
:1087CC00125AF1E51075F007A42409FFF5177E0085
:0B87DC00E51212D4E17805EE2404FE43
:1087E700E012D4E1D8F6221288F612890CFD7C003B
:1087F700AE1CAF1B12546FBE003A8F00C3E57A95CB
:1088070013FFE55E9514FE402B7C007D2812547CF7
:10881700C3EF98401F75F0058404FB24F950027BD1
:10882700067E2CAF170F12DE6C0F12DE6C0F12DEF6
:108837006C0EDBEF2264B4602464B475F03284C03C
:10884700F012D4CECE2404CED0E075F00584C0F06B
:1088570012D4CECE2404CED0E02302D4CE90886AA0
:108867000277352D2D2D000140FFFFFFE0FFFFFFB1
:10887700FFC25030123F20283CE558F460372048AB
:1088870003200931D250E559F51030330665586099
:108897000205101288C012891C75A7049006DCE532
:1088A70012F0E511F0E517F0E510F075A704900652
:1088B700E0ECF0EBF075A7002275A70475830712AB
:1088C7005AF17813E0F608B819FA9006D07811E64D
:1088D700F008B819FAE51CF516F0E51BF515F012C6
:1088E70088F69006DAE514F0E513F075A70022750F
:1088F700A704758306E51023541E24B0F582E0F51E
:1089070013E0F51422120E71E5BD2487E5BD923BF5
:0289170050020C
:1089190024912212890C75F005A485F012F511E451
:10892900F519FEF51CF51D12BE80C23DC2567F3CED
:1089390012CAC9303D05751900807DDFF3E5596517
:1089490058700A301007EE24D35002D2568C1B8D72
:108959001AE519FD24E250DEAE1CAF1D7C0012544D
:108969006FEFF51924F650CEAC1BAD1A12CA0E20C2
:10897900D1108E048F05E51975F0A7A4AEF0FF128A
:10898900546FAC12AB117AA012539AEB33FBEC3350
:10899900FC20D11AEF9BEE9C5014C3E51213FCE5A1
:1089A9001113FBC3EF9BEE9C4004AC06AB072048B8
:1089B90007203B048C128B119006E2E519F0128A0C
:1089C90004AC16AB157AC8125371A912A811125525
:1089D90015ED7005EC249E50057C807B0822C3E5CB
:1089E9007A305602E55C9513FFE55E305602E55D87
:1089F9009514FEC3EF9BFBEE9CFC22AE16AF157CD3
:108A090000E519FD24F6501A12546F7C007D0612F8
:108A1900534F7C007D0512546F8F10EEF51724E932
:098A290050037517FF2212CA1F49
:108A3200128A4C128A8F12D283128AB520480912E6
:108A42008BA3128BD3028C3680747F177E20204832
:108A52000E748A204D101258B5500E742F80077470
:108A62006A305F02746712D51375A7049006D07836
:108A720011E0F608B819FA7F177E00781275190509
:108A8200E60812D513EE2406FED519F42275A704C2
:108A92009006D8E0F516E0F515E0F514E0F513E0E0
:108AA200F512E0F511E0F517E0F510E0FCE0FB75DA
:108AB200A700227F187E26AC14AB1302D3159006B2
:108AC200E4E0F51CA3E0F51B7F2A304E13120E677B
:108AD200E5BF90A482B4010390A67A1276F0804298
:108AE2000F7E00745312D4E19005CBE0F830E70515
:108AF200E53F30E0091F7E00E8540F12D4F99004DC
:108B0200EEE0FEF51EA3E0FFF51F128B4BE51E24DF
:108B1200E9500C7E06742B12D5137E0C12D513125B
:108B22008B7BC20375172A751627125C7C202415CD
:108B3200205F15D2037F2A7E1E908B69304E0390F0
:108B42008B7202D53F205FEB227C007D3C12547C6D
:108B5200A805EF7F2A7E0812D41C7E12743B12D520
:108B62000F7E14E802D4160707384C9EBAF2643816
:0F8B72000707387CE6C2E67C38AC1CAB1B7A48A0
:108B8100305D027A27125371A91EA81F125515EDE7
:108B91004C60027BFF7F207E28EB12D4227E3902BB
:108BA10091237F2B90A42B127733E517F46022AE2B
:108BB10017AF107C007D3C12547CA805EF7F2A7E04
:108BC1000C12D41C7E16743B12D50F7E18E812D4F9
:108BD1001622AE12AF117C007D0A12547CA805EF5B
:108BE1007F207E3012D41C7E3A742C12D5137E3C29
:108BF100E812D4F90F7E29744502D4E17485800707
:108C0100748720560274867E2912D5133017077493
:108C11002D7E3A12D513227C007D0A12547CA805C0
:108C2100EF7F2A7E3012D41C7E3A742C12D5137E2B
:108C31003CE802D4F9128D67E54824F65005128C00
:108C41001880B9E559046558600D128C18128BFD16
:108C5100E559655860AA22A217923D8E1E8F18858C
:108C610015179006D0E0F51185581015101245B46E
:108C7100C3E51195105002F404F924A65005C374FC
:108C8100B399F9E975F00584F924EE500279119050
:108C91008DA7E993F5F0120920E5CC7004E930E7DE
:108CA10002747F23A4A9F0E51B2517FDE51C3516E9
:108CB100FEC3ED99F515EE9400F51675A7007583C1
:108CC10006E55823541E24B0F582E0A3F513E0F520
:108CD10014128D67203D2C201729120E71E5BD2439
:108CE10087E5BD5002249175F007A4FB9518E5F0C6
:108CF100951E400FEB9FE5F09E4008EF9518EE950D
:108D01001E500EA23D9217AE1EAF18128C18028B88
:108D1100FD306B10128D04E53F20E00774867E2242
:108D210012D5132275A7009006E0E516F0A3E5150C
:108D3100F0128C18128C0174857E2312D51385587C
:108D4100101288C0128A4C128A8F8C168B15128AC7
:108D5100B51289CA1288B212D2839006E2E0F519DF
:108D6100128A04028BA3C3E57A305602E55C95139F
:108D7100FFE55E305602E55D9514FE921750031231
:108D810055E6AC16AB157AC8125371A906A807129D
:108D910055157E037FE7ED700CEB2418EC34FC4095
:108DA10004AE04AF032200172E43576C8092A4B681
:108DB100C5D3DFE6EDF3F8FD305E4F30504C75A7BB
:108DC100009006E0E0A3FCE0FBECA2E79217402054
:108DD10024FE50047F3B8022AE04AF037C007D144F
:108DE10012547C74542F2017029F9FFF7462800CD1
:108DF1001255F6EC24FE50E07F6D743D7E0012D4D6
:108E0100E17E017D197C03128E0C227F3D12DE6C06
:108E1100EF2DFFDCF822E537B40206E534243750A4
:108E2100292212DF2712D6B612CF93128FA312C8AE
:108E31006912CE00128FFB125B477F207E2B12D06E
:108E41007112D74812DC811238A812D1A9128ED121
:108E510012514502DD5120041EE579FD24A0500286
:108E61007D5FED24CD401E744520750C2DFFF5125C
:108E7100128EA61FBF44F922C39DFFF512128EA6C2
:108E81000FBF46F92220750EED2413FFF512128E45
:108E9100A60FBF78F922C374779DFFF512128EA633
:108EA1001FBF12F922EF24BA40082433FCC37432E5
:108EB1009C1404FC24D750047C238009EC2375F016
:108EC10005842413FC7E0512DE6C0EECB506F82237
:108ED100E59020E206E53424374003128E577F45A2
:108EE1007E047D1212DE6C0EDDFA7F437E00746417
:108EF10012D4E17F4F7D12128F8C7F3B7D12128F36
:108F01008C7F597D16128F8C7F317D16128F8C7F4D
:0F8F1100637D1A128F8C7F277D1A128F8C7F6DD4
:108F20007D1E128F8C7F1D7D1E128F8C7E057F19FA
:108F300012DE6C0FBF72F97804E57924CD50027807
:108F400009E8305C0123F87F1B128F7B7F6B128F47
:108F50007B18305C01187F25128F7B7F61128F7B1D
:108F600018305C01187F2F128F7B7F57128F7B1870
:108F7000305C01187F39128F7B7F4D7E00E875F0E1
:108F80000A847004E802D4CEE802D469EF65126066
:108F90000C7E04EE20E00712DE6C0EDDF62212DEFF
:108FA0009C80F790A5407F287E2C1277357E3B125F
:108FB000D32CAC5EAB7A7F307E19C23D12D36B905E
:108FC000A42F7F5D7E2D12773578B9C3E57A961888
:108FD000FBE55E96FC7F507E19D23D02D36BE51116
:108FE00064B4700122E51112DCF17831790F7D0B48
:108FF00012DDEF1F1E90908B02D53FE5716012E5E8
:109000007012DCF17831790F7D0412DDEB0DBD0AB1
:10901000F97F011290637F1D1290637E2312906D81
:109020007E3F12906D7E247F171290777E397F02EB
:109030001290777E247F071290817E397F1C1290D8
:10904000817E317F0212DE6C7F1C12DE6C7F0F7E10
:109050002412DE6C7E3E12DE6C7F0C7E2E90D834A5
:1090600002D53F7E2A12DE6C0EBE39F9227F08122D
:10907000DE6C0FBF17F9227D0612DE6C0E0FDDF9D4
:10908000227D0612DE6C0E1FDDF9220303E0A0E054
:1090900012CA1F7F18909D601277337F217E017462
:1090A0004112D4E17F2A7E01745312D4E19005BEAF
:1090B000E0F51AA3E0F519A3E0F51EA3E0F51D8580
:1090C0001A1C85191B751720129140E519251DF5ED
:1090D0001BF51DE51A351EF51CF51E751729129195
:1090E000409005BA129130AC1AAB19751720129046
:1090F000FE9005BC129130AC1EAB1D751729EC70AB
:1091000006EB24CD4001227A48305D027A271253C3
:1091100071125515ED4C600122AF177E07EB12D38B
:10912000C87E1A0F90A603305D0390A6060277351D
:10913000E0FEA3E0FD12BFD6C3EB9DF8EC9EF92242
:10914000751627025CAD12BFD675A7049005B478DA
:10915000737F06E6F008DFFBECF0EBF0E0E0E0FC0C
:10916000E0FDE0FEE0FFEF2DFFEE3C9005C0F0EFEC
:0B917000F0801275A7049005BAE0FB28
:10917B00E0CBF0EBF0E0E0E4F0F075A7002275A790
:10918B00049005B478647F06E0F608DFFB75A70052
:0E919B00125EBC9005BEE51CF0A3E51BF022A1
:10393A00D23C799E77008002C23C12BE80E4F51028
:10394A00F511F512F513F514F515F516F517C23D2F
:10395A00123C8A203D1F123C8A203D19E51F30E5A2
:10396A001130E40E1239B1303C08799EE724F55043
:10397A000122D510DBAE14AF157C00AD12125449EA
:10398A008F55AE16AF177C00AD1312546F125670D6
:10399A007E00E55530E7011E2DFFE43E30E7027F49
:1039AA0000740A2FF55622C235E51CAF1DBFFF056C
:1039BA000FD235F404FABF003F532CF8E518AF19BB
:1039CA00BFFF050FD262F404BF002D20E72A205B57
:1039DA000123FF24AA4021E51AAE1BBEFF050ED221
:1039EA0061F404BE00128547F0A4E5F020E709203F
:1039FA005B0123FE24AA5001227C807B8030516621
:103A0A00302163C006C0078AF0E545A4AEF0FFE5A1
:103A1A0056205B011375F009A4ACF0FD12546F74C3
:103A2A00FFBE0001EFFA24C050027A3FD007D00649
:103A3A00E55212DCF1303504B2D5B2D1EA8CF0A4E9
:103A4A0030E70205F0748025F020D10495F095F056
:0A3A5A00FCEA8BF0A430E70205F04F
:103A6400748025F030D50495F095F0FBC3EC2F203D
:103A74006203C39F9FFFEB2E306103C39E9EFE2013
:103A84003C64200C05123B1E4064123B00405F1254
:103A9400DE6CE51EFD24FB50550E12DE6CED24F6A3
:103AA400504C1E1F12DE6CED24F150421E0F12DE2C
:103AB4006CED24EC50380F12DE6CED24E7502F1F10
:103AC4001F0E0E12DE6CED24E250231E0F0F12DEC9
:103AD4006CED24DD50180E12DE6CED24D8500F1E50
:103AE4001E1F1F02DE6C123B004003799E0722E971
:103AF400242AFFE82461FE123B1E401DEF2460408F
:103B040018243F5013EE2460400F243F500AEF2442
:103B1400D6FFEE249FFEC322D322532CF8432C0459
:103B2400EE10E706D2E7F404D261FE24D340EAEFB4
:103B340010E706D2E7F404C262FF24D340DBEFB5FA
:103B440006005003CED26070057480FE8062FF24AC
:0D3B5400FD5060903C0A938EF0A4AAF0335F
:103B6100CA33CA33CA33CA33CA33FA903C34938F47
:103B7100F0A433C5F033CA903C5593FB123BD29568
:103B810070500224B412DCF1EA8BF0A430E7020594
:103B9100F0C3748095F020D50425F025F0FEEA8C61
:103BA100F0A430E70205F0C3748095F030D104250C
:103BB100F025F0FFC3227A01EE6F70097B16BF0278
:103BC100BB7A0380B7BF01047B0080B07B0D0A8004
:103BD100ABE52C540723C3903BDC73800E800E8031
:103BE10024801E8010800A80108012EB22742D9B8D
:103BF10022742D2B22745A9B22745A2B2274879B78
:103C01002274872B2274B39B22FFFFCCAA9280716E
:103C1100665D554E4944403C383533302E2C2A28B8
:103C2100272524232221201F1E1D1C1B1A1A1918A7
:103C31001817178181818282838384858687898A87
:103C41008B8D8F90929496989B9D9FA2A4A7A9ACCF
:103C5100AFB1B4B400010203040405060708090A60
:103C61000A0B0C0D0D0E0F0F10111112131314145A
:103C7100151516161612BDB812BC46E4F5F7C2B2F8
:103C8100C2B2E5F7D2B264C022203D07123C767081
:103C910003D23D22056D056D12BC467D008DF7C234
:103CA100B2C2B285F71F8DF7C2B2C3E5F79573F5BE
:103CB100188DF7C2B2C2B2E5F79574F5198DF7C246
:103CC100B2C2B2E5F78DF7C2B2C3E5F79576F51A40
:023CD1008DF76D
:103CD300C2B2C2B2E5F79577F51B8DF7C2B2C2B295
:103CE300E5F78DF7C2B2C2B2E5F7F51E8DF7C2B2A2
:103CF300C3E5F7957AF51C8DF7C2B2C2B2E5F78D2D
:103D0300F7C2B2C2B2E5F7D2B2543F30E50244C0C3
:103D1300955EF51D156D156DE51024784001227E25
:103D230000AF55EF30E7011E0512E51FA2E592D55E
:103D3300400EE515951EF515E5149400F514800B5A
:103D4300E515251EF515E43514F5147800E51E6018
:103D53000620D50318F404C39FF5F0E89E30E7016D
:103D6300220513E5F0A42517F517E5F03516F5162A
:103D730022303D03D23D22123C7660F8123C76603D
:103D8300F3E546600A123C7660EA123C7660E5058C
:103D93006D056D056D12BC467D008DF7C2B2C3E59E
:103DA300F79573F5188DF7C2B2C2B2E5F79574F5BE
:103DB300198DF7C2B2C2B2E5F78DF7C2B2C3E5F708
:103DC3009576F51A8DF7C2B2C2B2E5F79577F51B72
:103DD300D2B2156D156D156D2230742412BE80C2DA
:103DE3003D75101E123D74203D167902123E484067
:0A3DF3000CA806A907123AF34003DA
:103DFD0012DE6CD510E422200F4030123D2006CF8C
:103E0D00304806200C03204FC6E546790260147930
:103E1D000614600F791614600A79361460057976E8
:103E2D0014701712BE80C23D7896123D74203D0A63
:103E3D00123E48400312DE6CD8F022532CF8AB181A
:103E4D00E519FC339262123E9ABC002BEB89F053BC
:103E5D00F00784FF24DF401FAB1AE51BFC33926192
:103E6D00123E9AAA4712539ABC000CEB89F053F0FC
:103E7D000784FE24DF5002D32274562F2062029F46
:103E8D009FFF741F2E3061029E9EFEC322500312AF
:103E9D0055F6E920E40122C3EC13FCEB13FBE920FA
:103EAD00E50122C3EC13FCEB13FBE920E60122C371
:103EBD00EC13FCEB13FB2274542F2062029F9FFF27
:103ECD00741D2E3061029E9EFE2279B4203249204F
:103EDD001D46EFB506009260AC06AB074004AC077B
:103EED00AB06903F26EC2304938BF0A4A9F0EC23B2
:033EFD00938BF0B4
:103F0000A429F9903F8693C9904086E52C540793E5
:103F100013E95001F490408EF9E52C54079329756C
:103F2000F0B484A9F022FFFFFFFF7FFF55553FFF4C
:103F300033332AAA24921FFF1C711999174515556E
:103F400013B1124911110FFF0F0F0E380D790CCC60
:103F50000C300BA20B210AAA0A3D09D8097B0924BF
:103F600008D30888084207FF07C107870750071CC6
:103F700006EB06BC06900666063E061805F405D15B
:103F800005B005900572000000000001010101016B
:103F90000101010102020202020202020203030302
:103FA00003030303030304040404040404040405D6
:103FB00005050505050505050606060606060606A9
:103FC000060607070707070707070708080808087E
:103FD0000808080808090909090909090909090A55
:103FE0000A0A0A0A0A0A0A0A0A0B0B0B0B0B0B0B2A
:103FF0000B0B0B0C0C0C0C0C0C0C0C0C0C0C0D0D02
:104000000D0D0D0D0D0D0D0D0D0E0E0E0E0E0E0ED9
:104010000E0E0E0E0F0F0F0F0F0F0F0F0F0F0F0FB4
:10402000101010101010101010101010101111118D
:10403000111111111111111111111212121212126A
:104040001212121212121213131313131313131347
:104050001313131313131414141414141414141426
:104060001414141414151515151515151515151505
:1040700015151515151616161616161616161616E5
:1040800016161616161600FFFF00FF0000FF002E82
:10409000B5875B2D5A88E537607414603EB40258CA
:1040A0007F347E12E5342437400810644B90A3FF20
:1040B000801AF89041E012D53FE824FD501179A113
:1040C000E77E0590A23520E70390A23E0F803A24B8
:1040D000040F7E2312D500D26480627F357E02E514
:1040E000342437401410641090A11F30081B12773D
:1040F000027E1A90A3FE801122700590A1318009E2
:10410000909D8D200C03909D9812770280C97F3579
:10411000E5342433402A2404501B7D0F600C7D1E9F
:104120001460077D3C1460027D78ED305D02C3139E
:104130007E2B12D3C87E0090A13212770202DD518D
:104140007E0524FE5005909F758009909D70200F7C
:1041500003909D7C12770280E4E546604A14603C3F
:1041600014602E14602014601290A637205D4190D8
:1041700041D97F367E3412D53F803C90A637305DE2
:104180000390A633802A90A633305D0390A62F803B
:104190001F90A62F305D0390A62B801490A62B3085
:1041A0005D0390A627800990A623305D0390A61F8B
:0241B0007F3658
:1041B2007E331277357E3C7422305D02748302D5E1
:1041C20013305D0890A60F305BE4800690A617209E
:1041D2005BDC90A61380D70508B28D8DB5BA0910A5
:1041E20006000A10F248922492249224F2480A10FD
:1041F2000600305E5220434F20284CE55864FF6091
:1042020046E54824F640407F3FE55804F9C23D1296
:10421200424A1211AE601AB404047401D23D75F020
:1042220003A4243CB5070A7E3A303D027E36124290
:104232004C0F0F0FD9D7E55975F003A4243EFF1296
:10424200424A0F0F12424A227E3D12DE6C0EBE40DF
:10425200F922C248C249305E56202853E55864FF0D
:10426200604DE54824F640471211AE6042D249B48F
:104272000402803B1465597036D248304E31E559FC
:104282006558602B3074281242B7120E67E5BFB42E
:10429200011DE5BD20E618202416205F129006E4D9
:1042A200E0700CA3E024CE400624255002055922DA
:1042B200305FFC80E820113375A7009006E4E070BF
:1042C20028A3E0302402F404305F02F4042404F949
:1042D20024F74015E924FC4003D26C2270012230FD
:1042E2006C097536A7D22ED22FC26C22305E0830EE
:1042F2007405E558B4FF0122C244C24D780075A787
:0B4302000475830712463688188A1ED7
:10430D008E168F17C23EC23BE54824F6500302437A
:10431D00C7D23EE55860F7E8655970F22048EF12B4
:10432D00447C30D13BAE16AF17A818E54670551238
:10433D000920E5CC49604DD244E5CC7033E924CD5C
:10434D00402EE975F038A4ACF0FB12558512558559
:10435D00EBFDF5111243DD304D2CC206C23B8043FF
:10436D00E546705C120920E5CC7005E924CD50506E
:10437D00124F7C75A704758307A8181246368A1E3E
:10438D008E168F178037120E67E5BDA2E0B3923BF4
:10439D005011307428123AF34026A907A806D20608
:1043AD0012CAB01243F91243F01244398907880634
:1043BD001E1F90463112D53F800630D10312441195
:1043CD00A81808C3E55898400302430075A70022BA
:1043DD0074562F2062029F9FF9741F2E3061029E2A
:1043ED009EF822E51865586001227D057A00EA12D3
:1043FD00DCF112DDEF0A0AED24F240020A0AEA248A
:10440D004C50EB22AE16AF17123EC41E303E021EAC
:10441D001EE51E12D4E1EE2404FEE51212D4E130A5
:08442D003E09EE2404FEE51334
:1044350012D4E122E5186558603CC001C000C012E5
:10444500C0138518101245B4D013D012D000D00176
:10445500E510303B07C39570500224B412DCF120FF
:104465003B07AE16AF171243DDE5112402FD7A06B0
:1044750012DDEF1DDAFA221211AEB40457E87054BA
:10448500120E85E5BD604D78C6A61308A61208A6CE
:104495002C12C85D75A704758307751001125AC2E1
:1044A50012C8571510125AC21256DC8E628F63124B
:1044B50057648B1C8A1B12C86320320E1245642078
:1044C5003B08D24D1266FF1244DA78C68613088679
:1044D5001208862C22120E85AABD7C027BB31253CC
:1044E5009A8C128B13AA1DA91F1253DCA91CA81B99
:1044F5001255158C1D8B1FAC12AB13AA19A91A12D4
:1045050053DCA91CA81B1255158C198B1AE56E25B1
:104515001AF9E56D3519F8C3E56E951AFBE56D9544
:1045250019FAC3E554951FFDE56F951DFCE5542566
:104535001FFFE56F351DFEE52C23652C30E206ECEB
:10454500CEFCEDCFFD75A7049005C2E8F0E9F0ECCF
:07455500F0EDF0EAF0EBF0DD
:10455C00EEF0EFF075A70022D23BC3E5649573C56E
:10456C00659574F564E5669575600404600822E54C
:10457C006424E0500822E5642420400122C3E5674E
:10458C009576F567E5689577F566E5699578600940
:10459C0004600122E566F48002E5668562F0A4748D
:1045AC00E025F04002C23B2212C85D75A70475835A
:1045BC0007125AC212C8570510125AC2C02C125AEE
:1045CC00DBD02C891002C86330125120064E7800C3
:1045DC0075A70475830612463630D139123EC4E5F0
:1045EC004624FE500A0E0F90462C12D53F8026EA28
:1045FC007007745D12D4DD801C75F06484ADF070AE
:10460C000FED75F00A847008E5F00E12D4CE80051B
:10461C001EED12D46308C3E55A9850B475A7002256
:10462C00030340A040030340E040D2D1E8C4F5822C
:10463C00E0FA797312468F30D146AF06532CF8ED61
:10464C00BFFF07F40460390FD262BF00331247C3B7
:10465C00402E797612468F30D126E5822403F582DE
:10466C00E0F512E0F513EEA2E713FEED13BEFF0723
:0A467C00F404600C0ED261BE0006CB
:104686001247E0400122C2D122C3E09709FDE0971C
:1046960009FEE097600904700AEE30E7068007EE2F
:1046A60030E703C2D122E546600E14600BF9EDCE69
:1046B600A2E713CE13D9F8FD227C007B44E54660C1
:1046C600207C007BCC1460197C017B981460127CE2
:1046D600037B3014600B7C067B601460047C0C7BCF
:1046E600C08C148B157AE9125371A8471255138C96
:1046F600168B1775C70075C6047510DF75B901E509
:10470600BC20E76FF51385BD1205C605C675B90150
:10471600532CF8C3E5BE9573FBE5BF9574FC05C63F
:1047260075B901E5BC9575FD5005D2621255FEC3FB
:10473600E5159BE5149CE49D40338C198B18C3E565
:10474600BD9576FBE5BE9577FCE5BF9578FD5005F2
:10475600D2611255FEC3E5179BE5169CE49D400DFC
:104766008C1B8B1A12478AE5322428401305C6E5AE
:10477600C68006E5C62404F5C6700205C7D5100135
:0F47860022024702AE19AD181246ACED1247C31E
:10479500AE1BAD1A1246ACEE13ED131247E0123EF6
:1047A500C4E54624FB50080E0F90463102D53F1E46
:1047B500E51312D4E1EE2404FEE51202D4E175F00E
:1047C500067FFDA946B9000575F0027FFF84C5F097
:1047D5002F500205F0C5F0FF24DE228547F0A430F6
:1047E500E70205F0E5F0A946B9000280050475F079
:1047F5000384FE24E022E537B4020122E537700286
:10480500D23964027002C239E53724FC799EE7602B
:1048150005640B600C22D27E20081E401C107F1000
:1048250022D27F2008134011107E01227537012204
:104835007537002039037537022275F9FF75FB00BE
:10484500800E75F9FF75FBFF801C2053F512487D1E
:10485500759E85759D2D801412487D759E84759D68
:104865002D800912487D759E83759D09C2AC75988A
:1048750052C26DC26EC26F2212166EC253E4F5F9B2
:10488500F5FB30340215FB22D2A47F3212DE49C279
:10489500A412D9C812DD5112DE32C214C215124853
:1048A5003F74C012DC7C74A312DC39748F12DC39BE
:1048B5001248D374C012DC7C75A7049048DD7F10C4
:1048C500E49312DC39DFF91248D375A70022E538E5
:0548D50012DC3974CA79
:1048DA0002DC39A29494859C8080808080818380C8
:1048EA00819E8075A60A12489FD269D2ACE5A62499
:1048FA00FA500C306DF712DBCEB4E0F1124935C232
:10490A00ACC26975A6FF22D21EC274C273E4FDF559
:10491A0071F570C22D12483FD2AC12DBCEC5F070D1
:10492A0005DDF7C2AC22C5F0B4E0EFF538E4F532A4
:10493A0012DBC9A2E19273A2E2927475A7049004F1
:10494A00B4F012DBC9C2D1124B1C20690330740BBC
:10495A008D758E748F73E514C4F57D124B9C124BC2
:10496A001C20690330740C8D788E778F76E51425B8
:10497A007DF57D124B9CD2D1124B1CEEF0F55DEF0A
:10498A00F0F55C207303E4FEFF79BCA70609A707CC
:10499A0012DBC97D0A124B898F71EE60037571FFB4
:1049AA007D14124B89C22DED24F150010F240A50B7
:1049BA0002D22DBFB4027F008F7012DBC9F05407F8
:1049CA00C52E54F8252EF52EE571700EE4F571F515
:1049DA0070C22D9004BFF0F0F0F012DBC9E5386028
:1049EA0009D21EC27412AF158005C21E12AF11126F
:1049FA00DBC9B4E1FA75A7049004C412DBC9F0124A
:104A0A00DBC9F0F53A12DBC9F0F53B12DBC9F0F568
:0B4A1A003C12DBC9F0F53D12DBC9F0D7
:104A2500F53E12DBC9F0F53F12DBC912DBC9B4E272
:104A3500FA12DBC9F07E0C12DBC9FF12DBC912DBEF
:104A4500C912DBC912DBC920E1027F00EFF012DBDE
:104A5500C9DEE412DBC9B4E3FA12DBC9FF12DBC914
:104A6500CF60027F7F9004E4EFF0E4F012DBF99071
:104A750004D8124B8912DBC9B4EAFAC2AC75A70493
:104A85009004DAE561F0E560F0E55EF0E57AF0E5E1
:104A950079F0E52EF0E55FF0E57BF0E551F0207467
:104AA50012E4F571F5709004B4F09004BDF0F0F0E7
:104AB500F0F0F075A70078ABA63A08A63B08A63C2F
:104AC500120E7BE5BF253D240C75F0188478AEA643
:104AD500F0186005640260182216E670121816E6D2
:104AE5007004760C181678ACE6904B0F9308F622F6
:104AF5000618E608904B0F930466700D76011806AC
:104B0500E6640D70047601180622001F1D1F1E1F86
:104B15001E1F1F1E1F1E1F12DBC9FC12DBC9FD1243
:104B2500DBC9FE12DBC9FFECA2E692E7921713FC84
:084B3500ED92E713FDEE92E79B
:104B3D0013FEEF92E7301701F4F513ECA2E713FC27
:104B4D00ED92E713FDEE92E7301701F4F512ECA2AA
:104B5D00E713301701F4F510ED92E7301701F4F576
:104B6D00111255A620D10E8C1C8D1D8E1E8F1F125D
:104B7D00B31D1255A630170312B2F72212DBC9C3AB
:104B8D0013FEF012DBC992E7FFF07C0002547CACFF
:104B9D001CAD1DAE1EAF1F30170312B2F7ECF0EDBA
:104BAD00F0EEF0EFF022124BBC0202C612BC85C231
:104BBD00101248F07F5A7E0590A40E12770212DD76
:104BCD0051D214D215C255122CEC789F76800876EE
:104BDD000012BCC51232FA7570FE853A71853B72B2
:104BED00853C73853D74853E75853F7612BD2412D7
:104BFD0032FA7570C0757B03757A54E4F57FF57ED6
:104C0D0012BD24751421751348755F01757B0075F0
:104C1D00750475745275780175776CE4F57DF551F1
:104C2D00757F0190DF5C85836E85826DC23D124C70
:104C3D009A851C1D75A6FF305505C221022EA7129F
:104C4D004C9AE572A2E59275A2E79277D274D2736F
:104C5D00E51275F008A4AEF0FF2075031255E612AB
:104C6D00C7AD12C7F6124D1DE51C251D13F5718537
:054C7D001C1D12BC9D8E
:104C820012BCF5757F02E56A70B57F5A7E2FE54149
:104C920012D3C812DD5180A7856E83856D82C255FD
:104CA2007873124CFE7876124CFEE493F570B4B42D
:104CB20002D255A3E493F51CA3E493F512A3203D7D
:104CC2000FA97BE493F57BC399502A20E702055F85
:104CD200A385836E85826D103D16D23DE582240543
:104CE200F582E43583F583E493F52654F0F57222D8
:104CF200E526C480F630E7D8155F80D48601E493B8
:104D0200F6A308C399500A20E70606B60002080671
:104D12002230E70616B6FF0218162230750DE5138B
:104D22002579F513E43514F514800DC3E51395794F
:104D3200F513E5149400F514AE14AF137C007D0A4C
:104D420012547C8E5E8F7A22124DDF851617203D1B
:104D520001227F5A909C831276F07F64E5166404E8
:104D6200700C909C9B12773312DD5102DE2C909CCA
:104D72008F1276F07F6E7E0890A5FF127702121EC8
:104D82000312DD517515B87514047F6E7E20C2249E
:104D9200A815E82404F9C23DE7124E27203D06E695
:0A4DA20012D5138008E6128460E8C1
:104DAC00A815F60515EE2406FED514DA851716128D
:104DBC001E5112DD5110000510018D80F878B812CB
:104DCC000E8F86BC0886BD0886BE0886BF124EE6CE
:104DDC0012DF27120E8FC23D75160078B87F4B7EFE
:104DEC000890A5FF1277027E20E5BC12D513124E57
:104DFC001E7E26E5BD12D513124E1E7E2CE5BE126C
:104E0C00D513124E1E7E32E5BF12D513124E1E0262
:104E1C00DD51F608080808F618181824D050052497
:104E2C00F64001220516D23D2275C70375C6FE1247
:104E3C00766E124EE675C6FC75BC2675BD6475BEE5
:104E4C00A975BF70124EE675C6FB12766E124EE651
:104E5C0075C6FA75BC1475BD1475BE0075BF0C1201
:104E6C004EE675C6F975BC4E75BDBF75BE0075BFF7
:104E7C0019124EE675C6F875BC0A75BD7E75BE0076
:104E8C0075BF01124EE675C6F775BC0175BD23756D
:104E9C00BE4575BF67124EE675C6F675BC0275BD8C
:104EAC00AB75BE0175BF01124EE675C6F512766E76
:104EBC0075BE0275BF0A124EE675C6F412766E7593
:104ECC00BCE1124EE675C6F312766A124EE615C6B2
:104EDC00124EE615C6124EE615C675B90575B90221
:104EEC0022751500127D6775B901E5BC64816003FC
:104EFC001276510515E515242050E975C70375C6C2
:104F0C008075B90505C6E5C6241C50F5124F1E0266
:034F1C007BBDE476
:104F1F00F5C7F5C6742612766F75BD4E124F38124F
:104F2F004F35E4124F3512766F124EE605C6227FCB
:104F3F00357E00E54B12D47F7E10E54C12D47F7E78
:104F4F0020E54D12D47F7E30E54E12D47F227F466E
:104F5F007E00E56C12D47F7E10E56B12D47F7E202D
:104F6F00E56A12D47F7E30E57F12D47F2220740150
:104F7F0022D24475A700758307E559C454F024075E
:104F8F00F582E0F51A244C40E7A3E0F512A3E0F513
:104F9F00131209208938120E67E5BDA2E0923BE596
:104FAF001A40069570500224B4F51A203B05D2061C
:104FBF0012CAB0E51A1250DFE5152437F51DE43596
:104FCF0014F51CE5172437F51FE43516F51E85CCAF
:104FDF0012853813AC12AB137A0412536375380170
:104FEF0024FA401A05382402401405382401400ED3
:104FFF000538053824014006053805380538C3E55E
:10500F001A945A500224B4F51AC23BC23CC23D75E1
:10501F001B00A23B823C406D203B2CE51A75F0082B
:10502F00A4951BFBE5F0303D04940180029400FC35
:10503F005008EB24A0FBEC3405FC1250E6125095FF
:0A504F00923B40031250B8203C2CA5
:10505900E51A75F008A4251BF9E4303D010435F083
:10506900FAE994A0FBEA9405FC5004AB01AC0212E6
:1050790050E6125095923C40031250B8E51B253872
:10508900F51B5094203D04D23D808D22E51F251744
:10509900FEE51E35167016EE24914011E51D251505
:1050A900FFE51C35147006EF2491400122D3228EAE
:1050B900027C8A7B3B125371ED2402FE8F027C8AAB
:1050C9007B3B125371ED2439FF02DE6C1256CF80FF
:1050D900311256C2804675F008A4ACF0FB75190070
:1050E900C3EB9468F9EC9401FA40080519AC02ABDA
:1050F9000180ED8C108B11531903E51920E0CD12B5
:1051090056C212513AAF05E51924FE50031255E66D
:105119008E168F17E51920E0B81256CF12513AAF03
:1051290005E5191460061460031255E68E148F15EF
:1051390022AC06AB07AA12A9130253DC125227208C
:105149003D4974857F227E0812D5137E0830173CAD
:10515900AC1EAB1FEB2418EC34FC402F125342E574
:105169001B60077F207E0812D52E7F207E10E51A4E
:0951790012D52E7F237E17742E3F
:1051820012D50F7F207E1BE51B7011E519C2E012BC
:10519200D52E227F207E0E740A02D52EE51975F0D7
:1051A200058475F005A402D52E125227203D5E74A7
:1051B200857F227E3A12D513301753AC1EAB1FEBFC
:1051C2002418EC34FC4046EC7033EB249C402E7ED9
:1051D2002D125219125585C0E07F2A7E2EEB12D570
:1051E2002E7E39D0E0C2E012D52E7F347E3712DE19
:1051F2006C1E12DE6C1F12DE6C0E02DE6C7E301232
:105202005219125585EB7F2A7E3112CE52227F2A05
:105212007E39740A02D52E7F2912DE9C0FBF34F923
:105222000EBE40F322D23D301266120E71E5BDF57C
:105232001C75F00AA4F824E15002781EE4FCFBFE7F
:10524200FFC23D12BE80125293203D44D8F8751D14
:10525200CEE51C146009751D9C146003751D6AC29D
:1052620017EC30E705D2171255F68C018B00E9488E
:105272007003D23D22EE7008EF251D4003D23D227D
:10528200AC06AB077A1C1253711255158C1E8B1F7C
:1052920022203D07123C767003D23D22056D12BCDE
:1052A20046E4F5F7C2B2C2B2ADF7F5F7C2B2C2B286
:0252B200E5F71E
:1052B400FAD2B230E4E3ED2FFFE43EFEE56D2408BC
:1052C400F56D12BC46E4F5F7C2B2C2B2ADF7D2B284
:1052D400EA30E508EB2DFBEC3400FC22C3EB9DFB2C
:0552E400EC9400FC2227
:0100030055A7
:10DF5C0069FC362E06FD69FC372F071169FD383038
:10DF6C0007FD69FD3931061169FE383107FD68FE80
:10DF7C003732091168FF373008FD68FF372D07115C
:10DF8C006800362909FE680036290C116801372B08
:10DF9C000CFF6801372F0A116802383009FF68023C
:10DFAC00372E08116803372C0AFE6803372E081128
:10DFBC006704373208FE67043633091167053535B7
:10DFCC0005FF6705353303116706362F02FF670619
:10DFDC00362B05116707362B07FF6707352F051101
:10DFEC006708353104FF6708332E0511670931289E
:10DFFC000700670931250A11670A35240B01670AE6
:10E00C003A240A11660A3C210801660B3D1E0B11CD
:10E01C00660B3D1E0C00660B3D200A11660C3B2165
:10E02C000CFF660C39220E11660C37231100660D9D
:10E03C0036240D11660D34260F01660E3226111191
:10E04C00660E32251401660F35251311660F37271E
:10E05C0016016610392918116610392B1502651135
:10E06C00392D11116511372E0C026512332F081141
:10E07C006512312F07026513302C0A1165132D29F7
:10E08C000E0265132A271011651429270E02651438
:10E09C002C290C1165153129080365153726071134
:10E0AC006515321F09036516411B09116516411CC4
:10E0BC0008036416461F081164164D2105046416E6
:10E0CC005922031164166425040563156A2407118B
:10E0DC0063156D23090663156C230D1163156C25EF
:10E0EC00130762146E2B151162146E2F1406621333
:10E0FC006E30161162136E30150761136F311211E9
:10E10C0061126F350F0761126F380D116011723A81
:10E11C000A086011763F0611601079420209600FFF
:10E12C007A3A0533600F7832040A5F0F742C01338E
:10E13C005F0E722B030A5F0E732E08115F0E743084
:10E14C00050C5F0D722C02135E0D6C2B010C5E0D19
:10E15C00622C05315E0D5F2B030D5D0D5E290833BE
:10E16C005D0D5F23030B5D0D5F1B01335D0D5A16B7
:10E17C00020A5D0D521B00115C0D4D26000C5C0E4D
:10E18C00462802335C0E3926040C5C0F2C2B08330A
:10E19C005C0F23320C0F5D0F172E0A335D0F0C2E04
:10E1AC0009105D0F043507335E0FB23C080F5F0F8B
:10E1BC00AB4209335F0EA43E070F5F0EA2430B3335
:10E1CC00600EA746120B600D9F490C73610C9C49A5
:10E1DC000F0C610B97460973610B8B440A0C610A97
:10E1EC008B420B336109843A080C6108823A043380
:10E1FC0061087934030C60086F2F063360086228BD
:10E20C00050C6008572505336008511F040D5F0885
:10E21C004E1B05335F08491B090D5F094120103760
:10E22C005F0938270D0D5F0A302F06335F0B2B3239
:10E23C00070F5F0B282F0A335F0B262E0E0E600C78
:10E24C0023361137600D1F3F160F600D18411277E2
:10E25C00610D0F320A13610D042B0633610D022E72
:10E26C00040E620D043A0231620E0343050D630D78
:10E27C00B1470113630DA94A000B640CA14D0511A4
:10E28C00640C9B44070E650B99490911650A944768
:10E29C00090D65098E49021365088848060D650845
:10E2AC0081400E336407793B130F6407722F187784
:10E2BC0064076D231A106407692911776407651CBC
:0DE2CC00080F63075D180B33630751190D30
:10E2D9000D630746220E336308402B110F6308387C
:10E2E900291837630932271B0D6309312B1477620B
:10E2F9000A372C0F0A620A3C280973620A441E0B6A
:10E309000C620A48150E33620B46190C0A620B4758
:10E31900260D33610B4C280C0B610B54251037610A
:10E329000B5E24170C600B63291A77600A66361492
:10E339000A600A68390B735F0A6C2C100A5F09724C
:10E349002015775F097422120A5F0873300F775F0F
:10E35900087639140A5F077D3816775F0785370F06
:10E36900095F068D3B0D735F058B4410075F048BB6
:10E37900490C735F048E3F0C075F03863604335FD5
:10E389000394280708600299300E1160029E400527
:10E39900076102A34A0C336101AA4810086201B15E
:10E3A90042127762020131150A6202062B13776362
:10E3B900020830110C63020B361277630310331114
:10E3C9000C6403182B147764032223110A640426AE
:10E3D90023107764042226110A64051C2715776423
:10E3E900051D251508640521271277640628270FBE
:10E3F9000764062F1D11776406350F140764063E5E
:10E409000A19776406401216086407431B117763DB
:10E41900074A22120663075228127763075A2713FD
:10E429000662075E2314776206612011076206649B
:10E439001E0E7362066A1E0E076206742110376289
:10E44900057828130661057A2F157761047A332038
:10E459000661047A301B7761037A281B0761037F01
:10E4690023187761028429160661028832177761B9
:10E47900018D371305610193340C7362009A2E09DB
:10E489000562009D2E043362009D370C0663FFA0D0
:10E4990040103763FFA844140564FFAF4612776440
:10E4A900FF014511056500043F12776500053E101F
:10E4B900076600073F117766000B430D07670110D8
:10E4C9003D117367011539120767021A321277670E
:10E4D900021A2C12076702192C107768031B2E0FDA
:10E4E9000668031F2C117768042729100468042E75
:10E4F9002A0F776705322F130467053330127767C0
:10E5090006362D140567063B291677670643231B34
:10E51900046706471E16776607491E150366074CEA
:10E529001B157766074C2217046607522214776574
:10E53900075B26150265066229157765066D291799
:10E549000165067529137765057D281A0265058217
:10E5590028187765047F1F160265048F2A117765CD
:10E5690003953211006602993D157766029C401C9D
:10E57900FF6602A13E1F776701A43F1CFF6701A741
:10E589004314776801AB4710FF6901B1490F7769F7
:10E5990001024911026A0207490D736A020B480C0C
:10E5A900056B030F480B336B03144A0D026B0419F7
:10E5B9004914376B051F491CFE6C06224824776CE9
:10E5C90006233F21FC6C07203023776C0721272184
:10E5D900FC6C07262420776C08292812FC6C082873
:10E5E9002C0F776C0927230CFF6C09251802316C55
:10E5F90009350F05FC6C094C1401116C09561D01F4
:10E60900FC6B095F2003136B086B2108FB6B087413
:10E619002509336B08772507FC6B0778210D336BC8
:10E62900077A1E0AFB6B077F220C336B06832E0ABF
:10E63900FA6B05853C09336B0489410EF96B048C2F
:0DE649003E10376B038D3C0FFA6B038D40C4
:10E6560013776B02904112FA6C01934110776C01AB
:10E66600984410F86C009B471A776D009F461EF879
:10E676006DFFA24519776EFFA14019F86EFFA640FF
:10E6860014776FFEAA4417FA6FFEAF4A127770FE30
:10E69600B34D18FA70FF024B1B7771FF054718FD43
:10E6A60071FF0942177772000E4012FD7200163D87
:10E6B6000C7372011B3510FA7201232E1577720244
:10E6C60029321AF872032C371D7772032F3014F88B
:10E6D600720336210F77710346190DF87103502026
:10E6E6000B33710353290EF87003572B143770033D
:10E6F600612712F870036F2911777002793017F7C6
:10E706007001803722777001843D1FF67000883FC4
:10E71600197770FF8D3F11F670FF933D0C7371FEF4
:10E72600973D0EF571FE9B3E0C3372FD9F4310F62E
:10E7360072FDA448127773FDAB4C13F573FDB14F10
:10E74600167774FD034F14F775FE074C127775FEA6
:10E756000A4510F975FE0E400F7776FF124111F843
:10E7660076001745167776001C4614F67601214288
:10E7760017777602263D17F3760229382177760336
:10E786002A3315F276032B3009737604302A07F004
:10E79600760439220A337604472110F07504512590
:10E7A60012777504552416F1750459210F777504EF
:10E7B6005F2111F0740463231477740468240EF245
:10E7C600740370230933740379270AEF74028030C7
:10E7D6000B33740185360DEF74018B3913377400D2
:10E7E600903D1BF075FF94441E7775FF984823EF04
:10E7F60075FE9B46207776FE9F4221F076FEA13F6E
:10E80600177777FDA44313EF77FDA747157778FDB4
:10E81600AA4915EF78FDAD4C157779FDB04D19EE87
:10E826007AFDB34D1C777AFD024E19F07BFD054F3C
:10E836001B777BFE094F24F37CFE0D531D777CFF6F
:10E84600114619F37CFF173F12777C001F3810EF33
:10E856007C00263613777C012B3115ED7C012F2B9E
:10E8660015777C02332513ED7C02392214777C025E
:10E87600402110EE7C0249210B737B02531F0FEBE4
:10E886007B02601E15777B026A2214EA7B017428DC
:10E8960019777B017B2D1AEA7B00833122777B0077
:10E8A6008A3320EB7BFF91371A777BFE953C1FEA74
:10E8B6007CFE983C26777CFEA74621EC7CFD9939A8
:10E8C60023777CFC9A3B1FEA7DFC9A3F1C777DFBF5
:10E8D6009A401EE87DFB9B3F20777EFA9B3F1FE612
:10E8E6007EFA9C431A777EF99E4717E57FF8A04A81
:10E8F6000E737FF8A34A0AEA80F8A548073380F822
:10E90600A94402EA81F8AE46041182F8B24C00E747
:10E9160082F80351021183F8085304EA83F90E4D75
:10E92600061183F914430CEC84FA1A400E1184FB89
:10E93600203F0AE884FC2540061384FC2B4008E6A9
:10E9460084FD3039073383FD36300EE483FE3C2BDD
:10E95600193783FE402A1EE783FE3D25187783FE7E
:10E96600371B16E783FF3114137783FF35170FE440
:10E9760083FF3E220D738200412C15E58200432C55
:10E986001A77820046251BE782004C201577810006
:10E99600552116E581005E2510778100682718E469
:10E9A60081FF72291E7780FF7A2E22E580FE7E3057
:10E9B600277780FE812B22E680FD85251C7780FD4A
:0DE9C600882618E281FC8A2F187781FC8DCD
:10E9D3003821E181FB903F287781FA924025E0813D
:10E9E300FA943D237782F9973C18E082F99A3F1510
:10E9F3007782F89E4412E083F8A347107783F8A741
:10EA03004A0CDF84F8AA4D133785F7AC5214E2851C
:10EA1300F7AF56107786F7B2580DE087F802560223
:10EA23003387F8055002E388F8094C051188F90C7F
:10EA33004E02E489F91052011189FA155004DF8955
:10EA4300FB1D45041389FB233304DE89FB292306BD
:10EA53003389FC2B1F05DE89FC2F23093389FD3302
:10EA6300280ADC89FD3B23103788FD471E0EDD880D
:10EA7300FD511E0E3388FD53200CDD88FD54210B00
:10EA83003387FD57200DDD87FD5C20093387FD5D4E
:10EA93002403DE87FD5B29013386FD592C04DE86C2
:10EAA300FD5D2C093385FD622F0CDC85FD652D0B87
:10EAB3003385FC672908DF85FC6722093385FC6BF6
:10EAC300210CDD84FC72280A3384FB783005DD8455
:10EAD300FA7C37073384FA7E390ADC84F9813B06F2
:10EAE3003384F8843F05DB84F8873F023384F78A55
:10EAF3003C04DB84F78D390A3384F6903908D985D1
:10EB0300F5923F113785F595430FD985F498440A5B
:10EB13007386F49B440AD986F39C440C3386F39C96
:10EB23004507DA87F29C47063387F19E4C0AD9885A
:10EB3300F1A251103788F1A65516D989F0A7571FAE
:10EB4300778AF0A9541BDA8AF0AA4D12778BF0ACBE
:10EB5300460DDB8BF0AC4906338CEFAB4D05DB8CFC
:10EB6300EFA95002318DEEA85209E28DEEA7530EA4
:10EB7300118EEEA75316E58EEDA44A20118FEDA05A
:10EB83004423E28FEC9C4821118FEB9A4A22E090B8
:10EB9300EB95411D1190EA8E391DDF90EA893621EC
:10EBA3001190E9873223E590E9852C2C118FE87DBC
:10EBB3002A26E08FE8762124118FE8662122E08F50
:10EBC300E856221F118EE947201DE08EE9392116F0
:10EBD300118EE9302518E28EEA2D2917118EEB30BC
:10EBE3003213E18EEB333711118EEC373C10E18E8B
:10EBF300ED393E07138DED3B4203DD8DEE3B3E09C0
:10EC0300338DEE3B310DDE8DEE392812378DEF3823
:10EC13002319DC8DEF382A18778DF0372A12DC8D13
:10EC2300F0382214778DF0361B0EDC8DF1361B0C79
:10EC3300338CF1371F0DDB8CF136250E378CF23414
:10EC4300270CDC8CF22A270D338DF31F2A0CDC8D65
:10EC5300F3173409338DF4143A08E48EF4123A0CA2
:10EC6300338EF4103D11EA8FF50E411A778FF50CB0
:10EC73004917EA90F50A50157790F5054F13E79178
:10EC8300F5B24F107792F5AD5408E492F4AB5A0104
:10EC93003393F4AB5C05E893F4A9500A3394F3A4DB
:10ECA300450CE094F3A041093394F29A3A05E295B6
:10ECB300F29734043395F1913208DC95F19E310DCE
:10ECC3003395F08A320CDA95F0872D0B3395EF806C
:10ECD300250EDE94EF73220C3394EF6C2412DD9433
:10ECE300EF6928157794EE6B2812DF93EE69280EEF
:10ECF3007393EE64270DDF93EE5C260B3392EE578E
:10ED0300270EDB92EE5828123792EE5E2610DB9226
:10ED1300EE64240D7391EE6C2108D991ED722304F6
:10ED23003391ED782904D991EC7C320A3391EB7F4E
:10ED33003A08D891EB833D093391EA883C0CD7918B
:0DED4300E98D3B103791E9903E12D792E820
:10ED50009143137792E794420ED792E7993E073397
:10ED600093E7A03901D993E7A63B0A1194E6A83F9F
:10ED70000CD794E6AB490E1195E6AE4F07D695E653
:10ED8000004D011396E6034601D996E6033E0811AD
:10ED900097E7043D0ED997E70740151198E70C4314
:10EDA00012DA98E812460F1198E918490CDA98E936
:10EDB0001D44081198EA243D05D898EB293A03111F
:10EDC00098EB2C3707D898EC2D38093398ED2E3D69
:10EDD0000ADC98ED2E3E0A3398EE2D3F0BDB98EFC0
:10EDE0002C420C3398F02B430ED998F02B3D113761
:10EDF00098F12D3710D898F130340D7398F23433E0
:10EE00000FD698F237330F7798F339331CD597F331
:10EE10003C32167797F43E2F11D797F440280973A8
:10EE200097F4422109D797F4461F0AB396F44B2171
:10EE300008D796F45325083396F45C2505D796F445
:10EE40006723023395F4722503D695F3782B0231AC
:10EE500095F37B3102D695F27E31063395F1832FFF
:10EE600004D695F18A2F023395F0913201D596F0B0
:10EE70009638061196EF9A3F02D497EF9D450213FC
:10EE800097EE9F4704D497EEA247073398EEA64427
:10EE900008D398EEAA430B3399EEAD440CD499EE07
:10EEA000B1400D339AEE013F11D39AEE054512772A
:10EEB0009BEE064A15D59BEE064712779CEF05425E
:10EEC00012D79CEF063E0F779DEF084111D39DEFBF
:10EED000094619779EF00B4718D39EF00D431C7717
:10EEE0009FF10F4015D69FF1114113779FF2134602
:10EEF0000ED9A0F2174A0B33A0F31C4A08D4A0F491
:10EF000023420333A0F42A3305D3A0F53127071198
:10EF1000A0F5382300D29FF53D2702339FF6442900
:10EF200003D39FF64F2808119EF55E2807D19EF562
:10EF30006C2D04119EF4752F01D09EF47C2D0433AA
:10EF40009EF3822B04D09EF3872E05119EF28B3503
:10EF500007D09EF2903D01119FF1954203D09FF0A2
:10EF600094400333A0F09F3F0BD0A0F0A13D0F379A
:10EF7000A0EFA33C0DD1A1EFA43C0C33A1EFA43C26
:10EF80000AD0A1EEA53D0533A2EEA63C00D1A2EE2B
:10EF9000A8390211A3EEAA3C04D0A3EEAD3F05119F
:10EFA000A4EEB24008D0A4EE03410C11A5EE064138
:10EFB0000AD2A5EE08450711A6EF094A05D2A6EF29
:10EFC000094C0111A7EF0A4807D3A7F00B420B1118
:10EFD000A8F00B420DD4A8F00D461311A9F111466B
:10EFE00014D9A9F1173F1B11A9F21E381ADAA9F397
:10EFF00021381811A9F31F3A17DFA9F41839151190
:10F00000AAF4163A1DDCAAF5183C1A11AAF51C3A06
:10F010001AD9AAF61F391A11ABF6203615D9ABF753
:10F0200021341711ABF8203B19D9ABF81E3F17114B
:10F03000ACF91D4011D9ACF91E3F0E11ACFA1F40BE
:10F040000CD6ACFB22410D11ACFC23450FD6ADFC18
:10F0500023490B11ADFD214A0DD6ADFE2047091104
:10F06000ADFE21450CD6ADFF22430E11AE00224568
:10F070000CD8AE01214B0A11AE0220500DD7AF03C0
:10F080001D4F0B11AF031A5109D9AF04174A0D11C7
:10F09000B00418470BDBB0051A500A11B0061C5516
:10F0A0000ED7B1071C560B11B10719470ED9B1087D
:10F0B000173C0C11B208183D0CDCB2091C490E11AA
:0DF0C000B20A1E4E0AD9B30B1D500B11B33E
:10F0CD000C1A5109D9B30C174F0711B40D17490B71
:10F0DD00DBB40D17480D11B50E19490ADCB50F1922
:10F0ED004F0B11B50F185605DBB61017550711B696
:10F0FD0011174C0ADBB61116430B11B711173F0D43
:10F10D00DDB71219430C11B7131A480BDCB8131ADB
:10F11D00450F11B81419410DDCB81418400B11B975
:10F12D001518430DDBB91618470F11B91618490DEF
:10F13D00DBBA1718470A11BA1717450CDBBB1814A1
:10F14D00460F11BB18134C0EDBBC1912510A11BC22
:10F15D001A125007DBBC1A12470B11BD1A10400DC5
:10F16D00DCBD1B10400A11BE1B124509DCBE1C156F
:10F17D00490B11BE1D184A0ADBBF1D1B4A0811BFE2
:10F18D001E1B480CDBBF1F1A470E11BF1F1A490B60
:10F19D00DBC0201B4B0D11C0211C4910DBC0211DF4
:10F1AD00470F11C1221D4711DBC1231C4B0F11C18C
:10F1BD00231B4B0EDBC22419441111C224193D0F20
:10F1CD00DBC2251B3B1011C2261D3F0DDAC2261EC8
:10F1DD00411011C3271D3F12DAC3271C3D0F11C368
:10F1ED00281B3D10DBC4291C401111C4291C450FDF
:10F1FD00DCC42A1C460E11C42A1B4510DCC52B1974
:10F20D00431111C52C184511DDC62C164A1011C617
:10F21D002D174A11DEC62D18491211C72E19471088
:10F22D00DEC72F1A460E11C72F1C4410DFC7301F23
:10F23D00471111C731214B0CDBC832224D0E11C8BD
:10F24D0032224A10DAC83321471111C83420460F33
:10F25D00D9C83520461111C93521430CDBC93623D8
:10F26D003F0F11C937253D11DBC93725400E11C997
:10F27D0038254211DCC93925431311C939254312EB
:10F28D00DCC93A25431111CA3B24400DDCCA3C248C
:10F29D00411011CA3C23400EDCCA3D22401111CA57
:10F2AD003E20420FDECB3E20451011CB3F204714B0
:10F2BD00DECB4021441211CB40213F10DFCB412248
:10F2CD003C0D11CB42234011DFCC42233E1111CC1A
:10F2DD0043202F0EE0CC4319221211CC43122011E2
:10F2ED00E3CC4311250E11CD43132B10E3CD441266
:10F2FD002D1111CD440F2B0FE3CD44092B1211CE3F
:10F30D004404320FE2CE4401360E11CF44B3370D13
:10F31D00E0CF44B3330E11D04401370EE0D0440595
:10F32D003D0D11D0450A3B0CE3D14512330D11D1E2
:10F33D00451A2D0EE3D1461E2B0F11D1461D2E0F52
:10F34D00E4D1471D300F11D1471E320EE3D24821B3
:10F35D00330F11D248233510E2D24923350F11D284
:10F36D004A20360EE3D24A1D360E11D24B1B3410F5
:10F37D00E3D34B1B320F11D34B1B300EE4D34C1B7D
:10F38D00340D11D34C1B3A0DE5D44D1A3B0E11D44F
:10F39D004D1B360AE6D44E1D340E11D44E1E360DBD
:10F3AD00E5D44F1F360C11D5501F350EE5D5501F26
:10F3BD00340D11D5511E340EE5D5511E370C11D516
:10F3CD00521E390EE5D652203B0F11D653223C0F5B
:10F3DD00E4D65423391111D654243710E3D65524CD
:10F3ED00360F11D655253310E3D65626330D11D6CB
:10F3FD005627350BE2D657273A0C11D658273C0F16
:10F40D00E2D75827391011D75927370FE2D75A2786
:10F41D00381011D75A283B0FE2D75B293C1111D771
:10F42D005C2B3C12E2D75C2D391111D75D2C3910B4
:0DF43D00E3D75E2B3C0F11D75E293B0EE399
:10F44A00D75F27371011D75F26360EE3D760273CE0
:10F45A000E11D761284310E3D76229451111D762EB
:10F46A00293F0FE4D763283A1011D763293A11E4E8
:10F47A00D7642A3E1011D7652C4211E4D7662E4272
:10F48A001011D7662D3F11E4D7672F3A1011D768AC
:10F49A002D3B0CE4D7682E3D0711D7692E4204E4B0
:10F4AA00D76A2E470111D76B2E4702E4D76B2D403E
:10F4BA000513D76C2B3503E4D76C2A2B0711D76DAC
:10F4CA002B2909E5D76D2B300611D76E2A3A04E4A9
:10F4DA00D76F28400611D76F283E08E4D77027381F
:10F4EA000C11D87026320DE6D871252F0911D87162
:10F4FA0024310AE9D87221340811D8721B3A08EA71
:10F50A00D9730D420A11D973104909EADA730C4505
:10F51A000811DA730A3B06E8DB74093D0211DB7451
:10F52A000A4003E9DB740B3C0213DC75103406EA6B
:10F53A00DC7517350333DC761A3F06EADD771C469D
:10F54A000433DD771F4001E8DD7824360731DD78A2
:10F55A002C3206E7DC7933320413DC79373409E7D5
:10F56A00DC7A3A340C33DC7A3C3508E7DC7B3D370D
:10F57A000233DB7C3C3A05E7DB7C3C3D0333DB7D35
:10F58A003B3A04E7DB7D3B320331DA7D3E2D09EA63
:10F59A00DA7E43270D11DA7E4D230AE9DA7E5726F1
:10F5AA000B11D97D5E2C0BE9D97D61300C11D97D07
:10F5BA00632F08EAD87D662F0511D87C683005EAE2
:10F5CA00D87C6D330611D77B733608E9D77B7C3834
:10F5DA000511D77A853A04E8D8798B3B0711D8798F
:10F5EA008E3809E9D8788F371011D878903B0BE814
:10F5FA00D87791420D11D976954A08E7D976984974
:10F60A000411D9759D4008E8DA75A23A0B33DA7508
:10F61A00A53C0AE8DB75A8430031DB74AA4603E976
:10F62A00DC74AF460213DC74004A02EADD75054C4D
:10F63A000333DD75084D00EDDE75084B0533DF76C3
:10F64A00064902EDDF76044A0131E076044902EA0E
:10F65A00E076044C0513E176045006EAE176014DA2
:10F66A000D33E276B1450FEAE276AD3F1077E375E6
:10F67A00AB3F0DEAE375AC430A33E475AE4604EAE0
:10F68A00E475B0400131E575B23908EAE575013C27
:10F69A000611E675054607ECE6760A4B0311E7768E
:10F6AA000F4604EEE777163B0611E778203405EC9F
:10F6BA00E77827350611E7792D3409ECE7793234F2
:10F6CA000B11E77A3B260AECE67A45250B11E67A16
:10F6DA004D230BEAE67A56250711E67A5F270AEAEE
:10F6EA00E579672A0C11E579731F0AEBE578792E1B
:10F6FA000811E578843302EAE5778D3B0313E67651
:10F70A00954104EAE676993F0733E6759A3801EAA5
:10F71A00E67595310531E6748F3202EAE6748E3564
:10F72A000111E773923301EAE77398310413E77220
:0AF73A009D3304EBE872B4370911A7
:00000001FF
